:100000000000012065C300008DC300008FC3000005
:1000100091C3000093C3000095C3000000000000DE
:1000200000000000000000000000000097C3000076
:1000300099C30000000000009BC300009DC30000A6
:100040009FC300009FC3000039C800009FC3000089
:100050007D7900009FC300009FC300009FC3000084
:100060009FC300009FC300009FC300009FC3000008
:100070009FC300009FC300009FC300009FC30000F8
:100080009FC3000085CA00009FC300009FC30000FB
:100090009FC300009FC300009FC300009FC30000D8
:1000A0009FC300009FC300009FC300009FC30000C8
:1000B0009FC300009FC3000000000000000000007C
:1000C0009FC300009FC300009FC300009FC30000A8
:1000D0009FC300009FC300009FC3000000000000FA
:1000E0000000000000000000000000000000000010
:1000F0000000000000000000000000000000000000
:1001000000000000000000000000000000000000EF
:1001100000000000000000000000000000000000DF
:1004000010B5054C237833B9044B13B10448AFF34E
:1004100000800123237010BD88020020000000002E
:10042000B83E010008B5034B1BB103490348AFF3C5
:10043000008008BD000000008C020020B83E0100D2
:10044000154B002B08BF134B9D46A3F5803A0021A6
:100450008B460F461348144A121A0EF004FE0F4B37
:10046000002B00D098470E4B002B00D0984700205F
:10047000002104000D000D48002802D00C48AFF305
:1004800000800EF043FD200029000CF011FB0EF05F
:100490008BFB00BF000008000000012000000000EE
:1004A0000000000088020020540800200000000026
:1004B00000000000002070470020704700207047B7
:1004C000F0B5044685B00E46684611461F4606F054
:1004D000EBFE23686A465D6A31463B462046A847E4
:1004E00005B0F0BDF0B5044685B00E46104669462D
:1004F0001F4606F0E9FD23686A465D6A31463B46C1
:100500002046A84705B0F0BD70B590B00C46154622
:100510001E4603F0BFFD48B364B32146402268463F
:100520000FF061FD2F2168460FF0F4FC28B9234637
:1005300003224021684606F039FE402231466846D3
:100540000FF02BFD0C480AF099FE78B10B4B93F994
:100550000030062B0CD10A4B93F9003043B901232C
:100560002A46694604480BF0C0F8012010B070BD5F
:100570000020FBE72046F9E7BC030020B003002081
:100580008803002007B5002300931A461946034844
:100590000BF01EFD03B05DF804FB00BFA4020020B9
:1005A00007B5002300931A46194603480BF010FDC7
:1005B00003B05DF804FB00BFAC02002000207047D0
:1005C00013B5002204461146684602F077FB6068C6
:1005D00001F00EF902280CD005280AD0616800222B
:1005E000684602F0D5FE0021684602F0C7FD02B061
:1005F00010BD0020FBE7406808B510B1022101F0F2
:1006000005F908BD13B5002204461146684602F0FC
:1006100055FB2046FF22694602F02BFE204602B021
:1006200010BD000007B5002300931A461946034881
:100630000BF0CEFC03B05DF804FB00BFB402002059
:10064000704743683BB1B0F90A00012806D002DBCD
:100650000338012801D900207047022070470000AC
:100660002DE9FF4102AC84E8060006463C493D48BE
:100670009DF828501F460BF0EBFC204602F0DAFFF5
:10068000204602F06AFC40BB204602F073FE0528BB
:1006900004D8DFE800F01522160303160546324998
:1006A00030480BF0D5FC0A2229462E480BF039FDC4
:1006B0002C480BF0DDFC204602F0BCFF002009E0D6
:1006C000012533680095DD6B94E806003B46304613
:1006D000A847012004B0BDE8F0812046756802F00B
:1006E000B9FD0146284601F091F8204602F0B2FD1E
:1006F000012812D002282FD01C491A480BF0A8FC60
:10070000204602F0A7FD0A22014616480BF022FD02
:1007100014480BF0ADFC0125C1E70021204602F092
:100720007FFC18280DDC2821204602F0E9FC7168C6
:100730000022204603F0A0FA4FF42061706801F017
:1007400031FC336801250095D3F83C8094E806001D
:100750003B463046C047BCE700230393F1E700BFA8
:1007600088250100400300209E25010091250100FD
:1007700008B511B9B0F9080008BDB0F90A208A42DD
:1007800003DC0089084400B2F6E7406801F0B6F8DF
:10079000F9E7000007B5002300931A4619460348FD
:1007A0000BF016FC03B05DF804FB00BFBC02002098
:1007B00007B5002300931A46194603480BF008FCBE
:1007C00003B05DF804FB00BFC402002038B500236D
:1007D00083608380036804460D46002B47D0274A78
:1007E0001268002A43D0002908BF1D462B7C03F065
:1007F0000F03062B10D1224A224829460AF077FA25
:1008000008B143692371204A1E4829460AF06FFA4D
:1008100000282DD0436963711C4A216819480AF0E9
:1008200066FA054608BB1A491A480BF011FC0A2261
:10083000617918480BF08EFC174916480BF008FC3C
:100840000A22217913480BF085FC12480BF010FCAA
:100850002B460E4A21680B480AF084FA0B4A21689D
:1008600008480AF044FA054608B11435A56038BDB9
:1008700028680EF081F96071CEE700BF0C040020FB
:10088000E9380100540600200432010074260100FA
:100890007726010040030020022E010010B5044617
:1008A00001601146FFF792FF204610BD41790C4AC6
:1008B000002352F82300884203D10A4A52F8230049
:1008C000704752F8230028B942F82310054A42F82D
:1008D000230070470133052BEBD10020704700BF88
:1008E000D4020020E802002010B50A4A4079002313
:1008F00052F82340844203D1074A42F8231010BD26
:1009000052F8234014B952F82320F5E70133052BA0
:10091000EED1F4E7D4020020E8020020F0B52DED7E
:10092000028B9BB00546FFF7C1FF04460CF082F82E
:100930004FF0FF33014643F69822204606F0E0FCD4
:10094000002800F0D68006231622697905A80AF04F
:1009500091FF372105A80AF09DFF0022114605A846
:100960000BF0B2F8002108EE900A05A80BF044F94C
:10097000624908EE100A62480BF06AFB0A226979A4
:100980005F480BF0E7FB5F495D480BF061FB18EE39
:10099000900A0DF033FD022402460B46009458489D
:1009A0000BF09EFC584956480BF052FB18EE100A0B
:1009B0000DF024FD00940B46024651480BF090FCCC
:1009C00052494F480BF044FB4D480BF051FB504A45
:1009D000296850480AF08BF94F4A296807464D4864
:1009E0000AF085F90AAC064618EE901A204602F085
:1009F00072F994E80C004FF0FF31384606F09AFC8B
:100A000018EE101A204602F066F994E80C004FF038
:100A1000FF31304606F08EFC404A29683D480AF016
:100A200066F9064600285ED0037C03F00F03042B12
:100A300059D1F5EE408AF1EE10FA54D0B5EE408A65
:100A4000F1EE10FA4FD0F4EE688AF1EE10FA4AD1C6
:100A5000B4EE488AF1EE10FA45D100213C220BA8F1
:100A60000A910EF000FB7169402220460FF0BBFA9C
:100A70002F2120460FF04EFA28B973690322402136
:100A8000204606F093FB264920460FF034FA18EE74
:100A9000900A02A906F018FB22480AF0EFFB40B1C9
:100AA000214B93F9003023B902AA21461D480AF0D0
:100AB00007FE20460FF069FA1AAB1844482300F8E5
:100AC000413C02A918EE100A06F0FEFA15480AF099
:100AD000D5FB40B1144B93F9003023B902AA21464B
:100AE00010480AF0EDFD0BF0A5FF01462846FFF780
:100AF000FBFE1BB0BDEC028BF0BD00BF70260100F9
:100B0000400300207C2601008C2601009326010072
:100B100095260100540600209A2601009E26010019
:100B2000E9380100BC03002088030020F8B5044622
:100B300000680D461646002800F08880A06800284E
:100B400000F084800378FF2903F0100340D1002BCC
:100B50007BD0032A79D04578664967482D090BF088
:100B600077FA0A22294664480BF0F4FAA3685B7806
:100B700003F00F03AB4220D060495F480BF068FAE6
:100B80000A2261795C480BF0E5FA5D495A480BF09E
:100B90005FFAA368584859780A2201F00F010BF058
:100BA000D9FA584954480BF053FA0A2229465248B8
:100BB0000BF0D0FA50480BF05BFA0C2D40D8DFE870
:100BC00005F00B46377577375437797B657D7F00A5
:100BD000002BCBD0002039E0A3685B7803F00F0333
:100BE000023B082B24D8DFE803F00523232B230F37
:100BF00023231900444A216844480AF078F8A3687E
:100C0000197801F0010119E0414A21683F480AF0D2
:100C10006EF8A3681978C1F340010FE03D4A2168DE
:100C20003A480AF064F8A3681978C1F3800105E036
:100C30002168394A35480AF05AF80021002841D184
:100C4000A3685A7865F303025A700120F8BD334A4D
:100C500021682E480AF04BF8A2681378DF4303F0AE
:100C6000010167F300031370E8E72D4A2168274864
:100C70000AF03DF8A7683B7883F00202C2F3400215
:100C8000C3F3400162F341033B70D7E7254A216873
:100C90001E480AF02CF8A7683B7883F00402C2F3E0
:100CA0008002C3F3800162F38203EDE71E4AA2E7EC
:100CB0001E4AA0E71E4AA8E71E4AA6E71E4AAEE75C
:100CC0001E4AACE7A368032E5A780AD065F30302E4
:100CD0005A7006F059FCA3681A786FF304121A7060
:100CE000B3E7C2F3030161F307125A701A7842F0B6
:100CF0001002F4E7F825010040030020043201004F
:100D0000B838010010260100142601005406002006
:100D1000132601001A2601002126010026260100C3
:100D20002B26010031260100372601003C26010058
:100D300042260100482601004F26010055260100E9
:100D40002DE9F0435C4A95B00746884601685B4848
:100D500009F0CDFF5A4A39688146584809F0C7FF63
:100D60000646B9F1000F01D1002879D0554A3968FB
:100D7000524809F0BCFF544A396805464F4809F00B
:100D8000B6FF5249044652480BF062F90A227979BB
:100D90004F480BF0DFF94F494D480BF059F90A2243
:100DA00041464B480BF0BDF949480BF061F95EB381
:100DB000337C03F00F03042B26D14022716904A871
:100DC0000FF011F944480AF059FAE8B1434B93F98E
:100DD0000030CBB92F2104A80FF09CF828B9736913
:100DE0000322402104A806F0E1F9B8F1000F40D039
:100DF00025B12B7C03F00F03042B34D0384A012398
:100E000004A935480AF071FCB9F1000F28D099F80F
:100E1000103003F00F03042B22D1D9F8141004A8CA
:100E200000F0E6FE04A800F03FFEB0B1B8F1000FFC
:100E300033D025B12B7C03F00F03042B24D002AC5C
:100E400001220021204601F039FF0123009394E89C
:100E50000600002304A801F0FFF804A800F0BEFC7F
:100E600015B0BDE8F0836A691378002BCCD001235C
:100E7000C6E724B1237C03F00F03042B02D0012327
:100E8000184ABDE76269EFE769690B78002BE4D087
:100E9000002204A801F0A2FCDFE724B1237C03F0C8
:100EA0000F03042B02D002AC0222CAE761690B785F
:100EB000002BD2D04246ECE7642601005406002005
:100EC0009E26010026260100212601006926010038
:100ED0004003002091260100BC030020880300206D
:100EE000D12A0100D52A010070B598B0054602ACA0
:100EF00084E80600374838490BF0AAF80A226979D5
:100F000034480BF027F9354932480BF0A1F8204658
:100F100002F090FB2968324A324809F0E8FE94E872
:100F20000C004FF0FF3106F005FA29682E4A2D48D3
:100F300009F0DDFE29682D4A06462A4809F0D7FE49
:100F4000054660B3037C03F00F03042B27D14169EE
:100F5000402208A80FF047F82F2108A80EF0DAFF6A
:100F600028B96B690322402108A806F01FF9002365
:100F7000102200930DEB02014FF40073204602F0A3
:100F80005DFA1B480AF07AF948B11A4B93F9003020
:100F90002BB9012304AA08A915480AF0A6FBBEB183
:100FA000337C03F00F03042B12D1716908A800F001
:100FB0001FFE08A800F078FD38B10123009394E8E3
:100FC0000600002308A801F047F808A800F006FC76
:100FD00018B070BD4003002070260100912601006A
:100FE0006026010054060020642601009E260100B0
:100FF000BC0300208803002010B503788B42044610
:1010000004D14378402B01D1408810BD402321708A
:10101000637008460BF0C4FD80B26080F5E7000005
:10102000F8B5836804460D46002B00F051810A464E
:10103000FF21FFF77BFD637926790E3B072BC6F373
:1010400040062ED8A64A2168A64809F050FE074659
:1010500038B3037C03F00F03052B22D16179A2483A
:10106000FFF7CAFF0022064639469E4809F037FEC0
:1010700043699E421CDA0026A3685A7802F00F02E8
:10108000013A0B2A56D8DFE812F01E00E3004000B8
:101090006700E3006E00E3008C009C00A300CB001F
:1010A000DC0060790BF0ACFE311A4E424E41E3E7B2
:1010B000012239468B4809F012FE43699E42CCBF9B
:1010C00000260126D8E75F880BF0B4FC4FF6FF73CB
:1010D00081B24FF47A72384606F012F950B3834A5F
:1010E0002168804809F003FE28B12A4603212046E2
:1010F000FFF71CFD1EE07E4A21687A4809F0F7FDE3
:101100000028F2D12A460D21F1E75F880BF092FC0E
:101110004FF6FF734FF4967281B2384606F0F0F83E
:1011200040B12A4604212046FFF700FD0BF082FC67
:10113000A3685880A2681378C3F3C001B14200F0DD
:101140000F8113F0E00F00F09480C3F342110139D6
:1011500061F347131370BBE05F880BF06BFC4FF635
:10116000FF739622D8E75F880BF064FC4FF6FF739D
:1011700081B24FF47A72384606F0C2F80028D9D00E
:101180005C4A2168574809F0B2FD10B12A4608218F
:10119000ADE7594A2168534809F0A9FD0028F5D167
:1011A000B0E75F880BF046FC4FF6FF734FF4967282
:1011B00081B2384606F0A4F80028BBD02A4609219F
:1011C000B1E75F880BF036FC4FF6FF739622EFE72E
:1011D0005F880BF02FFC4FF6FF7381B24FF47A72E9
:1011E000384606F08DF80028A4D0444A21683D48CE
:1011F00009F07DFD10B12A460B2178E7404A2168AD
:10120000384809F074FD0028F5D13E4A2168354878
:1012100009F06DFD00287FF475AF2A46062166E7C8
:101220005F880BF007FC4FF6FF734FF4967281B2A4
:10123000384606F065F800283FF47CAF2A460C21BA
:1012400071E75F880BF0F6FB4FF6FF739622EEE72F
:101250005F880BF0EFFB4FF6FF7381B24FF416720D
:10126000384606F04DF800283FF464AF2A460021C6
:101270003DE70BF0DFFBA36858802279D2070BD53E
:1012800036B3197841F008011970204601F00101C8
:10129000BDE8F840FFF754BD31462046FFF750FD4A
:1012A000A3685B7803F00F0376B3072B0BD8DFE856
:1012B00003F0040A100A0A100A132A4601212046E4
:1012C000FFF734FC20B1A3681A7866F3C3021A70E2
:1012D000F8BD2A460621F2E72A460A21EFE700BFB9
:1012E0005C26010054060020FC0200203726010085
:1012F0003C26010042260100482601004F2601003D
:101300005526010031260100013B0C2BDBD801A240
:1013100052F823F049130000C71200004F130000D9
:101320004F130000C712000055130000C712000041
:101330005B1300005B1300005B1300005B130000F5
:101340005B1300004F1300002A460221B7E72A462C
:101350000521B4E72A460721B1E72A460021AEE776
:101360000321F5E62DE9F0470168634A86B081461E
:10137000624809F0BCFC99F8051006466048FFF782
:101380003BFE05B2002E69D0337C03F00F03052B22
:1013900064D13146594809F09AFC032853D90022F8
:1013A0003146564809F09BFC0122446953483146B6
:1013B00009F095FC0222D0F814A05048314609F0FB
:1013C0008EFC43694D480A270322314607FB03F888
:1013D00009F085FC43695F43214600974346524626
:1013E00028460BF054FA04463146444809F06FFC95
:1013F000052830D104223146404809F070FCB0F98C
:1014000014A03E48BC42C4BF3C4640F2FF353146C2
:101410004445BCBF4446002509F059FC022826D1AA
:1014200000223146354809F05AFC4369AB4251DC91
:1014300001223146314809F052FC4369AB4258DB86
:1014400006B0BDE8F08705EB850464004FF00008A6
:101450004FF42057C8E74FF0010AD2E705EB8504A7
:1014600064004FF000084FF420574FF0010AD9F8FC
:101470000830B3F902002A1A002AB8BF5242524576
:1014800007DC1A785109052907D8013161F34712A1
:1014900002E01A786FF347121A701B789F2B03D95A
:1014A000444501D0BC42CBD1A842C9D0002211464C
:1014B00004AE02A801F002FC224602A9304601F067
:1014C000F8FE96E806004846FFF70EFDD9F808300A
:1014D0005D80B5E70024D9F80830B3F90230A342A3
:1014E000AED021464846FFF72BFCD9F808305C8087
:1014F000A6E70124EFE700BF5C26010054060020A8
:10150000FC02002008B583680246F3B1012916D019
:101510000ADB032908DC0379402B0CD006D8032B07
:1015200002D81046FFF77CFD002010E0422B02D0CD
:10153000FAD3803BF3E71046FFF714FFF4E7037993
:10154000042BF1D1FFF7EAF9EEE74FF0FF3008BDC9
:101550007FB5037C03F00F03062B054623D101461C
:10156000124A134809F0C3FB90B1037C03F00F0348
:10157000052B0DD1C4680026ACB1294601A8019401
:10158000FFF724F9039B1E600BF090FA6468F3E701
:1015900004AC002144F80C5D2046FFF717F9022146
:1015A0002046FFF7AFFF04B070BD00BF602601000A
:1015B0005406002038B583680446BBB1124B1B6843
:1015C000A3B10068FFF7C4FFA36800251D6023795D
:1015D000032B0CD8012B94BF0221294660790BF014
:1015E000D5FBA3685A7865F303025A7038BD402BC7
:1015F00003D0422BFAD1294600E002216079BDE8F0
:1016000038400BF0C3BB00BF0C0400200023038054
:101610007047000013B5002423460094224621465B
:1016200003480AF0D5FC034B1C8002B010BD00BF7C
:10163000CC020020FC02002010B5044670B3204903
:101640000EF075FC58B31F4920460EF070FC40B3F5
:101650001D4920460EF06BFC28B31C4920460EF0B5
:1016600066FC10B31A4920460EF061FCF8B1194926
:1016700020460EF05CFCE0B1174920460EF057FC06
:10168000C8B1164920460EF052FCB0B114492046AC
:101690000EF04DFC002814BF00200E2010BD0120CC
:1016A000FCE70220FAE70520F8E70620F6E70A2023
:1016B000F4E70B20F2E70C20F0E70D20EEE700BF87
:1016C000CC260100E326010005270100F7260100D2
:1016D0000A27010000270100FB260100C3260100A4
:1016E000D326010010B50446002836D00378002B1D
:1016F00034D024490EF01BFC90B3234920460EF051
:1017000016FC78B3214920460EF011FC60B3204945
:1017100020460EF00CFC48B31E4920460EF007FC94
:1017200030B31D4920460EF002FC18B31B49204679
:101730000EF0FDFB00B31A4920460EF0F8FBE8B1AD
:10174000184920460EF0F3FBD0B1174920460EF0A1
:10175000EEFB002814BF00200C2010BD1846FCE74B
:101760000220FAE70120F8E70820F6E70520F4E771
:101770000620F2E70720F0E70920EEE70A20ECE771
:101780000B20EAE7EF260100CF2601000F2701001A
:10179000DB260100E7260100D7260100DF26010035
:1017A000EB26010014270100F326010010B50446C2
:1017B000406960B103689B69984718B16069036824
:1017C0005B69984760690368DB689847012010BD32
:1017D000406910B103685B691847704710B504464B
:1017E000406910B103685B689847204610BD00004F
:1017F00008B503220168044809F071FA08B1007DB8
:1018000008BDFF20FCE700BF5406002010B50322EE
:101810000C4601680B4809F062FA90B143690A4925
:1018200003F47F432343436108480AF011FC214637
:101830000A2206480AF08EFC0448BDE810400AF06F
:1018400017BC10BD540600204328010040030020AF
:1018500010B503220C460168044809F040FA20B193
:10186000406924F0FF04204000B210BD540600205F
:1018700010B503220C4601680B4809F030FA90B10C
:1018800043690A4904F47F421343436108480AF05C
:10189000DFFB21460A2206480AF043FC0448BDE863
:1018A00010400AF0E5BB10BD540600205728010087
:1018B0004003002010B503220C4601680C4809F0D3
:1018C0000EFA98B1E34363F47F4243690949134038
:1018D000436109480AF0BCFB21460A2206480AF087
:1018E00020FC0548BDE810400AF0C2BB10BD00BF97
:1018F00054060020842801004003002038B50C461F
:101900004168054609B9002038BD0B7C03F00F0380
:10191000022B03D1002CF6D14869F5E7052BF2D153
:10192000054809F0D4F98442EDDAE2B26968024868
:1019300009F0D5F94069E7E75406002008B5416889
:1019400069B10B7C03F00F03022B06D0052B06D1E7
:10195000044809F0BCF900B208BD0120FCE70020F2
:10196000FAE700BF5406002008B5816809B90020D5
:1019700008BD0B7C03F00F03022B01D14869F7E788
:10198000052BF4D10022034809F0A9F90028EED074
:101990004069EDE75406002008B5816809B90020C8
:1019A00008BD087C00F00F039A1E012A01D8000927
:1019B000F6E7052BF3D10022034809F090F900283F
:1019C000EDD0007CF3E700BF54060020826862B1CE
:1019D000137C03F00F03023B012B06D8516183688F
:1019E0001A7C022161F303021A747047826842B1C3
:1019F000137C03F00F00023801289CBF61F307132A
:101A00001374704708B5C16809B9002008BD0B7C84
:101A100003F00F03022B01D14869F7E7052BF4D13E
:101A20000022034809F05BF90028EED04069EDE799
:101A3000540600202DE9F041C36804460E46ABB9B8
:101A400001681648154F09F042F90546042D0DDCD2
:101A500000213846D4F8008009F078F94146024662
:101A6000E060384609F050F90135EFE7E3689BB1D3
:101A70001A7C02F00F02022A0ED15E610849094861
:101A80000AF0E6FA31460A2206480AF028FB054821
:101A9000BDE8F0410AF0ECBABDE8F0815406002040
:101AA0004B28010040030020006828B1007C00F0B2
:101AB0000F00431F5842584170470000F8B50446D4
:101AC000FFF7F2FF002831D021682A48294F09F09A
:101AD000FEF80546032D26680ADC0021384609F089
:101AE00035F931460246384609F00EF90135F1E77D
:101AF000002231461F4809F0F2F84369237401229D
:101B000021681C4809F0EBF802226060216819483E
:101B100009F0E5F80422A0602168164809F0DFF812
:101B2000237CE060032B02D00C2B19D0F8BD1020D1
:101B30000AF0D2FF104B03600546446000212046A6
:101B4000FFF7DCFE03B2002BB6BF40422B81288199
:101B50006868FFF7F3FE094B68812B606561E5E774
:101B600014200AF0B9FF064B44600360054604F0F8
:101B7000F9FCF3E754060020B8250100F034010019
:101B80008034010010B500230446016043610376F0
:101B90004362FFF793FF204610BD000070B5056853
:101BA00006462F2128460EF03FFA044698B100233E
:101BB00000F8013BFFF796FD0B4905460B480AF07C
:101BC00047FA0A22294609480AF0ABFA07480AF000
:101BD0004FFA284670BD2846FFF784FD05460028C9
:101BE000F7D03460F5E700BFA326010040030020D2
:101BF0002DE9F04389B0002400F118080546CDF81E
:101C000004804461047644620E4600293BD01F4B99
:101C10001F68002F37D02F2130460EF07BF9814608
:101C200050B3234602AAF05C19B238B12F2805D070
:101C3000142B02D0D0540133F5E7194608AB1944F0
:101C4000002301F8183C1248394609F050F80A22DE
:101C5000286009F1010140460EF0C5F901A8FFF71F
:101C60009DFF019B686203B92B762846FFF726FF8C
:101C7000284609B0BDE8F08332463946044809F0E9
:101C800036F82860F1E700232B60EEE7AC03002074
:101C90005406002018B1034903480AF0D9B9034992
:101CA000FAE700BFAF26010040030020B82601007C
:101CB00070B500229AB005460C4603A8114600F004
:101CC000FDFF0122294603A801F062FB4FF4407199
:101CD0002846FFF7BDFD00260443314610220AA81E
:101CE00009960DF0C0F9CDE90566E60518D503A8FB
:101CF00001F0B0FA172855D8012303FA00F041F695
:101D00004243184208D1984B0340002B4ED110F0AB
:101D1000240F47D0954900E0954905A80EF011F928
:101D200003A801F099FA082866D8012606FA00F0FF
:101D300010F4837F60D08F4809F0A0FA002800F0EB
:101D4000A3808D4B93F90030002B40F09D8003223F
:101D500030210EA805F02AFA2B682F2219680EA848
:101D60000EF01BF900964FF40073142209A903A882
:101D700001F064FBA0051CD4E1053DD5012305AAB3
:101D80000EA97C4809F0B1FC7C497D480AF060F955
:101D90000EA97B480AF065F97A4979480AF058F9A2
:101DA00005A923E0784976480AF052F924F48074B2
:101DB000B6E703A801F04EFA0228DDD003A801F02F
:101DC00049FA0528D8D0334609AA0EA9694809F06E
:101DD0008CFC6A496A480AF03BF90EA968480AF087
:101DE00040F9684966480AF033F909A964480AF0DD
:101DF00038F963480AF03CF9A2055CD500230322B8
:101E000030210EA805F0D2F92B682F2219680EA8F0
:101E10000EF0C3F85D490EA80EF06DF803A801F0AE
:101E20001BFA0438012836D8172203A907A801F0A5
:101E30009AFA002300934FF44073142209A903A8CF
:101E400001F0FCFA03A801F007FA51490EA80EF0C0
:101E500052F84A494A480AF0FBF80EA948480AF0E5
:101E600000F9484946480AF0F3F809A944480AF03D
:101E7000F8F843480AF0FCF83E4809F0FFF918B1B9
:101E80003D4B93F900305BB1284621B2FFF7F0FCDF
:101E900000201AB070BD002300934FF40073CCE70C
:101EA0000EA9012309AA334809F01FFC4FF4007161
:101EB0002846FFF7FFFCE3054DD503A801F0CAF95A
:101EC00001380B280BD8DFE800F04A0A0A0A0A4A50
:101ED0000A0A0A06484D2F4905A80EF032F80023D9
:101EE000032230210EA805F061F92B682F22196812
:101EF0000EA80EF052F825490EA80DF0FCFF264959
:101F00000EA80DF0F8FF1D491D480AF0A1F80EA912
:101F10001B480AF0A6F81B4919480AF099F805A9C8
:101F200017480AF09EF816480AF0A2F8114809F07E
:101F3000A5F90028A8D0104B93F90030002BA3D1AD
:101F40000EA9012305AA0B4809F0CFFB4FF48071BD
:101F50002846FFF7AFFC01209BE71049BCE72B7C2C
:101F6000052BBCD10E49B7E701008000E326010034
:101F7000CC260100BC030020880300203827010084
:101F800040030020102601002A270100022E010034
:101F9000EF2601000A270100CF26010000270100DB
:101FA000FB26010038B50B0505460C460CD405F0A0
:101FB00084F8952808D902F06DF828B12146284602
:101FC000BDE83840FFF774BE04F440712846FFF7BF
:101FD0004FFC034903480AF03BF84FF0FF3038BD8F
:101FE000192701004003002010B54FF4407104464A
:101FF000FFF72EFC014670B1074B93F90030062B1A
:1020000009D12046FFF7CEFF20464FF44071BDE8CE
:102010001040FFF74FBC10BDB0030020012970B580
:1020200005460C4601D1FFF7DFFF686950B1036830
:102030009B69984730B16869036821B29B68BDE825
:1020400070401847002070BD43691BB11A681846DC
:10205000526B1047007C70472DE9F04F8FB004AEF3
:10206000039304469DF860300293304686E80600EC
:1020700001F080F90746054602F00CF8039B834601
:102080001BB11A78002A40F05B83237E13B104F160
:1020900018030393002D40F05F83039B002B40F057
:1020A0005083676A002F00F05783304601F062F9D1
:1020B000002840F05183FAB231460CA801F05EF9D5
:1020C0004AE3304601F0B6FA2368002B00F0738330
:1020D000204600F023FD00288146A448D4BF4FF0DD
:1020E00000084FF0010809F0C3FF237C072B1AD02A
:1020F0000398FFF7A1FA82462046FFF779FB05B265
:102100000DB90FFA88F5BAF1000F0CD055450AD079
:102110009749964809F09CFF0A22294693480AF0FD
:1021200000F8924845E3002206AD1146284600F02B
:10213000C5FD00222146284601F02AF98246E0B971
:102140008C498A4809F084FF2046FFF77DFF294625
:1021500002B20CA800F0E2FD29460CA800F0F0FD48
:1021600021465246284601F087FD284601F062FAD2
:102170004FF420612046FFF715FF304601F06AF862
:10218000092800F25281DFE810F0B0005001500140
:102190001E000A00500150013B0062006200B9F1CC
:1021A000000FCCBF0222012229460CA801F0DBF867
:1021B000284601F04FF8314602460CA801F0D3F84A
:1021C0004FF0010806E1237C072B00F00381204635
:1021D000FFF70EFB0528804636D16749634809F0B2
:1021E00037FF0A224146614809F09BFF5F4809F02A
:1021F0003FFF237C052B0CBF0C2201222946DCE784
:10220000237C072B00F0E6802046FFF7F1FA062832
:1022100080460DD15949554809F01AFF0A22414616
:10222000524809F07EFF514809F022FF0222E5E7FB
:1022300053494E4809F00CFF0A2241464B4809F029
:1022400070FF4A4809F014FF6FF002064DE10CA838
:102250000022294601F087F8304600F083FEA8B935
:102260004FF0050A304600F0F5FF092804BFCAF117
:10227000000A0FFA8AFA0A2F00F2AC80DFE807F0B2
:102280000FAA11AAAAAAAAAAAA233000304600F0CF
:102290007CFE0FFA80FABAF1000FE1D0E2E74FF0CE
:1022A00001085146284600F0E7FD002800F0928022
:1022B00021460022284601F0DFFC4FF42061204631
:1022C000FFF770FE86E05146284600F014FE002815
:1022D00000F08080022229460CA801F04FF8E7E7C1
:1022E0005146284600F029FEF1E7304600F03AFE5C
:1022F000824600286ED00C2F6CD8DFE807F0076B01
:10230000346B6B6B6B6B6B867E8E6700B9F1000F65
:10231000304640F3F48100F038FE20B9022229460D
:102320000CA801F020F8284600F094FF0146204652
:10233000FFF76CFA4FF410612046FFF733FED046EA
:10234000284600F089FF04281CD1304600F084FFA5
:1023500002281CD1304600F07FFF294602460CA817
:1023600000F07DFF13E04FF0000AE9E74003002092
:10237000672701007D2701009A270100A927010096
:10238000BA270100284600F067FF0528DDD0237C2E
:10239000072B08D1304600F0ECFD20B1022229467F
:1023A0000CA800F05CFF2046FFF74EFE00B2009044
:1023B00096E80C0029460CA801F0B6F9BAF1000F16
:1023C0003FF476AF284601F07FFC71E796E8030002
:1023D00085E80300D4F814A0BAF1000F00F0CB8018
:1023E000304600F037FF092800F2AE80DFE800F049
:1023F0009EA983ACAC5F2BAC9E9E304600F03AFDAC
:10240000C1B2284600F0E0FC61E7304600F02BFD49
:102410000146284600F0BEFC59E7304600F009FDB1
:102420000146284600F0E1FC42E7304600F012FF8A
:10243000294602460CA800F096FFFAB229460CA8DD
:1024400000F09CFFBCE6B9F1000F2BDCAF49B048AF
:1024500009F0FEFD676908AE3B6830460122294657
:10246000D3F8288000F07FFF0123009396E8060050
:10247000039B3846C047062106462046FFF7C6F9AB
:102480004FF480712046FFF78DFDA249A04809F066
:10249000DFFD0A2231469E4809F043FE9C4809F0C0
:1024A000E7FD22E09C499A4809F0D2FDCCE6B9F15B
:1024B000000F1EDD67690AAE3B68304602222946DE
:1024C000D3F8288000F04FFF0123009396E8060020
:1024D000039B3846C047052106462046FFF796F97C
:1024E0004FF480712046FFF75DFD30460FB0BDE828
:1024F000F08F8A49D7E72046FFF77AF9052813D0ED
:1025000067690CAE3B68304602222946D3F8288022
:1025100000F029FF0123009396E80600039B38464C
:10252000C04702210646A8E77D49BCE76069036809
:10253000CDF800809C6A039B95E80600A0470646FC
:10254000A3E7B9F1000F13DC606901220368009270
:102550009E6A039B95E80600B0470646284600F0B1
:10256000FCFC002891D0284600F074FE014684E768
:102570004FF0FF3689E7237C062B5AD0072B42D039
:10258000052B4FD1022F00F09D800C2F4AD1204601
:10259000FFF738FA030C074605D1236861491A682A
:1025A000614809F08DF8284600F010FD0BF026FF79
:1025B0005E4B00220BF07AFF0CF028FA0FFA80FA3B
:1025C000082004F0F2FF6AF30F07804660F31F470C
:1025D00057494F4809F03CFD0A2251464C4809F042
:1025E000A0FD54494A4809F033FD1FFA88F10A2238
:1025F000474809F096FD464809F03AFD394620461D
:10260000FFF718FA0EE0029B63B16068037C03F0E9
:102610000F03052B06D1BBF1000F03D0039A3146FF
:1026200000F006FA284600F098FC002850D1012658
:102630005BE751462046FFF761F90FFA80F807463D
:10264000284600F007FEB8F1000FEBD0BCBFC7F181
:1026500000080FFA88F808F1FF339BB2B8BF4FF0BB
:10266000010A132BDED807B2012140460AF08EFB87
:10267000BAF1000F20D0012F1CD0063F18BF012750
:10268000394640460AF0AAFB2B49214809F0E0FCF4
:102690000A2241461E4809F044FD28491C4809F019
:1026A000D7FC0A2239461A4809F03BFD184809F0C0
:1026B000DFFCB7E70027E3E7012FE1D0BB1F5F4254
:1026C0005F41DDE752462146284601F0D5FAA9E7E9
:1026D000304600F0BFFD052801460BD1B9F1000FCF
:1026E000A5DD2046FFF792F84FF480712046FFF7F2
:1026F00059FC9CE7284600F0ADFD0146F1E700F0EB
:1027000044FC00283FF40FAE012208E6D227010066
:102710004003002011280100DF270100EF270100FE
:102720000128010022280100BC03002000005940BC
:1027300031280100352801001D28010091260100E3
:1027400057B91B78002B3FF4ACAC03A8FFF726FA6F
:10275000074600283FF4A5AC04F0AFFC1749054636
:10276000174809F075FC0A222946154809F0D9FCDA
:102770001449134809F06CFC23681148196809F0E2
:1027800070FC11490E4809F063FC03990C4809F0EC
:1027900068FC0E490A4809F05BFC0D49084809F03D
:1027A00057FCC72D3FF78DAC0A490B4809F050FC88
:1027B000094809F05DFC4FF0FF3696E63E27010020
:1027C00040030020432701004A2701005027010051
:1027D00056270100592701005C0300202DE9F0472E
:1027E0008EB00746CDE90221002900F01B810AB115
:1027F000137823B93B7E13B107F118030293029BB0
:102800005BB9D7F824800024039D2E5D7EB130464D
:102810000DF0AAFD28550134F6E71B78002BF0D007
:1028200002A8FFF7BBF980460028EAD0EBE728466C
:1028300000F012FA7C4905467C4809F009FC0A229E
:1028400029467A4809F06DFC04AC784809F010FC80
:10285000EAB23146204600F031FAB8F1050F21D036
:10286000B8F1060F08BF17255FFA88F60DF12809A1
:1028700032462146484600F081FD092D14DC082D22
:102880003DDAAA1C03DB6B1C40F3CC80B5B10123FD
:10289000009394E80600029B3846FFF7DDFB0EB07C
:1028A000BDE8F0871825DFE7172D00F08980182D87
:1028B000EDD100222146484600F055FD06AD03A9A2
:1028C000284604F0B0FB32462946484600F056FD43
:1028D000284600F0C1FC061C18BF01264FF0000A74
:1028E000039A0FFA8AF3A2B1BAF1030F10D003A82A
:1028F00004F078FB49F82A000AF1010AF0E703A87E
:1029000004F070FB21460246484600F0C6FCBEE7D4
:102910005346B8F10A0F0DD0B8F10B0F12D0B8F131
:10292000090F17D1284600F030FB81B2204600F095
:1029300031FAACE7284600F028FBC1B2204600F08F
:1029400043FAA4E7284600F020FB0146204600F0A9
:102950004CFA9CE733449BB2013B032B97D8DFE84A
:1029600003F00207122095E8030084E803008EE7D5
:10297000284600F00AFB9DF8283082B2214608A8BC
:1029800000F0BAFC83E7284600F0FFFA9DF82C20FF
:1029900000929DF8283082B2214608A800F095FCEC
:1029A00075E7284600F0F1FA9DF82C2000922146A8
:1029B00082B29DF8283008A800F087FC0C99C5E782
:1029C00000222146484600F0CEFC0025039A2BB297
:1029D00042B1042D0BD003A804F004FB49F82500F4
:1029E0000135F3E7032B11D0042B7FF450AF9DF892
:1029F000341001919DF8301000919DF82C309DF815
:102A00002820214608A800F09BFC40E79DF83010E4
:102A100000919DF82C309DF82820214608A800F050
:102A20007FFC34E700203AE73A2801004003002009
:102A30002DE9F0470E468CB0914600285FD0037C0C
:102A400003F00F03052B60D1314DC4682B78DFF8FC
:102A5000C4A0DFF8C48001332B70002C52D0237C3B
:102A600003F00F03042B38D16269DAF800104046F6
:102A700008F03DF9074680B3037C03F00F03052BF4
:102A80002BD1014602A8FFF77DF85EB102A8FFF73F
:102A90000BF838B100230093316872684B4602A8E6
:102AA000FFF7DAFA00223946404608F018F9B0B1CB
:102AB000037C03F00F03022B11D14369072B0ED1C6
:102AC00001223946404608F00AF94A463146FFF7E6
:102AD000AFFF76B102A8FEF781FE6468BDE7002E65
:102AE000F8D102A8FEF7E0FF0028F3D002A800F01A
:102AF00015F80028EED002A8FEF770FE01200CB0F9
:102B0000BDE8F0872B78013B2B700020F7E700BF72
:102B10003D030020AC0300205406002073B50022C2
:102B200005461146684600F0C9F82B683D4819680B
:102B300009F097FA2846FEF7B7FF58B93A493948DD
:102B400009F086FA374809F093FA4FF0FF3420462F
:102B500002B070BD2846FEF74BFE2B7C072B16D02B
:102B600001300D2813D8012606FA00F043F684043C
:102B7000044006D110F0490F09D02046FFF78AF82B
:102B8000E5E72A49274809F063FA3446DFE76A692E
:102B90003AB113681046DB6A9847041C18BF012439
:102BA000EBE72946684600F0F3FB2B7C033B062B42
:102BB0002FD8DFE803F02A152E2E042A15006B68A3
:102BC0001B7C03F00F03052B29D11949154809F087
:102BD0003FFA002211466868FFF72AFF0446CDE756
:102BE0000021684600F0CAFA044612490D4809F06F
:102BF0002FFA21460A220B4809F093FA094809F0F6
:102C000037FA003418BF0124A1E7684600F0BDF987
:102C1000EAE70949034809F01BFA002497E7002472
:102C2000E3E700BF4003002060280100AF26010059
:102C300069280100792801006F28010007B50023E9
:102C400000931A461946034809F0C2F903B05DF82B
:102C500004FB00BF00030020F8B50646F0B103787E
:102C6000E3B12D2B1ED0A3F13002092A1AD9252B4E
:102C70001AD07B2B1AD0232B1BD00F4F012404EB2F
:102C8000C4053D4428460DF080F9294602463046E9
:102C90000DF097F920B10134192CF0D14FF0FF3429
:102CA0002046F8BD0024FBE70824F9E76FF0010493
:102CB000F6E71724F4E700BF8D28010010B50023C4
:102CC0004370C370037143718371C37161F3071360
:102CD0008370027010BD10B5002307240370437089
:102CE000C37064F307138370416010BD89B20C296F
:102CF00010D8012000FA01F141F2592319420CD1F8
:102D000011F4A46F08D140F6060319420CBF00204D
:102D100002207047002070470820704738B50C46E5
:102D2000054611462046FFF7E1FFA37860F307133D
:102D3000A37023682B6063686B60284638BD000071
:102D40008B781B09013B082B1AD8DFE803F0160E1D
:102D50000E19191919050C000C4B4B600B68036018
:102D60004B68436070470A4BF7E764238B71CB795C
:102D700023F00103CB7100234B71FF230B71EDE7AF
:102D800000230B714B718B71CB71E7E70000A04101
:102D90000000964283781A0903D0022A05D0002049
:102DA0007047022262F30713837040F26D13994259
:102DB000A8BF1946C379817123F00103C1F3002133
:102DC0001943C1710120704783781A0903D0022A80
:102DD00005D000207047022262F307138370642934
:102DE000A8BF642141710120704713B564230446D4
:102DF0000093084600234FF4FA72992109F047FD29
:102E0000A3781A090ED0032A11D820EAE0706428AA
:102E1000E379A8BF6420013060F34703E371012028
:102E200002B010BD022262F30713A370EDE7002089
:102E3000F6E707B5C27912F0FE0F11D083781B09AF
:102E4000013B022B0CD850084FF4FA730093642214
:102E500099230021013809F01AFD03B05DF804FB45
:102E60004FF0FF30F9E7C379827903F0010342EABA
:102E7000032070474079704783781B09013B0A2B78
:102E800037D8DFE803F006063636362A1616160D52
:102E90000D000379194481F3080101710120704785
:102EA0004368194421EAE1716429A8BF64214160A3
:102EB000F4E7436807EE903AFDEEE77A17EE903AB2
:102EC000194421EAE1716429A8BF642107EE901A30
:102ED000F8EEE77A17EE901AE9E743680A2211FB49
:102EE000023121EAE171B1F57A7FA8BF4FF47A711E
:102EF000DDE70020704783781B09022B1BD1C279C4
:102F0000837902F0010243EA02231944B1F5B77F45
:102F10000FDA40F26D1331EA210128BF1946C37957
:102F2000817123F00103C1F300211943C171012014
:102F300070470021F3E70020704783781B09022BBC
:102F400009D14379194421EAE1716429A8BF6421B8
:102F5000417101207047002070470078003018BF91
:102F600001207047837813F0F00F14BF0120002078
:102F70007047807800F0E000202804D0A0F14003E2
:102F80005842584170470120704783781B09013B24
:102F90000A2B18D8DFE803F00808170606120A0AF9
:102FA0000A0606004068704700797047406807EEDF
:102FB000900AFDEEE77A17EE900A704740680A2300
:102FC00090FBF3F0704700207047000083781B09E6
:102FD000013B0A2B1ED8DFE803F013131D06060E73
:102FE000191919060600436807EE903AF8EEE77AD9
:102FF00017EE900A704743680A2293FBF2F3F3E757
:10300000037907EE903AF8EE677AF1E7436807EE46
:10301000903AEDE7DFED017AEAE700BF000000003B
:1030200083781B09013B07B50A2B5FD8DFE803F063
:1030300016165E5E5E44245E5E060600406839B188
:10304000D0F1640055D46428A8BF642001B201E027
:103050000028F8DA084603B05DF804FB007931B1C6
:10306000002100916423FF2209F011FCEEE76423A4
:103070000093FF220B46F7E7436807EE903A99B1B9
:103080009FED1E7A77EE677AF5EEC07AF1EE10FAD0
:103090002FD4F4EEC77AF1EE10FA2CDCFDEEE77ACD
:1030A00017EE903A19B2D5E7F5EEC07AF1EE10FAC4
:1030B000D0D49FED127AECE7406861B140F2F13371
:1030C000984216DC10F1090F15DB6FF0090390FB35
:1030D000F3F06430BAE710F1090FBBDB40F2F133D3
:1030E000984208DC0A2190FBF1F0AFE74FF0FF3186
:1030F000B0E70021AEE76421ACE700BF0000C842A2
:1031000013B504460846A3781B09013B0A2B32D8A5
:10311000DFE803F00F0F313131281A313106060094
:10312000FF23009300236422194609F0B0FB60607E
:1031300007E0FF23009300236422194609F0A7FB50
:103140002071012002B010BDFF23009300236422F0
:10315000194609F09CFB07EE900AF8EEE77A17EEA5
:10316000900AE4E740F6F613009300236422194620
:1031700009F08DFB60600020E4E7000083781B0904
:10318000013B0A2B5FD8DFE803F017175E5E5E464F
:103190001E5E5E060600406841B1002839DBFF284C
:1031A000A8BFFF20C0F1FF0001B20AE0002808DB41
:1031B000FF28A8BFFF20F7E700790029F4D0C0F16D
:1031C000FF01084670474368A9B107EE103AB5EE13
:1031D000C07AF1EE10FA1CD4DFED1D7AB4EEE77A76
:1031E000F1EE10FA32DC77EEC77AFDEEE77A17EEF1
:1031F000903A19B2E5E707EE903AF5EEC07AF1EEB3
:1032000010FADED49FED127AF4EEC77AF1EE10FADE
:10321000EBDDFF21D5E7406859B110F1090FF8DB6C
:10322000B0F5206F12DA6FF0090190FBF1F0FF307A
:10323000BAE710F1090FC4DBB0F5206FE9DA0A2113
:1032400090FBF1F0B0E74FF0FF31BAE70021B8E7AB
:1032500000007F43007870478078000970478B78C2
:1032600010B562F307138B700B6803604B68436003
:1032700010BD8B7810B51C09013C012C84BF0124C2
:1032800064F3071382F30802D2B288BF8B700B6815
:103290000A7103604B68436010BD8B784A6030B59B
:1032A0000A2565F307138B700B6803604B68436056
:1032B00030BD8B784A6030B5062565F307138B70F7
:1032C0000B6803604B68436030BD70B58C788A71C1
:1032D000022666F307148C70C2F30024CA794B717E
:1032E00022F001029DF810300B7122430B68CA7165
:1032F00003604B68436070BD70B58C788A7103269B
:1033000066F307148C70C2F30024CA794B7122F063
:10331000010222430B68CA7103604B68436070BDB1
:1033200070B58D784B71042666F307159DF8103043
:103330008D700B718A710B6803604B68436070BDC0
:1033400070B58D784B7105269DF810300B7166F3C2
:1033500007159DF814308D70CB718A710B6803606E
:103360004B68436070BD10B50A700B6803604B6812
:10337000436010BD807800F00F0070478B7810B567
:1033800062F303038B700B6803604B68436010BDEE
:103390002DE9F041044690460D4619B90026304605
:1033A000BDE8F0810846FEF77FFB06460028F5D011
:1033B0002846FEF7F1FA074680B12846FEF7D4FA10
:1033C000A378606067F30713A370B8F1000FE6D02D
:1033D0002846FEF70DFA46462070E0E7AA68137CFF
:1033E00003F00F03022B03D0032B09D00646D6E7C8
:1033F000A378526962600A2161F30713A370CEE7D4
:103400005369A27807EE903AF8EEE77A072117EEB3
:10341000903A61F30712A2706360C0E710B5002212
:103420000446027042708270C270027142718271F1
:10343000C271FFF7ADFF204610BD00002DE9F0433B
:103440002DED028B85B00446154698469DF83890C0
:103450000F4600293ED0002A00F0D28000230B70D6
:10346000017821B318F4807F21D0664B01EBC101B4
:10347000194438460CF0B7FD2A46634938460CF02B
:103480008CFD38460CF081FD2D1A3E18013D18F4D4
:10349000007F1FD0A3781B09013B0B2B1AD8DFE854
:1034A00003F00835669BA125707070221FA93E4667
:1034B000EDE72079B9F1000F06D0642300930023D3
:1034C000FF22194609F0E3F9504A034629463046DF
:1034D0000CF050FC384605B0BDEC028BBDE8F08323
:1034E00063684B4AF2E763684A4AEFE761680A2279
:1034F00091FBF2F302FB1312002AB8BF5242009272
:10350000454A294630460CF035FCE3E72046FFF7F4
:1035100090FCE279A37994F8058001B20029207922
:1035200002F0010202DBB9F1000F14D043EA0224D9
:10353000B9F1000F06D0642300930023FF2219463F
:1035400009F0A5F9CDE900802346344A29463046E2
:103550000CF010FCBEE7CDE90101CDF8008043EA94
:1035600002232F4A294630460CF004FCB2E7E379E7
:10357000A2796179009103F0010342EA0323294A09
:10358000BFE7636808EE103AB5EEC08AF1EE10FAB4
:103590004CBFF1EE487AF0EE487AFDEEE78AB8EEDD
:1035A000E87A77EEC77A9FED207A67EE877A17EE92
:1035B000900A09F0D9FC07EE900AB5EEC08AFDEE3C
:1035C000E77AF1EE10FACDED007A18EE903A01D5D7
:1035D000164A96E7164A94E72279A379019262790E
:1035E0000092B2E7E279A37902922279019262799C
:1035F0000092B6E72A46616830460CF0F4FC69E7B1
:10360000174667E78D280100B8380100DA29010064
:10361000DD290100E1290100E5290100EF29010070
:10362000EC290100F22901000000C842F82901003C
:10363000F929010030B58BB0134C002320220093F0
:1036400002A94FF440730546FFF7F8FE02A9204691
:1036500008F007FD0D49204608F0FAFCA9780A2277
:103660000909204608F076FD0949204608F0F0FCDB
:10367000A9780A2201F00F01204608F06BFD2046D0
:1036800008F0F6FC0BB030BD40030020C729010054
:10369000CC29010070B58B78B2EB131F86B00546BC
:1036A0000C46164606D123682B6063686B6028467B
:1036B00006B070BD1849194808F0CAFCA17817482F
:1036C0000A22090908F046FD1549144808F0C0FC13
:1036D0000A223146114808F03DFD12490F4808F012
:1036E000B7FC0023CDE9043366F3071322788DF885
:1036F00012304FF0FF338DF81020009302A863685A
:10370000226804A900F010F8029B2360039B636009
:103710002046FFF78FFFC6E7012A01004003002083
:1037200010260100B83801002DE9F04F8DB00C468D
:1037300004ADBDF958108046204685E80C00FFF71F
:10374000D5FA02902846FFF774FB011E02DB2046E3
:10375000FFF74BFB9DF81230A278C3F3030161F32E
:103760000302A270C2F303120B2A38D8DFE812F06A
:1037700098000C000C009C001401F0009800A700B9
:10378000A700A700980098001B095A1E0A2A6ED8A5
:10379000DFE802F0514317090638546D6D2F2F00F2
:1037A0009DF81720E2719DF81620A2719DF8152052
:1037B00062719DF814202271A27863F30712A2703F
:1037C0000DE0BDF81630C3F30802E379A27123F0CF
:1037D000010343EA1223E3719DF815306371029BE4
:1037E000002B00F0CF801A46214606A8FFF752FFB3
:1037F000C8E0059B002B36DBFF2BA8BFFF23DBB205
:103800002371ECE7059B13F1090F2CDBB3F5206F57
:103810002BDA0A2293FBF2F3F1E7BDF81630C3F37B
:103820000802E379A27123F0010343EA1223E37152
:103830009DF8153063719DF81430E1E7DDED057AF0
:10384000F5EEC07AF1EE10FA0DD49FEDBF7AF4EEEA
:10385000C77AF1EE10FA08DCFCEEE77ACDED037AD8
:103860009DF80C30CCE70023CAE7FF23C8E7B7492F
:10387000B74808F0EDFB9DF81210B5480A22090977
:1038800008F068FCB349B24808F0E2FBA178B04800
:103890000A22090908F05EFCAD4808F0E9FB9EE742
:1038A000059A62601B0987E700212846FFF766FC3E
:1038B0002071A378022262F30713A3708FE71B091C
:1038C0005A1E0A2AD3D8DFE802F011292F29290627
:1038D00023232318200005980AF07EFD00229E4B2A
:1038E0000AF00EFF0BF0DAF8606078E79DF814300C
:1038F00007EE903AF8EE677A03E0DDED057AF8EE30
:10390000E77A17EE903A636069E7DDED057AF1E753
:10391000A27863F30712A270059BF4E7A2780598DA
:1039200063F30712A270DFE700212046FFF726FCB1
:10393000BDF816302071C3F30802E379A27123F0B9
:10394000010343EA1223E3719DF815306371B0E778
:1039500001271B0903F10F0202F00F010A2986D883
:1039600001228A4040F265610A4217D1910735D49D
:1039700012F0180F3FF47BAF059A6260A27863F3F0
:103980000712A2702368C8F800306368C8F80430D2
:1039900040460DB0BDE8F08F0027DAE7013B0A2B67
:1039A00000F2C380DFE803F0B0C106C1C1B5BAC1FF
:1039B000C1B3B300FF23BDF816208DF81430642185
:1039C00061F30802ADF8162000228DF815209DF84D
:1039D0001220022161F307128DF812200023FF2527
:1039E0009DF8150000956422194608F050FF002844
:1039F000C0F29D8000239DF81500009564221946B1
:103A000008F045FFA84208DC002300959DF815004A
:103A10006422194608F03BFF05469DF81400FCF7A8
:103A20000FFE0646002F47D09DF817707F08013F14
:103A30003FB27B1C40F098807F2D4FF0FF0778DC71
:103A40000023C5F17F00194647F681627043009755
:103A500008F01DFF4FF4FF73009300231946E07137
:103A60007F22284608F013FF0023194600903A46AB
:103A7000304608F00CFF00970646642328467F2254
:103A8000002108F004FFBE420546A8BF3E46334968
:103A90002F4808F0DDFA0A2229462D4808F041FB9C
:103AA0002F492B4808F0D4FA0A223146284808F05A
:103AB00038FB274808F0DCFA00231A46194606A806
:103AC00008F047F9BDF816004FF6FF730093002386
:103AD000194640F26D12C0F3080008F0D8FEF2B2A9
:103AE000E9B280B208F04BF9030CA371030A6371C9
:103AF00020711C49164808F0ABFA2046FFF79AFDE2
:103B000006A808F0BBF86AE69DF8143053E7059B59
:103B100051E7059B0A2293FBF2F34CE7DDED057AB2
:103B2000FDEEE77A17EE903A45E7002343E70025DC
:103B300073E76423284600973A46802108F0A7FEE1
:103B400000230546E371A2E700007F436E290100D0
:103B500040030020102601000000244080290100BD
:103B60008D290100C02901004FF01E0B64231A4665
:103B7000CDF800B00021384608F089FE4FF0640906
:103B80005B468246CDF8009038464A46002108F050
:103B90007EFE7F2D83464FF0FF0754DCC5F17F008A
:103BA0000023704319462D4A00970BFB00F008F0E4
:103BB0006EFE4FF4FF73009300231946E071E32279
:103BC00005EB0A0008F063FE0023194603900090FD
:103BD0003A46304608F05BFE00230646009728462A
:103BE0007F22194608F053FEBE420546A8BF3E4656
:103BF0001B491C4808F02CFA0A225146194808F0C3
:103C00006EFA1949174808F023FA0A22594615484E
:103C100008F065FA1549134808F01AFA0A222946ED
:103C2000104808F07EFA12490E4808F011FA0A22EC
:103C300031460C4808F075FA0E490A4808F008FAAF
:103C40000A22039932E74B46284600973A468021DC
:103C500008F01DFE00230546E371C9E7646A3100E0
:103C60009B29010040030020A1290100A729010090
:103C7000AF290100B7290100F8B5054617460C46E3
:103C800011B900263046F8BD0846FDF70DFF06467F
:103C90000028F6D069682046FDF798FEA9782046EE
:103CA0000909FDF7A3FE1FB129782046FDF7AEFDF7
:103CB0000349044808F0CCF92846FFF7BBFCE1E7CC
:103CC000D32901004003002083781B09013B012B0D
:103CD00037B5054620D80023FF24007900946422DC
:103CE000194608F0D4FD002814DB0023287900943D
:103CF0006422194608F0CBFDA04207DC00230094A3
:103D000028796422194608F0C2FDC4B22C71012042
:103D100003B030BD0024F9E70020F9E707B5002320
:103D200000931A461946034808F052F903B05DF8AB
:103D300004FB00BF0803002002F0EAB902F0ACB9AE
:103D400007B5002300931A461946034808F040F9C6
:103D500003B05DF804FB00BF1003002070470000B3
:103D60002DE9F041044692B00D46474847491646B2
:103D700008F06EF92146444808F073F94449424876
:103D800008F066F965B10023AB5503F096F9F92800
:103D900009DC4049404808F05BF93F4808F068F901
:103DA00012B0BDE8F08104213C48DFF8DC8003F06C
:103DB00057F82F462E44BE4205D017F8011B404647
:103DC00008F053F9F7E7304808F052F9344B93F90B
:103DD0000030052B4FF0000314D10322412101A82C
:103DE00003F0E4F901A80CF0D0F806B2324601A9BC
:103DF00020460CF0E6F800B2B8B12A49224808F093
:103E000027F9CDE70222412101A803F0CFF901A84B
:103E10000CF0BBF806B2324601A920460CF0D1F8EE
:103E200000B210B100230122D8E734441E492046D5
:103E30000CF07DF840B928460CF0A7F8012803D90A
:103E4000284606F0FFFFABE72F2120460CF062F872
:103E5000064628B1002303704378242BA0D00136F6
:103E60002378242B9CD0214601A8FDF7C1FE01A890
:103E7000FDF71AFE20B13246294601A8FEF7AEFC36
:103E800001A8FDF7ABFC8BE740030020D92A010015
:103E9000DC2A0100DF2A01005C0300201C03002053
:103EA000B0030020EC2A0100F72A010038B5084DC4
:103EB00001244FF47A7008F0D7FD214601340A221C
:103EC0002846E4B208F046F9142CF2D138BD00BF00
:103ED0008C03002008B50449044808F0B9F8BDE88F
:103EE000084003F0FDB900BF342D01008C03002011
:103EF00010B586B00F4C10494FF0FF3203920F4AB5
:103F0000009200234C222046CDE90423CDE9013361
:103F100008F09EF80A4B0B4819686A4606F0B0FE96
:103F2000684606F0C3FA0849204608F091F806B042
:103F300010BD00BF8C030020AA2C010088390100AD
:103F40000C04002054060020C42C010010B50024ED
:103F5000214600220F48013406F01BFA4D2CF7D100
:103F60004C2246210B4806F014FA48224721094802
:103F700006F00FFA43224821064806F00AFA4921C2
:103F80004622044806F005FA03490448BDE81040FB
:103F900008F05EB818030020E72F01008C03002012
:103FA00030B52DED028B8DB0304B04930C4608EEEE
:103FB000102A00211C2205A80BF055F804AA08219C
:103FC000204602F0C7FF00238DF82130284B1B68E4
:103FD000002B47D0274808F04BF82749254808F020
:103FE00037F818EE100A0AF009FA02230246009385
:103FF00020480B4608F074F920491E4808F028F8BC
:1040000004A91C4808F02DF81D491A4808F020F8AA
:10401000184808F02DF81B4B1B48196804AA06F035
:1040200066FEDFED1A7AB4EE678AF1EE10FA054605
:1040300018D0DFED177AB4EE678AF1EE10FA11D0DE
:10404000B5EE408AF1EE10FA0CD002AC18EE101A60
:104050002046FEF740FE94E80C004FF0FF31284662
:1040600003F068F90DB0BDEC028B30BD4E494C0039
:104070000C040020400300203228010047320100D8
:104080001126010000040020540600200000FEC29A
:104090000000AA42034B93F90000053818BF012025
:1040A000704700BFB00300202DE9F04116491748C2
:1040B000174E184F154D07F0CBFF002406F10108ED
:1040C00016F8013F0F2B03D83946284607F0C9FFE1
:1040D000052C4FF010020DD03178284607F0FFFF75
:1040E0000D49284607F0B4FF0134E4B2062CE7D1AD
:1040F000BDE8F08198F80510284607F0F0FF284643
:1041000007F0B6FFF0E700BFD42C01008C030020BD
:10411000B00300206C390100232F010070B5184C4A
:1041200088B00DF11F030493631E0293A31E019335
:104130000D46E31E00930394231F621F1149686814
:104140000BF04CFE052809DC0F49104807F080FFF2
:1041500069680E4807F085FF08B070BDFFF7A4FF3F
:104160000B4E0025053C625D29463046013506F0C0
:1041700010F9062DF7D10749074807F069FFEBE76B
:10418000B6030020462D01005A2D01005C030020DB
:10419000180300206C2D01008C03002008B508B91D
:1041A000002008BD037C03F00F03052BF8D1CAB231
:1041B0000146064806F093FD0028F1D0037C03F089
:1041C0000F03042BECD14069EBE700BF540600203D
:1041D0002DE9F0430024C9B03C22214609A80894E7
:1041E0000AF041FF7C22214629A828940AF03BFFCF
:1041F00023460122402108A802F0D8FF7F49804EC3
:10420000804D08A80BF077FE80227F4928A80BF08C
:10421000EAFE012328AA08A97C4807F066FA23468B
:104220000122402108A802F0C1FF794908A80BF03B
:1042300062FE8022774928A80BF0D5FE764928A88F
:104240000BF059FE012328AA08A9704807F04DFA7F
:1042500023460122402108A802F0A8FF6F4908A8C0
:104260000BF049FE80226E4928A80BF0BCFE01230A
:1042700028AA08A9654807F038FA234601224021F8
:1042800008A802F093FF674908A80BF034FE8022CB
:10429000654928A80BF0A7FE28AA012308A95B48B6
:1042A00007F023FA32782F6801323270002F00F0C5
:1042B0009E805E4BDFF8A091B3F80080ADF80080DF
:1042C00021461E220DF102000AF0CDFE21463E22BB
:1042D0000DF16200ADF860800AF0C5FEDFF87C8168
:1042E000FC68534F2A68002A77D0002C75D0237CB5
:1042F00003F00F03052BF6D12146384606F0E7FC04
:104300000028EFD000222146384606F0E8FC436939
:10431000092B0ED8DFE803F059515159590546468B
:1043200059592022434968460BF05DFE00238DF861
:10433000603000230122402108A802F037FF40220C
:10434000216808A80BF029FE3B4908A80BF0D3FD13
:104350003A4908A80BF0CFFD01236A4608A92B486B
:1043600007F0C3F99DF86030C3B10023012240215A
:1043700008A802F01BFF4022216808A80BF00DFEE0
:104380002D4908A80BF0B7FD2D4908A80BF0B3FD87
:10439000012318AA08A91D4807F0A7F908F086FB11
:1043A00064689FE72022274968460BF01CFE2649D7
:1043B000402218A80BF017FEBBE7202223496846CD
:1043C0000BF011FE40222249F3E7202241466846C5
:1043D0000BF009FE40224946EBE740210023012271
:1043E00008A802F0E3FE1B4908A80BF084FD33780F
:1043F000013B337049B0BDE8F08300BFDE330100FC
:104400003D030020AC030020D8330100BC03002092
:10441000B83301000E340100FB330100E533010025
:1044200052330100CA3301004C3301000D2A010050
:1044300054060020C4330100022E0100393301006C
:10444000EC330100B333010074330100BE330100CB
:10445000A7330100D133010062330100AB33010007
:1044600010B5114C1149204607F0F2FD10492046C5
:1044700007F0F7FD4FF4FA7008F0F6FA0121152065
:1044800008F084FC0021152008F0A8FC4FF4FA7015
:1044900008F0EAFA1520012108F0A0FC4FF4FA70A8
:1044A000BDE8104008F0E0BA8C030020163301008C
:1044B0003633010013B50E4C0E490F4807F0C8FD06
:1044C0002146684603F0DBFF684602F049FE2146BC
:1044D000684603F0ECFF684602F042FE214668465B
:1044E00003F0D9FF684602F03BFE02B010BD00BFEA
:1044F000E4050020FF2E01008C03002070B588B079
:104500002F231522002102A801930AF0ACFD1649C1
:104510001648174D174C07F09BFD0DF105020621BB
:10452000154802F017FD002614498DF8116001A806
:104530000BF0E1FC01A9284607F093FD01A92046F4
:1045400007F01CF90E498DF8116001A80BF0D3FC9F
:1045500001A9284607F085FD0A4A01A9204607F06F
:10456000AFF8012008B070BD752D01008C0300204C
:1045700040030020BC030020B10300208A2D01006D
:10458000922D0100C2380100FFF7B8BF18B10349EE
:10459000034807F05DBD0349FAE700BF143301008B
:1045A0008C030020B33E010010B5224C2249204666
:1045B00007F04EFD2149204607F04AFD204B1868C0
:1045C000003018BF0120FFF7E1FF1E49204607F029
:1045D0003FFD1D4B1868003018BF0120FFF7D6FFC4
:1045E0001A49204607F034FD194B1868003018BFEF
:1045F0000120FFF7CBFF1749204607F029FD164B96
:104600001868003018BF0120FFF7C0FF204607F0F0
:104610002FFD1249204607F01BFD02F04EFD0A2235
:104620000146204607F089FD2046BDE8104007F00E
:104630001FBD00BF8C030020922E01009F2E0100A1
:10464000AC030020A72E0100A8030020B02E01001B
:10465000B8030020B72E0100000400203E2701000F
:104660002DE9F843074608460E460BF08EFC04B2CF
:104670001F2CDFF83080A8BF1F243546A7EB0609A2
:10468000AB1B9C4207DD09EB0501404615F8012BE9
:1046900005F07FFEF4E7E11900220248BDE8F84387
:1046A00005F077BE1803002007B500238DF804300D
:1046B00050B149683620FFF7D3FF0449044807F09A
:1046C000C7FC03B05DF804FB01A9F3E7172B010059
:1046D0008C0300202DE9F04780460F460146114823
:1046E000164605F054FE0138C0B2FD2818D8DFF890
:1046F00034A00024013E25B208EB0401B54209B202
:1047000007EB050906DA504605F041FE01347855FD
:104710000028F0D1002389F800300120BDE8F0879F
:104720000020FBE7180300202DE9F04FA7B000237D
:1047300095488DF81330CDE90533CDE9073306F000
:104740009DFD924F054610B105233B70FAE0904C59
:10475000216809B90E23F8E78E4806F0B8FA0FFA77
:1047600080F8B8F1010F0646F4DD294620688A4D2D
:10477000FFF714FD89492860894807F069FC29681A
:10478000874807F06EFC864807F072FC854986482A
:1047900007F05EFC0A223146834807F0C2FC8248DB
:1047A00007F066FC01212068FFF7F8FCB8F1020F62
:1047B000824600F0CA8002222168764806F08FFA0D
:1047C000B8F1030FD0F8149000F0C18003212068E5
:1047D000FFF7E4FC0646102205A93620FFF77AFF12
:1047E000002840F0B780B8F1040F40F3B3800421F3
:1047F0002068FFF7D3FC6D490446694807F028FCA0
:10480000674807F035FC1FFA89F251465E4806F00A
:10481000E7FF0DF1240866495B4806F0E4FF0DF15F
:10482000340B1022634940460BF0DDFB00230122CC
:104830002021584602F0BAFC5F4958460BF05BFB5A
:104840005E49574807F004FC5146554807F009FCFB
:104850005B49534807F0FCFB0A224946504807F0E1
:1048600060FC58494E4807F0F3FB31464C4807F0CE
:10487000F8FB55494A4807F0EBFB33780BB91C4667
:104880001E46CDF80C804FF002094FF00108CDE92B
:104890000198CDF800B03246234629683A484B4E7D
:1048A00006F002FE002857D0494B4A493C480024F4
:1048B0001C6007F0CDFB2968394807F0D2FB384867
:1048C00007F0D6FB444B032283F8008041212346A6
:1048D00015A802F06BFC414915A80BF00CFB15A9BB
:1048E000294806F04BFF23464A46412115A802F00D
:1048F0005DFC3B4915A80BF0FEFA15A9394807F0F5
:10490000C7FB15A9204806F039FF2346424641213E
:1049100015A802F04BFC324915A80BF0ECFA15A9CA
:10492000304807F0B5FB15A9174806F027FFFFF739
:104930004FFC05233B7008F07DF82B493060184888
:1049400007F086FB27B0BDE8F08F40F25B790DF1F0
:10495000130640E705AC56E72449254807F078FBE5
:10496000094806F042FF0A220146214807F0D9FB18
:1049700020491F4807F06CFB1D4807F079FB08F041
:1049800059F80C233060E0E6BC030020B00300209F
:10499000B803002054060020580300209E31010077
:1049A0008C0300207126010040030020AB31010080
:1049B000613D000095330100DE330100CB31010081
:1049C000232F0100EB310100D9320100180400202F
:1049D000FC030020F23101003E0300200032010000
:1049E00004320100B006002006320100233201002B
:1049F0005C0300202F320100F8B5074E07460D1D5D
:104A00000024E11915F8012B09B23046013405F0F4
:104A1000C0FC042CF5D1F8BD1803002030B587B0D8
:104A20000023044600931A460D4602A8194607F0D3
:104A3000CFFA04A807F0C4FA042C12DD04A92869EF
:104A400002F043FB68B104A91220FFF7D5FF04A9C7
:104A5000E86802F03AFB50B104A90E20FFF7CCFF42
:104A60000BE002A91220FFF7C7FF032CEFDC02A91D
:104A70000E20FFF7C1FF022C17DD04A9A86802F081
:104A800024FB90B104A90A20FFF7B6FF04A96868C7
:104A900002F01BFB78B104A90620FFF7ADFF0D491A
:104AA0000D4807F0D5FA07B030BD02A90A20FFF77C
:104AB000A3FF012CEADC02A90620FFF79DFF012CD1
:104AC000EDD102A90620FFF797FF0449024807F03D
:104AD000BFFAE4E7102B01008C030020002B01003B
:104AE0002DE9F041104F80460C460E1D002508EBC5
:104AF000050109B2384605F04AFC0135042D06F8D7
:104B0000010BF4D1207958B1FF280BD16379FF2B29
:104B100008D1A379FF2B05D1E079FF3818BF012018
:104B2000BDE8F0810120FBE718030020F0B593B049
:104B300002A807F045FA04A807F042FA06A807F011
:104B40003FFA08A807F03CFA58495948594E07F06F
:104B50007FFA574807F08CFA02A90620FFF7C0FF3A
:104B600000287CD054495248544C10AD07F070FADC
:104B7000039B10942846119302F0F2FA04A90A202C
:104B8000FFF7AEFF002861D04D49494807F060FAB1
:104B9000059B11932846109402F0E2FA06A90E2014
:104BA000FFF79EFF0EAF002843D04649404807F06C
:104BB0004FFA079B10942846119302F0D1FA08A9E6
:104BC0001220FFF78DFF18B33F49394807F040FA2C
:104BD000099B11932846109402F0C2FA039B3B49AB
:104BE0003B480A94CDE90B34059BCDE90D34079B76
:104BF000CDE90F34099B1193CDE900750CAB0AAADE
:104C000003F08CFB2A4807F033FA022333703FE0AD
:104C1000039B0095CDE90D34059B2C492C480C9441
:104C2000CDE90F34079B11930CAA3B4603F092FB8E
:104C3000E8E7039B254926480E94CDE90F34059BF0
:104C400011933A462B4603F0AFFBDBE7039B1F496A
:104C50001F4810942A46119303F0C0FBD2E71D4968
:104C6000134807F0F5F94FF47A6342F6E06217490A
:104C7000174803F0F1FA68B91749184807F0E8F93E
:104C80001749164807F0E4F9F6233370FFF7E8FBFD
:104C900013B0F0BD1349064807F0DAF910A80C4923
:104CA00003F0EDFB10A802F05BFAAEE7252F010040
:104CB0008C030020B0030020322F0100783A01005D
:104CC000482F01004E2F0100532F0100B103002097
:104CD000E40500205A2F0100662F01005C0300202C
:104CE000A82F0100D72F010010B53E4C3E492046A9
:104CF00007F0AEF93D49204607F0AAF93C492046A5
:104D000007F0A6F93B49204607F0A2F9204607F034
:104D1000AFF93949204607F09BF93849204607F09A
:104D200097F93749204607F093F93649204607F0AE
:104D30008FF93549204607F08BF93449204607F0B2
:104D400087F93349204607F083F93249204607F0B6
:104D50007FF93149204607F07BF93049204607F0BA
:104D600077F92F49204607F073F92E49204607F0BE
:104D70006FF92D49204607F06BF92C49204607F0C2
:104D800067F92B49204607F06CF92A49204607F0BD
:104D90005FF92949204607F05BF92849204607F0CA
:104DA00057F92749204607F053F92649204607F0CE
:104DB0004FF92549204607F04BF92449204607F0D2
:104DC00047F92349204607F043F92249204607F0D6
:104DD0003FF92046204907F03BF92046BDE8104046
:104DE00007F046B98C030020F72F010019300100AD
:104DF0002C3001003A300100423001004F300100F8
:104E00005F3001006B3001008230010096300100FC
:104E1000AB300100BA300100C9300100D1300100CF
:104E2000DC300100E6300100EE300100FA30010014
:104E300036330100103101002F31010044310100EF
:104E4000513101005F3101006B310100733101000C
:104E50007E3101008B3101009331010008B5FFF76D
:104E600043FFFFF727FB03490348BDE8084007F06D
:104E7000EFB800BF292B01008C03002070B594B05F
:104E800002F01BF9064607F0D5FD0546234806F05B
:104E9000F5F900283FD0224B93F90040002C3AD17D
:104EA00023460122402104A802F080F91D4904A8EC
:104EB0000BF021F81C4904A80BF01DF81B4904A8AD
:104EC0000BF019F83146684602F0EEF901236A4604
:104ED00004A9124806F009FC23460122402104A837
:104EE00002F064F90F4904A80BF005F80E4904A874
:104EF0000BF001F80E4904A80AF0FDFF68464FF4D4
:104F00007A71B5FBF1F102F0CFF901236A4604A9E9
:104F1000024806F0EAFB14B070BD00BFBC030020DD
:104F200088030020E5330100022E01004333010015
:104F3000F43301002DE9F041144FDFF85C800025C7
:104F40002E463C462946404605F021FAE8550138F0
:104F5000C0B2FD2805F1010598BF0126062DF1D14B
:104F60007EB90B490B4807F073F8DE232370AD239D
:104F70006370BE23A370EF23E370FE232371FF232E
:104F80006371BDE8F041FFF78FB800BFB1030020A7
:104F90000D2D01008C0300201803002008B54FF4EC
:104FA000E13005F0F7FF1949194807F051F81949A0
:104FB000194805F089FF1949194805F085FF194975
:104FC000194805F081FF1949194805F07DFF194975
:104FD000194805F079FF1949194805F075FF194975
:104FE000194805F071FF1949194805F06DFF194975
:104FF000194805F069FF1949194805F065FF194975
:105000001948BDE8084005F05FBF00BFD92C01007A
:10501000400300205D4E0000DD2C0100F13E000049
:10502000E22C01000D610000E72C0100816100000D
:10503000583401001D410000EC2C0100AD3E000081
:10504000F02C010089450000F52C01001D4A0000EC
:10505000F92C0100A9460000FC2C01004D3F000086
:10506000002D0100D53E0000062D01002DE9FF476F
:105070003E4E3368002B76D03D4D3E4F2B783C683A
:1050800001332B7007F0D6FC4FF0FF3301460F229F
:10509000204602F035F900283CD03368DFF8E09074
:1050A000DC68DFF8E0A07CB3237C03F00F03062B61
:1050B00026D14A462146504605F019FEB8B1037C78
:1050C00003F00F03052B12D1D0F80C80B8F1000FBC
:1050D00016D02246414601A8FBF7E0FB022101A8B9
:1050E000FCF710FA07F0E2FCD8F80480EEE721465E
:1050F000002201A8FBF7D2FB022101A8FCF702FA6B
:1051000007F0D4FC6468CEE707F094FC38601A48D6
:10511000FCF77CFA194C276807F08CFC4FF0FF3342
:10512000014641F28832384602F0EAF82746B8B123
:105130003368DC688CB1237C03F00F03062B08D1A5
:105140002146002201A8FBF7A9FB012101A8FCF7D9
:10515000D9F907F0ABFC6468ECE707F06BFC38604A
:105160002B78013B2B7004B0BDE8F087A80300202A
:105170003D03002014040020FC0200202004002035
:10518000602601005406002010B5064C2378013338
:10519000237007F08BFCFFF769FF2378013B237036
:1051A00010BD00BF8803002030B5104B196885B0D2
:1051B000C9B10F4CCD6822780132227085B12B7CA9
:1051C00003F00F03062B07D10022294601A8FBF7A5
:1051D00065FB01A8FCF7EEF907F068FC6D68EDE7E8
:1051E0002378013B237005B030BD00BFA803002029
:1051F0003D0300202DE9F043354E364D3278013223
:1052000032702A688BB012B3D468334F2A68F2B177
:10521000ECB1237C03F00F03052BF8D1214638466F
:1052200005F055FD0128F1D921466846FCF7AAFC96
:105230006846FCF739FC18B102216846FCF7EEFE1F
:1052400007F034FC68466468FCF7C8FADEE7337898
:10525000013B3370214B93F90030052B35D0204EA4
:10526000346807F0E7FB4FF0FF3301464FF47A72E2
:10527000204602F045F8804638B3DFF868900027F2
:105280004C46D9F8001001B3FFB90B7C03F00F03B3
:10529000052B0ED16846FCF775FC01216846FCF72A
:1052A000BDFE18B107F0C6FB474630606846FCF704
:1052B00095FA23684BB107F0F9FB23685B6823601C
:1052C000002BDED12B68DB6823600BB0BDE8F083D8
:1052D0003D030020AC03002054060020B003002052
:1052E0001C0400200804002070B580EAE074A4EBE0
:1052F000E0740E4605460121204607F047FD6EB1D9
:10530000E943C90F204607F069FD0749074806F041
:105310009FFE0648BDE8704006F0AABEE90F204691
:1053200007F05CFD0249F1E7D02A010040030020AC
:10533000D42A01002DE9F04F2DED048B744B91B070
:105340001C6807F077FB4FF0FF33014647F23052FD
:10535000204601F0D5FF002800F0D4806D4B1A687C
:10536000002A00F0CF806C49D4680B789FED6B9ACF
:1053700001330B70002C00F0BB80237C03F00F0383
:10538000052B12D100222146654805F0A8FC43698F
:10539000052B0AD1214606A8FCF7F4FB06A8FCF76A
:1053A00083FB20B906A8FCF719FA6468E2E706A9AE
:1053B00004A8FEF733F806A8FCF724FB00210646F4
:1053C00006A8FCF79BFA054604A8FDF7FFFD08EECA
:1053D000900A06A8FCF70CFA33B207EE903AF8EE02
:1053E000E77A814687EE898A06A8FDF797FB4D4943
:1053F00007464D4806F02CFE4FF0020818EE900AC2
:1054000008F0FCFFCDF8008002460B46CDE9020112
:10541000454806F065FF4549434806F019FE18EE79
:10542000100A08F0EBFFCDF8008002460B468246DA
:105430003D488B4606F054FF3D493B4806F008FEC8
:105440000A224946384806F06CFE5FEA16484AD000
:10545000082002F0AAF84FF6FF7381B240F6271237
:10546000404601F04DFFA8B12168324806F0F9FD31
:105470003149304806F0ECFD30492268304806F0EA
:105480001FF9B1B206A8FCF7D5FA00212846FFF7AC
:105490002BFF87E7DFED2B7AB4EEE78AF1EE10FA07
:1054A00004DD22682849264806F00AF9002FECD0CE
:1054B0000022264BDDE9020108F040FE52465B4621
:1054C00009F084FA014608B10121DFE7F4EEC88A49
:1054D000F1EE10FADAD91E49134806F0B9FD124868
:1054E00006F0C6FD5EE71B490F4806F0B1FD59E71F
:1054F000094A1378013B137007F09CFA044B1860BB
:10550000FFF7BCFC11B0BDEC048BBDE8F08F00BF11
:1055100024040020AC0300203D0300200000C8420A
:10552000540600202D2A010040030020332A0100E8
:10553000CC2701005C030020392A0100492A010020
:10554000BC03002000001842552A01000000F03F73
:10555000622A01003F2A0100F0B5464E33688BB045
:10556000002B00F0848044494448454C454D464F4B
:1055700006F06EFD414806F07BFD94F90030ABB1BA
:1055800005F0FCFC2B781BB13B680BB101F0F0FB84
:105590003E4B93F90030052B01D0FFF72BFEFFF7B0
:1055A000C9FEFFF763FD07F081FAE6E738493348A3
:1055B000384D394F06F04CFD304806F059FD2B6848
:1055C000DC682B68E3B1DCB1237C03F00F03052B0F
:1055D00014D12146384605F07AFB78B12168684637
:1055E000FCF706FB6846FCF75FFA10B16846FCF76B
:1055F000EFF807F05BFA6846FCF7F0F86468E0E75C
:10560000264B27491D4800241C6006F021FD1B483D
:1056100006F02EFD234B244918481C7006F018FD97
:1056200001F04BFD0A220146144806F086FD316860
:10563000194804F04BFF1D4B1D491C601D4B0F48C2
:105640001C601D4B34601C600F4B2C601C6006F00E
:10565000FFFC01F032FD0A220146084806F06DFD0C
:10566000064806F005FD154B1C70154B1C700BB061
:10567000F0BD00BF0C040020C9320100400300202F
:105680003D0300200404002000040020B00300209B
:10569000DE320100AC030020540600200804002084
:1056A000F432010010040020FC320100A8030020A5
:1056B0007F28010028040020B80300203C030020BC
:1056C0003E0300202DE9F3410024214F009423469E
:1056D000224621461F48204E204D06F079FC3846D0
:1056E00002F0C4FF1E4804F04FFE304603F0DEF91E
:1056F00031461C4E0122284606F098FB4FF0010867
:1057000000942B4631460722174801F0E7FB2B4651
:105710003146CDF800800322144801F0DFFB2B4610
:10572000062200943146124C124801F0D7FB414644
:10573000114801F093FB3946204606F071F80F4AF4
:105740000F49204602B0BDE8F04107F007BC00BF9A
:105750007403002024030020500400202C040020A7
:1057600018030020B0060020400300205C03002046
:10577000BC0300208C0300201C030020000000203C
:10578000EDAF0000F7B53C4C2678002E6ED13B4BB8
:1057900093F90030012B69DD394D2B68002B65D062
:1057A00040F20221374803F05BF92968364A37484E
:1057B00005F09DFA0546002858D00146334805F00B
:1057C00086FA07B2002F51D031462846FEF7E6FC94
:1057D000012F06464CD0294601222C4805F07FFABD
:1057E00045692B49684602F04AFE1022294968465D
:1057F00001F090FC2849294806F02AFC3146274848
:1058000006F02FFC2649254806F02BFC0A222946E3
:10581000224806F086FC2249204806F022FC1D4959
:105820001E4806F01EFC1D4806F022FCAAB23146B6
:105830001C481D4D06F012FB16491A4806F012FBD3
:105840001A4B186818B10021FEF7A8FC28602968D7
:1058500011B1144806F00EFB0021124806F012FBAD
:10586000012313490D48237006F0F2FB03B0F0BD8D
:1058700040F20225B5E700BF10040020B00300206D
:105880000C04002050040020A12A0100540600202E
:10589000E40500202C030020A82A01008C0300202E
:1058A000232F01002C04002058030020B8030020FF
:1058B000B72A01002DE9F04F7C4C21688DB00029FA
:1058C00000F0EE807A4F7B4A3B787B487B4D01337A
:1058D0003B7005F00CFA7A4A28602168764805F09A
:1058E00006FA784B784A18602168734805F0FFF98A
:1058F000764B774A186021686F4805F0F8F9754BC8
:105900001860FFF73FFF744A21686B4805F0EFF914
:10591000724BA946186030B3714D2B781BBBC4681D
:10592000704801F0FFF8002814BF012300232B70FA
:1059300003D06D496D4806F08BFB6D4B00221A6059
:105940008CB12B787BB1237C03F00F03062B06D19F
:10595000206802A901F02FFB02A801F01FFA07F04E
:10596000A5F86468ECE7634A00231360D9F80030B7
:105970009246002B00F08780D3F80C80DFF890B1BE
:105980005D4CD9F80030002B00F08D80B8F1000F8D
:1059900076D098F8102002F00F02052AF3D1414684
:1059A000454805F094F90128EBD9414602A8FCF7D7
:1059B000E9F802A8FCF778F8A8B102A8FBF7F6FE10
:1059C000064680B9014602A8FBF798FF051E02A80B
:1059D000BCBF6D420126FBF70BFF9DF81820052A7E
:1059E00009D0062A26D007F061F802A8D8F804806A
:1059F000FBF7F4FEC5E718B9022102A8FBF706FF82
:105A00000121284607F0C2F90021284607F0E6F9EF
:105A10005946204606F01CFB29460A22204606F07D
:105A200080FB3649204606F013FB3549204606F038
:105A30000FFBD8E701900121284607F0A7F9019B49
:105A4000D6B113F1FF3618BF01263146284607F0BC
:105A5000C5F92C49204606F0FBFA0A2229462046C1
:105A600006F05FFB2849204606F0F2FA0A2231468A
:105A7000204606F056FBD8E7013B5E425E41E4E774
:105A8000DB68CAF800301C4806F0F2FAFFF78CFB1E
:105A9000FEF78AFD1D4B01221A703B78013B3B70DB
:105AA0000DB0BDE8F08FDB68FFDE00BF0C04002006
:105AB0003D030020712A010054060020AC030020A1
:105AC0001C32010028040020772A0100A8030020CE
:105AD0007A2A0100B80300207F2A01000004002078
:105AE00004040020A13F0000822A01008C03002052
:105AF000B004002008040020400300209A2A01007E
:105B00009F2A01001D280100912601003C0300206E
:105B1000922A010030B5BFB005460C461C22002178
:105B200012A8119109F09FFA012D40F3B6801F22AF
:105B3000616811A80AF057FA11A91620FEF790FD26
:105B400011A9734806F08DFA7249714806F080FA7F
:105B50006F4806F08DFA704A5179137804911179E3
:105B60000391D1780291917801915278009240216D
:105B70006A4A19A80AF0FEF86949654806F068FA09
:105B800011A9634806F06DFA19A9614806F069FA8F
:105B90005F4806F06DFA0CA802F068FD614906A89E
:105BA00006F0D3FE11AA0CA9502329A804F014F979
:105BB0004FF47A6329A8399304F03DF919A929A86B
:105BC00004F060FA044629A804F059FA002C40F0C9
:105BD0009C8029A804F064FA29A9044609A804F0C5
:105BE00075FB09A906A806F0F8FE09A806F068FEEC
:105BF00029A804F015F94C49454806F029FA0A226B
:105C00002146434806F08DFA414806F031FAC82C87
:105C100079D14649464806F01BFA06A909A806F0BC
:105C2000D2FE09A9424806F017FA414806F020FAC8
:105C300009A806F045FE3F493D4806F009FA01F083
:105C40003CFA0A2201463A4806F077FA384806F04C
:105C50000FFAFFF781FC3849354806F0F9F9344866
:105C600006F006FA3349324806F0F2F901F025FA57
:105C70000A2201462E4806F060FA2D4806F0F8F98F
:105C800006992E4804F03EFF2D4B1860D8B92D49D7
:105C90002D4806F0DDF90E242AE0202211A9162055
:105CA000FEF718FD00287FF456AF2022274911A8DF
:105CB0000AF099F92649164806F0CAF911A91448BC
:105CC00006F0CFF944E72349194806F0C1F901F07D
:105CD000F4F90A220146164806F02FFA144806F095
:105CE000C7F9FFF7E7FD1C49094806F0B1F904249C
:105CF0001A4B29933BA806F0E3FD06A806F0E0FD49
:105D000020463FB030BD1649C2E71649C0E700BF84
:105D10008C0300209C2D0100B1030020C12D010047
:105D2000F02D0100CE390100042E0100172E0100D4
:105D3000400300205B2E0100262E010054060020A7
:105D40000C0400203C2E01005C030020683301009D
:105D5000A32D0100532E0100612E0100F438010033
:105D6000682E0100822E010010B52049204886B01F
:105D700006F06EF91E4806F07BF94C211D4804F030
:105D800006FB7B282BD14FF0FF3203921A4A009278
:105D900000234C22CDE90133CDE90423FFF7DCFBDE
:105DA0006946164804F0AAFE154B186040B915491B
:105DB000154806F04DF9144806F05AF900200CE099
:105DC00012490B4806F044F9094806F051F9FFF76B
:105DD00071FD0F4802F030FD012006B010BD0D49E5
:105DE000034806F035F90248E6E700BFC02E01007F
:105DF0008C0300201803002088390100540600207D
:105E00000C040020DB2E01005C030020E72E0100C3
:105E100074030020EE2E010030B58D4C94F9003053
:105E20000B3393B0192B2BD8DFE813F0B000A00090
:105E30002A002A002A002A002A002A002A002A0012
:105E40002A001A003D004000490061006D009000EA
:105E50002A002A002A002A002A00C100CE00DD0004
:105E60007C4B7D481B78002B14BF0921012100F0D9
:105E7000F6FF7A4802F030FB022801D0FEF756FE0A
:105E800094F90030012B40F3BD80744802F0BCFA55
:105E90000138042800F2B680DFE810F0B800BD0039
:105EA000C900D600AB0002232370E9E76C4D2B78C4
:105EB0001BB9FFF767FC01232B700323F4E7654B45
:105EC00065481B78002B14BF0B21032100F0C7FF8E
:105ED000644B93F90030002B40F0B880624B197886
:105EE000002941D10846FFF715FE2070C8E7594B3D
:105EF00059481B78002B14BF0B21032100F0AFFF82
:105F0000FEF712FCBCE7594B1D6806F093FD4FF0FD
:105F1000FF33014641F28832284601F0F1F90028AA
:105F2000AED000230322412101A801F03FF95049DE
:105F300001A809F0E0FF01A94E4805F022FC062364
:105F40004D494E48237006F083F899E7414B42488B
:105F50001B78002B14BF0A21022100F080FF454866
:105F600005F08CF900288BD104239DE706F062FD33
:105F70003E4B1860F5232370364B37481B78002BB7
:105F800014BF0921012100F06AFF79E7374B1D6832
:105F900006F050FD4FF0FF33014641F288322846AB
:105FA00001F0AEF900283FF46BAF00237CE73148E5
:105FB00005F064F910B12F4805F02DF906F03AFD0F
:105FC0002A4B18600D236FE7284B1D6806F032FD41
:105FD0004FF0FF33014642F21072284601F090F96B
:105FE0000028C1D14CE7FFF7BFFE0028BCD1F62343
:105FF0005AE72349234806F02BF8224806F038F8E0
:10600000F623237094F9000013B030BD1E491D48DB
:1060100006F01EF8F4E71D49184806F019F801A823
:106020000E4902F02CFA01A801F09AF8EAE71849A3
:10603000144806F00DF80F4805F020F90028DFD0CD
:106040000C4805F0E8F8DBE71249E5E70320DBE759
:10605000B00300203C0300201C030020E4050020C6
:10606000A40300203D0300203E030020180400206C
:1060700000320100BC030020493201008C030020E3
:10608000603201005C030020693201007D320100B2
:106090009A320100AD32010008B5164800F0E1FE69
:1060A00006F004FD04F06AFFFFF7B6FE022802DDE9
:1060B000114805F00BFA06F0F9FC104B1B7823B1E0
:1060C0000F4B1B680BB100F053FE0E4B1B6853B116
:1060D0000D4B93F90030052B01D0FFF78BF806F03C
:1060E000E5FCFFF727F906F0E1FCBDE80840FEF704
:1060F000BDBF00BF1C030020BC030020040400201F
:1061000000040020AC030020B0030020FFF72CBEE9
:1061100070B5FEF743FFFEF7E7FD144E144D46241D
:106120002146304604F033F92B1913F8463C8342DC
:1061300017D000210846FDF709FFFEF7FBFE1420EB
:1061400006F092FC0B4800F071FE0B490B4805F07D
:106150004AFB4FF4FA7006F087FCBDE87040FFF789
:1061600003BE01344A2CDBD1E7E700BF180300204F
:10617000A23301005D3D0000613D0000BC03002032
:1061800008B5FFF7C7FC034B18700348BDE808408B
:1061900002F052BBB00300207403002007B50023B7
:1061A00000931A461946034805F012FF03B05DF844
:1061B00004FB00BF7404002001207047014B1868E5
:1061C000704700BF84040020032070477047000020
:1061D00010B504460B490C4805F05AFFA17C94F910
:1061E000080006F0FBFDA17C94F9090006F0F6FD1D
:1061F00060680021FBF71EFC044B00221A6001209E
:1062000010BD00BF5C340100B006002084040020F3
:10621000F7B56E460546304686E80600FDF7AAF853
:1062200004463046FCF799FE10B1002C08BF01244B
:106230004FF480516868FBF71BFB012C1CD0022C2B
:1062400004D044BB2049214805F002FF3046FCF74A
:1062500089FE002836D06868FBF7D4FB18B9012402
:10626000204603B0F0BD00206C6801F09EF90146A5
:106270002046FBF7DFFBF2E730466F68FCF7EAFFEA
:1062800001463846FBF7C2FA3046FCF7E3FF012827
:106290000AD0022808D00E490C4805F0D9FE0B4858
:1062A00005F0E6FE0024DBE76868FBF7ABFB00289F
:1062B000D5D000206D6801F078F901462846FBF73B
:1062C000B9FBCDE70446CBE71834010040030020BA
:1062D0002934010010B5044606F002FC204610BD2A
:1062E0002DE9F0434FF4805185B004464068FBF738
:1062F000AFFA002800F0AF804FF400516068FBF760
:10630000A7FA68B98D4D95F90030002B00F0A380F5
:106310004FF400516068FBF7ABFA2B78013B2B7010
:106320006068FBF76FFB00221146814602A8FCF76C
:10633000C5FC0022616802A8FDF72AF8002102A826
:10634000FCF71CFF80466068FBF752FA022801D078
:10635000052801D14FF0000894F90A00A0F10E03BE
:10636000DBB2072B00F2CF8006F01AFCFF25E28992
:10637000218A00950023074606F089FA061EC0F21E
:10638000BE80AE4200F3BD80B9F1000F40F0C18085
:10639000A8EB060507E06A496A4805F059FE694816
:1063A00005F066FE00256849664805F051FE0A22A0
:1063B00094F90A10634805F0B4FE6449614805F099
:1063C00047FE0A2239465F4805F0ABFE60495D484A
:1063D00005F03EFE0A2231465A4805F0A2FE5D490C
:1063E000584805F035FE0A224146564805F099FE08
:1063F0005949544805F02CFE0A222946514805F017
:1064000090FE504805F034FE15F10A0F2CDA94F98D
:106410000900A17C06F0E2FC6068FBF7F3FA30B9F2
:10642000666801F0C2F801463046FBF703FBA37C27
:106430006842A3B100210091FF23192206F027FA38
:10644000FF280146A8BFFF21462994F90800B8BFDC
:10645000462106F049FC002005B0BDE8F083FF228C
:10646000009219461922E9E70A2D27DD94F9080060
:10647000A17C06F0B3FC6068FBF7C4FA30B966682B
:1064800001F093F801463046FBF7D4FAA37C83B1C0
:1064900000210091FF233322284606F0F8F9FF2857
:1064A0000146A8BFFF214629B8BF462194F909003B
:1064B000CFE7FF22009219463322EDE7274928480B
:1064C00005F0E6FDA17C94F9080006F087FCA17CAC
:1064D00094F9090006F082FC00216068FBF7AAFA33
:1064E0004FF480516068FBF7E5F94FF400516068A4
:1064F000FBF7E0F9114A137801331370ABE700267C
:1065000042E72E4640E74FF0FF37B9F1000F10D0B9
:106510003E4606F08FFA4FF0FF330146B4F90C20E7
:10652000484600F0EDFE00287FF435AF731C7FF481
:106530002FAFA8F17F054FF0FF3634E704000020AD
:10654000353401004003002043340100473401008A
:10655000022E0100102601004D34010055340100C7
:10656000B0060020002110B5044681744068FBF796
:10657000C5F943B2002BBBBF4042207223720123F6
:10658000B8BFA374237A6068013B122B84BF202319
:1065900023720121FBF7B2F943B2002BBBBF40428B
:1065A000607263720123B8BFA374637A6068013BB1
:1065B000122B84BF212363720221FBF79FF9C3B220
:1065C000132B8ABF0023A072A37203216068FBF71C
:1065D00095F980B2431EB3F5806F26BF0023E38197
:1065E000E08104216068FBF789F980B2B0F5806F23
:1065F0008ABF4FF480632082238205216068FBF705
:106600007DF900B20028D6BF42F21073A081A381A9
:1066100010BD000010B50446F9F7EDFF2046FFF766
:10662000A1FF1849184805F033FD94F9080001212D
:1066300006F0ACFB94F90900012106F0A7FBA17C50
:1066400094F9080006F0CAFBA17C94F9090006F051
:10665000C5FB94F90A00002106F098FB6068002150
:10666000FBF7E8F960684FF48051FBF723F96068A5
:106670004FF40051FBF71EF9044B01201860044B46
:10668000187010BD6A340100B00600208404002098
:106690000400002007B5002300931A46194603485A
:1066A00005F096FC03B05DF804FB00BF7C040020FD
:1066B000014B1868704700BF90040020002070470D
:1066C0007047000010B51A4904461A4805F0C0FC8E
:1066D000184805F0CDFC236820465B6B98470128DD
:1066E00005D002280AD00021B4F9080019E00321DE
:1066F0002046FAF73DF8002106F048FB002120462D
:10670000FAF736F8002106F041FB01212046FAF79E
:106710002FF8002106F03AFB02212046FAF728F86C
:10672000002106F033FB044B00221A60012010BD4B
:10673000CD34010040030020900400202DE9F041F9
:10674000044688B040689DF8383002AE86E80600FE
:1067500000286ED0B4F90820002A69D0002B6BD035
:106760000021FBF7CBF8236880465B6B20469847F7
:1067700005B2022D51D0032D2BD0012D0CBF0521C8
:106780000121002204A8FCF799FA4FF0FF3300938F
:1067900096E80C0004A906A8FCF7C6FF012D3ED020
:1067A000022D38D19DF81610B4F9080006F09CFAB5
:1067B00001212046F9F7DCFF9DF8151006F094FA48
:1067C00002212046F9F7D4FF9DF8141006F08CFA48
:1067D00021E04FEAD8713046B4F90870FCF7CEFCDE
:1067E00001460546384606F07FFA1449144805F07C
:1067F0002FFC0A22B4F90810114805F092FC114947
:106800000F4805F025FC0A2229460D4805F089FCB1
:106810000B4805F02DFC01200BE00421B1E703211A
:106820002046F9F7A5FF9DF8171006F05DFAB9E7C5
:10683000104608B0BDE8F0811846FAE71D280100AF
:10684000400300209126010010B5044606F048F9E7
:10685000204610BD38B50446F9F7CDFE1D491E4847
:1068600005F0F6FB1C4805F003FC606870B3B4F952
:10687000083063BB236820465B6B984701280546B8
:1068800005D002280AD00121B4F9080019E003213B
:106890002046F9F76DFF294606F078FA00212046D8
:1068A000F9F766FF012106F071FA01212046F9F798
:1068B0005FFF012106F06AFA02212046F9F758FF2E
:1068C000012106F063FA054B0120186038BD002055
:1068D000FCE700BFDA3401004003002090040020F0
:1068E00010B504464068E0B1B4F90A30032B10D06B
:1068F000042B17D00A22017C0F4805F02BFC0F490E
:106900000D4805F0A5FB0C4805F0B2FB6368187C48
:1069100007E00B49084805F09BFB074805F0A8FB7A
:10692000022010BD0749044805F092FB024805F01B
:106930009FFB0120F5E700BF40030020BF340100AA
:10694000BC340100C434010007B5002300931A468B
:106950001946034805F03CFB03B05DF804FB00BF9B
:10696000880400202DE9F04F85B006F063F86049F7
:106970000290604805F082FB5F4B18689A4608B1A8
:1069800001F060F85D4C5E4F2568386800210BB25D
:10699000AB4201F10101C0F294805A4DDFF88091C1
:1069A000DAF80000002800F0938021682B6803EBE0
:1069B000C10101F0D7F9002840F38A802368132B26
:1069C00000F3868006F036F84FF0FF33014641F2BF
:1069D0008832029800F094FC0646002878D12B6893
:1069E0002068072103EBC00001F01CF82B6801931D
:1069F000019A236802EBC30B9BF807208242CFD198
:106A00000FFA86F84345039325DD019B082203EB2B
:106A1000C800594608F0F4FA0136039B0028EFD16C
:106A20003968019031F81830374843F0010321F8F4
:106A30001830364905F00CFB2B682068019A03EBEF
:106A4000C000082100F066FA31492F4805F016FB16
:106A5000B8F1000FA4DAD9F80030002BA0D03B68C1
:106A600022682948012123F812102A4905F0F0FA7A
:106A70000A222168244805F054FB2749224805F0E2
:106A8000E7FA2B682068002203EBC000082100F021
:106A900041FA1D4805F0ECFA22682B6803EBC201AD
:106AA00013F83230282B08D10C22D9F8000001F05D
:106AB0008CFADAF8000001F09FF8236801332360B4
:106AC0006EE730F8132022F0010220F813205EE771
:106AD00012490D4805F0BCFA0A2221680A4805F05F
:106AE00020FB094805F0C4FA012005B0BDE8F08F8D
:106AF000DE350100B00600209C040020B004002018
:106B0000B8040020B404002040030020F735010041
:106B1000FE350100053601000A360100E8350100A6
:106B2000A8040020F8B5424D2B6807460BB10120A0
:106B300054E040494048414E05F08AFA3E4805F08D
:106B400097FA3F493C4805F083FA00F0B6FA0A226A
:106B50000146394805F0F1FA374805F089FA142062
:106B600005F0BAFF044600F027FFA0202C6005F0D6
:106B7000B5FF344930603048334C05F069FA00F015
:106B80009CFA0A2201462C4805F0D7FA2A4805F05B
:106B90006FFA282005F0A2FF2C492060264805F056
:106BA00057FA00F08AFA0A220146234805F0C5FA8E
:106BB000214805F05DFA33680BB123687BB924499D
:106BC000244805F045FA00F078FA0A2201462148E7
:106BD00005F0B3FA1F4805F04BFA0020F8BD1E4B34
:106BE0001E481F6000F05AFD286800F0FFFE0446B2
:106BF000B8B11B49104805F041FA286801F03AF88D
:106C0000286800F0FFFE17490B4805F037FA28689E
:106C100001F074F800288AD01349074805F02EFACD
:106C200085E71249044805F029FA2046D6E700BF57
:106C30009C0400203F35010040030020B4040020E4
:106C40005B2E010060350100B80400206C350100A6
:106C5000793501005C030020A004002028050020F5
:106C600091350100A4350100C4350100D035010083
:106C70002DE9F041364E306800F0B0FE02280DD10B
:106C80003449354805F0E4F9334805F0F1F9306846
:106C900001F034F842F21070BDE8F0812F4C304F13
:106CA0002568EDB91C2005F017FF31682D4E804690
:106CB00001F0EEF84046C4F8008001F0C9F93A68E6
:106CC00020682BB2934205F1010506DA31680C22E7
:106CD00001EBC30101F079F9F1E7002101F00CFAB1
:106CE000214E3A68B6F900309342374606DBFFF78B
:106CF00039FE002333804FF4FA50CDE7194D286850
:106D000000EBC30110F8330028281AD1206801F0E5
:106D100083FA164B1B6802462BB1B6F900002968AE
:106D200001EBC00198472B68B7F90010206803EB0E
:106D3000C10101F017FA3B8801333B8040F6C410D3
:106D4000AAE701334FF4FA60338090FBF2F0A3E737
:106D50009C0400203035010040030020A8040020DE
:106D6000B0040020B4040020AC040020A0040020E3
:106D700038B5094C256805F05DFE4FF0FF3301463C
:106D800041F28832284600F0BBFA20B1FFF770FFCD
:106D900005F050FE206038BDA404002070B51C4CE6
:106DA0002368132B32DC1B4A1B4D1268012122F889
:106DB00013102968026841F8332001EBC3064268CA
:106DC00072601649164805F043F90A2221681448F2
:106DD00005F0A7F91349124805F03AF92B68206825
:106DE000002203EBC000082100F094F80C4805F0E5
:106DF0003FF922682B6813F83230282B03D10A4B55
:106E0000186800F0F9FE23680133236070BD00BFED
:106E1000B0040020B8040020B404002005360100AE
:106E2000400300200A3601009C040020034B014669
:106E3000186808B100F0D0BD704700BF9C04002066
:106E400007B5002300931A461946034805F0C0F819
:106E500003B05DF804FB00BF940400207047704746
:106E60007047704707B5002300931A461946034838
:106E700005F0AEF803B05DF804FB00BFBC040020D1
:106E8000134B1B7870B505460C4673B1114A0A299D
:106E90001368164611D1104A0021D154006910B16F
:106EA000298905F05BF800233360E86870B1036856
:106EB00021461B68BDE8704018474E2BF5DC0D29B4
:106EC0001FBF591C1160044AD454EEE7012070BD65
:106ED00010040020CC040020D004002030B5002590
:106EE00045600361034D9DF80C300560C16002816F
:106EF000037530BD1C36010007B5002300931A4608
:106F00001946034805F064F803B05DF804FB00BFC0
:106F1000C4040020F8B5441E0D4D16466718BC4247
:106F20000ED014F8011F10220909284605F0F9F8BF
:106F30002178102201F00F01284605F0F2F8EEE763
:106F400026B10348BDE8F84005F092B8F8BD00BF8F
:106F5000B006002070B501380C4D13464618B042FB
:106F600003F102030CD010F8014F24112C5D03F83B
:106F7000024C047804F00F042C5D03F8014CEEE79A
:106F800009B2002302F8113070BD00BF5A3601006B
:106F9000A0F16103052B02D85738C0B27047A0F1A9
:106FA0004103052B01D83738F7E73038C0B20A283B
:106FB00028BF0020704738B50139841C00F1120544
:106FC00014F8020CFFF7E4FF0001C2B201F8012F30
:106FD00014F8010CFFF7DCFF02341043AC420870D8
:106FE000EED138BD38B50546D8B10468ACB12478C7
:106FF0009CB1286803783BB12D2B05D0303B092B81
:1070000002D901302860F4E707F0B6FD2C210446D0
:10701000286808F07FFF10B92860204638BD01308D
:10702000FAE70446F9E72DE9F34100220D4606216F
:107030000646FBF743FE85B32B6873B31B7863B337
:10704000286803783BB12D2B05D0303B092B02D9A2
:1070500001302860F4E707F08FFDD5F8008007467F
:107060002E21404608F056FFD8B144782F2C18D96D
:10707000392C18D8303C2C21404608F04BFFA0B9E1
:107080002860A4B10A22002F02FB07F2D8BF644295
:10709000224431466846FCF70CF9304602B0BDE8A0
:1070A000F0810024E7E70924E5E70130E8E73A4604
:1070B00031466846FCF7F1F8EFE708B5002009F023
:1070C0004BF9ADEB000008BD704730B5441E2246B9
:1070D00012F8013F002BFBD11A460A2514F8010FC4
:1070E00070B1032A14DC2E2806D1FF2B10DC88187F
:1070F000013203710023F1E7303805FB0303EDE7AC
:10710000FF2B04DC032A02DC114401200B7130BD8B
:107110000020FCE72DE9F3410024DFF840800C70EB
:107120000D461746061D0A2201A916F8010B07F0A5
:1071300032FF3A4601A9284608F02FFF032C04D05D
:107140003A464146284608F028FF0134A3B2042BF2
:107150001CB2E8D1284602B0BDE8F081DC32010063
:107160002DE9F0410E4D0F4FDFF83C80064600241C
:10717000032C0ED033190A221979284604F0AFFFE8
:1071800041462846013404F063FF042CF0D1BDE8E9
:10719000F081F1790A22284604F0A1FF3946F0E790
:1071A000400300203D360100DC3201002DE9F047AC
:1071B000DFF8F0A0DAF8005004460E46174699466C
:1071C000002D49D02B7C03F00F03062B43D12C4A12
:1071D0002C48294603F08BFD022F804637D0032F21
:1071E00037D1294ADAF80010264803F080FD054619
:1071F000B8F1000F30D098F8103003F00F03042BD3
:107200002AD1D8F814103246204608F0ECFE324657
:107210001E49204608F0C1FE0DB32B7C03F00F037E
:10722000042B1CD169693246204608F0B6FE32466E
:107230001649204608F0B1FEB9F1000F04D03246DD
:107240004946204608F0A9FE2046BDE8F087104ACE
:10725000C8E70025CCE7002532460E49D4E7022FC7
:107260000AD0032F05D0012FE1D10B4B324619680C
:10727000DAE732460949D7E732460949D4E700BF81
:107280005036010054060020A3370100022E0100F1
:107290005536010074360100580300206E36010097
:1072A0006B3601002804002030B585B0002301AA08
:1072B0000A2541B1B1FBF5F405FB14113031D1546D
:1072C00021460133F5E71A44411EC41812F8015D46
:1072D00001F8015FA142F9D10022C25405B030BDCE
:1072E00010B5054C0549204604F0BBFE2046BDE81C
:1072F000104004F0BDBE00BF400300204036010036
:10730000024410B5B2FBF3F404FB13238B420DD2FD
:10731000884206D9012003E0884294BF0020012062
:1073200010BD98422CBF00200120F9E79842F3D30A
:107330000020F5E72DE9F04399B002AE0F4686E84C
:107340000C00044630B1037C03F00F03052B03D07F
:10735000062B13D000201DE07E4DC4682A78013230
:107360002A703CB1204696E80C003946FFF7E2FF50
:107370006468F6E72B78013B2B70EBE70146764A11
:10738000764803F0B4FC054638B196E80C0039465F
:10739000FFF7D0FF19B0BDE8F083714A6F4821466E
:1073A00003F0A5FC6F4A814621466C4803F09FFC20
:1073B000804677B1012F5CD02C4600231022009329
:1073C0000DEB02014FF440733046FCF737F80546E9
:1073D0001BE0654A6148214603F089FC0546634A83
:1073E0005E48214603F083FC0746002D5BD02B7CD2
:1073F00003F00F03042B56D16C69002FDDD03B7CCA
:1074000003F00F03042BD8D17D69B9F1000F5CD0D4
:10741000D9F814105648002C47D004F022FE5549E4
:10742000534804F015FE2146514804F01AFE504816
:1074300004F01EFE3046FCF7FDF8B8F1000F47D10E
:1074400099F8103003F00F03042B7CD1D9F81410F5
:1074500008A8FAF7CDFB08A8FAF726FB28B15CB319
:107460000022214608A8FBF7B9F908A8FAF7B6F9EF
:1074700069E0414A3948214603F039FC3F4A054654
:107480002146364803F033FC0746002D5DD1364ACD
:107490003248214603F02BFC0546002F9FD00028E0
:1074A000A5D10446ABE70024A7E704F0DAFD314993
:1074B0002F4804F0CDFDBDE70123009396E80600B8
:1074C000234608A8FAF7C8FDCFE7B8F1000F3AD075
:1074D000D8F81410264804F0C4FD2649244804F0C6
:1074E000B7FD2946224804F0BCFD214804F0C0FD48
:1074F0002DB398F8103003F00F03042B1FD1402256
:10750000D8F8141008A808F06EFD1D4803F0B6FE68
:10751000A8B11C4B93F900308BB92F2108A808F0B3
:10752000F9FC30B9D8F814300322402108A8FFF73D
:107530003DFE01232A4608A9114804F0D6F8B9F106
:10754000000F7FF47DAF012024E700287FF44FAFC8
:1075500045E700BF3D0300206026010054060020DF
:10756000642601009E260100243601002936010010
:1075700040030020383601002E360100333601006A
:10758000BC0300208803002073B500226C4605462A
:107590000E4620461146FBF791FB94E80C0031465D
:1075A0002846FFF7C7FE02B070BD10B5044605F0CF
:1075B00041FAE04008BF012010BD000007B50023DC
:1075C00000931A461946034804F002FD03B05DF823
:1075D00004FB00BF200500202DE9F84380460D463E
:1075E000174601EB02090C464C45A4EB05060BD0EF
:1075F000D8F8003014F8011B1B6840469847002853
:10760000F2D13046BDE8F8833E46FAE770472030B5
:1076100004F091BE203004F080BE203004F091BE12
:1076200038B5437F0D460BB9002038BD00F1680422
:10763000204604F08EFE0028F6D12046294604F0AC
:107640005DFE0120F1E700002DE9F0411E46002516
:107650004FF47A73C0E901530E4B044640F8203BC7
:107660001746884604F041FE04F1680004F03DFE30
:10767000C4E90487084B9DF81820267653F8222089
:1076800062769DF81C2053F82230A3766577204659
:10769000BDE8F08184360100083A0100827E4FF097
:1076A000A04102F5E07210B5012340F20C64C376EC
:1076B00041F82240427E02F5E07241F82240026920
:1076C0004FF0CC71C2F8241502690621C2F80015EA
:1076D0000269817EC2F808150269417EC2F80C1564
:1076E00090F91820510902F01F02934060310F4AAF
:1076F00042F8213090F91830002BBDBF03F00F0382
:1077000002F6FC32D2189B18B5BF402340221376F4
:1077100083F8002390F918300122590903F01F0360
:1077200002FA03F3014A42F8213010BD00E100E003
:107730002DE9F041044688461F461546002A50D0E0
:1077400000F12006304604F0E4FD2369C3F8888583
:10775000236901221A622369C3F834652369C3F8D7
:10776000385523691A602269D2F84C311BB9D2F816
:107770002431002BF8D00023C2F84C312269D2F812
:107780005C311BB9D2F82431002BF8D00023C2F8A9
:107790005C3122696FB9D2F8243153B90123D36126
:1077A0002369D3F84821002AFBD00022C3F84821DE
:1077B00009E0012353612369D3F80421002AFBD097
:1077C0000022C3F804212369D3F8242112B1002236
:1077D000C3F824212369D3F83C052066C0B2BDE874
:1077E000F0811046FBE70123FFF7A2BF10B5044666
:1077F00080F8B010683004F08CFD0123637710BD71
:10780000F8B500234377036990F8B020C3F88825C2
:10781000036901261E62036900F168050446C3F886
:10782000445528460F4604F086FD2369C3F84805F1
:1078300023699E602369D3F850211AB9D3F8242113
:10784000002AF8D00022C3F85021284604F073FD26
:10785000236930B1D3F860211AB9D3F82421002A62
:10786000F8D00022C3F8602123696FB9D3F824212E
:1078700052B90122DA612369D3F84821002AFBD0EA
:107880000022C3F8482109E001225A612369D3F894
:107890000421002AFBD00022C3F804212369D3F875
:1078A000240168B10022C3F824212369D3F8C40459
:1078B000C3F8C404022803D004280CBF032004200A
:1078C000F8BD0121FFF79CBF70B54369D3F864216F
:1078D000044692B10022012500F12006C3F864217C
:1078E0000577304604F015FD6369C3F834656369B4
:1078F0004022C3F8382563691D636369D3F86821A2
:10790000DAB10025C3F8685104F1680601236377F2
:107910002577304604F0FDFCD4F8B43003B1984725
:10792000636965773046C3F8446504F004FD636914
:10793000C3F84805636901225A636369D3F80421D7
:1079400062B10022C3F80421237F3BB16369D3F8FD
:107950003C05D4F8B830206603B198476369D3F882
:10796000242152B10022C3F824216369D3F8D02422
:10797000C3F8D024636901225A6170BD0148FFF742
:10798000A3BF00BF2805002007B516231722CDE9A5
:1079900000324FF04022042311460348FFF754FE03
:1079A00003B05DF804FB00BF280500200148FFF785
:1079B00088BF00BF2805002010B54FF4C0530380D6
:1079C00000230446837003610248FFF767FE2046E8
:1079D00010BD00BF28050020016170478078704706
:1079E00041780148FFF702BF2805002008B5FFF7DE
:1079F000F7FF0348FFF765FFB0FA80F0400908BDC4
:107A000028050020012303707047FF23C372002361
:107A10000373C370037143718371C3710372437243
:107A20008372704710B5064A01440023884204D08F
:107A300010F8014B6340D35CF8E7184610BD00BF57
:107A40009C360100FFF7E1BF38B5084C0D46FFF743
:107A5000C7FFE1212046FFF7E3FD29462046FFF757
:107A6000DFFDBDE83840FFF7A1BF00BF28050020BB
:107A700010B5054C417801222046FFF7B4FE2046A0
:107A8000FFF7C8FDC0B210BD2805002010B5F021D9
:107A90000446FFF7D9FF2046BDE81040FFF7E8BFD6
:107AA00070B5054604F0C6FF002400F57A7604F0B0
:107AB000C1FFB04246D22846FFF7E8FFC30704469D
:107AC00046D52B6903B198471420013800BF00BF89
:107AD00000BF00BF00BF00BF00BF00BF00BF00BFAE
:107AE00000BF00BF00BF00BF00BF00BF00BF00BF9E
:107AF00000BF00BF00BF00BF00BF00BF00BF00BF8E
:107B000000BF00BF00BF00BF00BF00BF00BF00BF7D
:107B100000BF00BF00BF00BF00BF00BF00BF00BF6D
:107B200000BF00BF00BF00BF00BF00BF00BF00BF5D
:107B300000BF00BF00BF00BF00BF00BF00BF00BF4D
:107B4000C3D1B4E70123AB700249034804F0A0FAA3
:107B5000204670BD9C370100B006002010B5E12121
:107B60000446FFF771FF2046BDE81040FFF780BFD5
:107B700010B50446FFF794FF2046FFF731FF96212A
:107B80000648FFF74DFDFFF711FF2046FFF788FF7E
:107B90002046BDE81040FFF7E1BF00BF28050020E8
:107BA000FFF7E6BF10B5C3210446FFF74DFF20469F
:107BB000BDE81040FFF75CBF38B504460D46FFF73F
:107BC0006FFF2046FFF70CFFD2210A48FFF728FD80
:107BD000E94345EA0111C9B20648FFF721FDFFF765
:107BE000E5FE2046FFF744FFA8421CBF0423A37014
:107BF00038BD00BF2805002010B50446FFF7D2FFAE
:107C000040F00401C9B22046BDE81040FFF7D4BFE0
:107C100070B5164604460D46FFF742FF16B12046E2
:107C2000FFF7EAFF2046FFF7DBFEA5210548FFF737
:107C3000F7FC29460348FFF7F3FCBDE87040FFF767
:107C4000B5BE00BF2805002070B500220C465521A6
:107C50000646FFF7DDFF651E073415F8011F0022F9
:107C60003046FFF7D5FFA542F7D170BDFFF7ECBF57
:107C7000FFF7CEBF10B50446FFF7B2FE2046002244
:107C8000F021FFF7C5FFBDE81040FFF78FBE0000F1
:107C900070B5164605460C46FFF702FF16B128469A
:107CA000FFF7AAFF2846FFF79BFE87210648FFF74C
:107CB000B7FC002C0CBF214680210348FFF7B0FC25
:107CC000BDE87040FFF772BE2805002010B5002205
:107CD00004460121FFF7DCFF2046FFF7E1FEC0F379
:107CE000401010BDFFF7F2BF10B50446FFF75AFF72
:107CF00020460021BDE81040FFF75EBF38B50446BE
:107D0000FFF7CEFEC30729D42046FFF7EDFF20463C
:107D1000FFF7C6FE2046FFF763FEB4211048FFF7C9
:107D20007FFCFFF743FE2046FFF7BAFE10F0040386
:107D3000054602D00223A37002E0A278022AFAD0FC
:107D4000237843B12046FFF72DFF40F00101C9B26F
:107D50002046FFF731FFC5F3400038BD0020FCE7A7
:107D6000280500202DE9F74F057B04460F46002D1E
:107D70007AD1FFF7C3FF40B93C493D4804F088F988
:107D80004FF0FF3003B0BDE8F08F2046FFF788FECC
:107D90002A46F0212046FFF73BFFDFF8DC804FF05A
:107DA000FF394FF0010A94F90B30EEB24FEAD60BCF
:107DB0009D4206F007060AFA06F62CDA04EB0B03DE
:107DC000DB78334020460193FFF76AFE2046FFF739
:107DD00007FE78214046FFF723FC019B002B0CBFD8
:107DE000194680214046FFF71BFCFFF7DFFD2046C8
:107DF000FFF756FE8206014600F040030FD59BB107
:107E000002221B4804F0A6F91A49194804F040F967
:107E10006FF00100B6E70CBF01230023D2E71BB9C6
:107E2000080658BF4FFA85F904EB0B03090693F9CE
:107E3000032076B205F101054CBF3243B243402D19
:107E4000DA70B0D1B9F1FF3F04BF0123237384F886
:107E50000B90E31C013F0B3413F8012B07F8012FA3
:107E6000A342F9D101208DE700208BE7A73701005D
:107E7000B0060020B33701002805002008B5FFF741
:107E800071FF20EAE070C0B208BDFFF737BF70474E
:107E9000054A8261002202710270092242700122A9
:107EA00081608270C27070478F7E000010B50C46F2
:107EB00020460721FFF7B6FDE3791B1A58425841C7
:107EC00010BD70B5044680680E461546FFF7DDFF0D
:107ED000B8B13146A068FFF7C9FE0022BE21A068F4
:107EE000FFF7C6FE6E1E0835A068FFF759FE06F8BC
:107EF000010FAE42F8D1A068FFF7C7FF431E5842FA
:107F0000584170BD10B51446FFF7DBFF38B10821AA
:107F10002046FFF787FD237A1B1A5842584110BDAF
:107F200070B504460D4680681646FFF7AEFF294639
:107F3000A068FFF79BFE00224E21A068FFF798FE85
:107F40000022B178A068FFF793FE0022F178A068C4
:107F5000FFF78EFE2B78102B04D000223179A06819
:107F6000FFF786FEA068FFF790FF2946A068FFF79D
:107F70007DFE2278A0684821FFF77AFE142004F0E5
:107F800073FD237813B10A2004F06EFDA068BDE8EC
:107F90007040FFF77ABF38B504460D468068FFF79A
:107FA00074FF2946A068FFF761FE0022B421A06893
:107FB000FFF75EFEA068FFF795FE0546A068FFF795
:107FC00064FFB5FA85F0400938BDF0B585B01446B8
:107FD00001AA07460E46FFF795FF054690B1337894
:107FE000102B0FD00B2C10D00C2C03D00A2C0ED140
:107FF0003F2300E07F2301AA314638468DF8083040
:10800000FFF78EFF284605B0F0BD5F23F3E71F237F
:10801000F1E71FB50B78102B10D001AAFFF772FF04
:1080200078B19DF808303F2B0ED003D81F2B0DD010
:10803000002006E05F2B03D07F2BF9D10C2000E05D
:108040000B2005B05DF804FB0A20FAE70920F8E7E9
:108050002DE9F04387B0044604F0ECFC00F51C5514
:10806000A068224F224EDFF88C80FFF7EBFC002344
:108070001035237101A9A068FFF700FF90B304F049
:10808000D9FCA8422ED201A92046FFF70FFF20B34A
:108090004146304603F0E5FF237833B901A9204675
:1080A000FFF779FF08B10123237003AA01A9204635
:1080B000FFF707FF01A9204694F80190FFF7A9FFF9
:1080C000814505D960782379607001332371D1E748
:1080D00001A92046FFF79DFFF5E73946304603F03A
:1080E000C0FFC7E707B0BDE8F08300BFC637010097
:1080F000B0060020C4370100817070471FB501AA87
:10810000FFF7DFFE9DF80400003018BF012005B026
:108110005DF804FB0939C9B20229F8B598BF104BC4
:108120000546164694BF33F9114040F2EE248AB159
:10813000C3787BB103786BB904F07CFC0746314609
:108140002846FFF7DBFF20B904F074FC001BB8429F
:10815000F5D3F8BD2046BDE8F84004F085BC00BF6B
:10816000BE370100F8B504460F46FFF752FF06463A
:1081700010B900252846F8BDA068FFF786FE002844
:10818000F7D03946A068FFF771FD2278A068442136
:10819000FFF76EFDA5782DB13A4631462046FFF730
:1081A000B9FFE7E70125E5E710785378C00040EA1A
:1081B000C3200B78102B00B20BD1D1799379C0007A
:1081C000CB1ADB0120F07F0093FBF1F3103B184446
:1081D00000B2704730B585B001AA04460D46FFF7DE
:1081E00091FE30B101AA29462046FFF7DDFF05B018
:1081F00030BD0148FBE700BF80E4FFFF10F5DC5F06
:10820000CABF07EE900ADFED037AFAEEEC7A17EEBA
:10821000900A70470000FEC208B5FFF7DBFFBDE81B
:108220000840FFF7EBBF042302461946012000F087
:108230003FBE042302461946052000F039BE02461F
:1082400006230421092000F033BE04230246194608
:108250000F2000F02DBE00002DE9FF41044600690B
:108260000E461746984608B104F03AFC782004F010
:1082700033FC78220546002106F0F5FE05F1540096
:1082800000F014FC217D2561234800F067FE0025E5
:108290003046FFF7D4FF2B462A462946009502A810
:1082A00003F096FE03A8FFF7D0FF29462E2000F02A
:1082B0002DFE10F001052BD043463A463146206989
:1082C00001F059FA0128054622D1216902A800F0DF
:1082D00078FF03A8FFF7B9FF216902A800F07FFF2C
:1082E00003A8FFF7A0FF216902A800F071FF03A80F
:1082F000FFF79FFF216902A800F078FF039B6360EE
:10830000206900F07AFFA060206900F078FFE0604B
:10831000284604B0BDE8F08127060020F8B50446E1
:108320000F46017D0A4816461D4600F017FE3846E6
:10833000FFF785FF301DFFF788FF06980430FFF731
:1083400072FF07980430FFF774FF6B686360F8BD35
:1083500027060020F0B58DB01E4600231746009377
:10836000FF2304460D461A46194602A803F030FEC4
:108370007A680C4B0493CDE905237268CDE9072395
:10838000129A5268CDE90923039B0B930AAB019320
:1083900008AB009304AA06AB29462046FFF7BEFFB0
:1083A0000DB0F0BD783A010010B554685B680A4A18
:1083B0008AB0CDE90732012303948DF80F30039B77
:1083C000099308ABCDE904240692009304AA06ABF6
:1083D000FFF7C0FF0AB010BD783A01007FB5094B26
:1083E00052680493CDE90232012301928DF80730DF
:1083F000019B059302AA04ABFFF7D6FF07B05DF817
:1084000004FB00BF783A010037B5044600212E2056
:1084100000F07CFDC3072ED5206970B301F0C4F9CC
:108420000228054601D0042822D12169684600F0BF
:10843000C8FE01A8FFF709FF2169684600F0CFFEDA
:1084400001A8FFF7F0FE2169684600F0C1FE01A80F
:10845000FFF7EFFE2169684600F0C8FE019B6360EC
:10846000206900F0CAFEA060206900F0C8FEE0604C
:10847000284603B030BD0525FAE70546F8E710B5F4
:10848000044603F09DFD0423E21800210F2000F0B4
:108490000BFE204610BD10B5044603F091FD0423E9
:1084A000E2180021052000F0FFFD204610BD10B5A8
:1084B000044603F085FD0423E2180021012000F0AA
:1084C000F3FD204610BD0000024A02604A68426087
:1084D000704700BF783A010008B5017D064800F0FA
:1084E0003DFD00212E2000F011FD10F0010F0CBF0A
:1084F0000220012008BD00BF2706002037B5002458
:108500000A4D0094234621462246094803F060FDA7
:10851000284603F055FD0A232B75064B2C6118786D
:10852000012103B0BDE8304004F030BCE405002078
:10853000FC0500202606002008B503681B6B984741
:1085400080F00100C0B208BD13B502AB026803F8A9
:10855000011D546819460122A04702B010BD007CDD
:10856000083818BF01207047037C087C984203D16B
:10857000083818BF012070470020704770B590B0D0
:10858000044604A815460E4603F01AFD07A800F09D
:108590008DFA684603F014FD0D4902A8FFF794FF19
:1085A00002A904A801F04BF96A46314604A801F07B
:1085B000F7FA012809D12368064A9B690292019AB9
:1085C000039202A92A462046984710B070BD00BF0A
:1085D000E4050020783A010038B50546007C0828FB
:1085E000144604D101236B600024204638BD92B2AA
:1085F00000F052FB0028F5D0F7E7000008B5017C39
:10860000082903D0024800F00BFD08BD0020FCE75C
:108610002706002007B501220DF10701007C00F0BC
:108620007DFB0028CCBF9DF807004FF0FF3003B062
:108630005DF804FB08B512B2007C00F06FFB08BDCA
:10864000036813B59B680446984740B10DF10701D4
:10865000207C00F091FB9DF8070002B010BD4FF0A8
:10866000FF30FAE7007C00F095BB000000214FF4DA
:108670007A72C0E90112024A02600822027470474D
:1086800008380100017C082906D04901083101F0B1
:10869000F801032000F03ABC002070472DE9F84FA4
:1086A0000E46017C08290446174609D00A2259487B
:1086B00003F050FD5849574803F0EAFC002099E0C8
:1086C0005448DFF86CA1DFF84C9103F0D1FC002591
:1086D0005FFA85FB4FEA4B11083101F0F8010320E6
:1086E00000F014FC51468046484603F0BAFC1022C4
:1086F0002946484603F015FD4849484603F0B1FCB9
:1087000010224146484603F027FDB8F1000F04D07F
:1087100008F0FB08B8F1180F43D1414984F810B0B4
:108720003C4803F09EFC1022217C3A4803F014FDE3
:10873000237C082BC2D03B4DDFF8D8802B88DFF894
:10874000F4A001332B8004F075F92B8853FA80F0E4
:1087500080B2B0F5806F36BF4FF4806328802B80E5
:108760002A88207C0023012100F03AFAF51C06F14A
:10877000070915F8011F0A22404603F0EBFC514699
:10878000404603F06EFC4D45F3D1224803F070FCE7
:108790003A46311D207C00F04BFA30B9082323748F
:1087A0008CE70135082D93D1C2E704F043F900F5B9
:1087B0006A55064618352046FFF764FF17281BD078
:1087C000AE4219D204F036F985421AD90A2004F0D3
:1087D0004BF9FCF7D9FC2046FFF754FF0028DDD009
:1087E0002046FFF74FFF1728E5D10F49094803F04E
:1087F0004FFC0120BDE8F88F04F01CF90028E5DBF0
:10880000E0E70A49034803F043FC236820465B6A1B
:10881000984753E7B0060020CF370100E237010048
:10882000EB37010006000020F43701009F370100FC
:10883000DE370100DC32010038B50446007C082830
:1088400026D000F021FA04F0F5F805462046FFF79F
:1088500019FF48B104F0EEF8401BB0F57A7F03D25F
:10886000012004F001F9F1E72046FFF70BFF10B1FA
:10887000207C00F0A7F9227C064B0748002123F852
:108880001210082323740549BDE8384003F000BCEA
:1088900038BD00BF04060020B0060020C837010024
:1088A00010B5037C082B044616D0FFF7EBFE182802
:1088B00006D80A4B23FA00F0C04300F0010010BDB7
:1088C0001C2807D1236820469B689847003018BFB2
:1088D0000120F4E70120F2E70020F0E70100100199
:1088E00007B5002300931A461946034803F070FBAE
:1088F00003B05DF804FB00BF1406002003681B6B87
:1089000018470000024A02608A694260704700BF4F
:10891000783A0100808B7047008C704713B502AB2A
:10892000026803F8011D546819460122A04702B0ED
:1089300010BD10B50446238C23B123682046DB68A4
:108940009847F8E710BD000010B50446007C0828E1
:1089500008D000F037F9227C034B002123F81210D5
:108960000823237410BD00BF040600200023C38326
:108970000431007C00F02CBA007C00F041BA10B544
:1089800093B204460A46C18B007C00F005FAE38BE3
:108990000344E38310BD13B5038C04461BB94FF0A9
:1089A000FF3002B010BD01220DF10701007C00F084
:1089B000B5F90028F3DD238C9DF80700013B2384E3
:1089C000EFE710B5038C044613B94FF0FF3010BD2C
:1089D000934294BF1AB212B2007C00F09FF90028B3
:1089E000F3DD238C1B1A2384F1E707B5038C4BB10D
:1089F0000DF10701007C00F0BFF99DF8070003B0FE
:108A00005DF804FB4FF0FF30F9E7000013B5036891
:108A100004465B699847217C104800F001FBD0B107
:108A200008226946207C00F079F9002813DD6946A8
:108A300004F1140003F0E0FA9DF804209DF80530DD
:108A40009DF8070003EB0223A3839DF8063000EB9B
:108A5000032080B2208402B010BD00BF2706002092
:108A6000F8B5037C082B04460E4601D00020F8BD63
:108A70000025EFB27901083101F0F801032000F080
:108A800045FA60B92774207C0828EFD0002366825D
:108A900023843246022100F0A3F80120E7E71828DA
:108AA000F0D00135082DE4D1EDE7000010B500222B
:108AB0004FF47A73C0E90123044B03600823044692
:108AC0000374143003F07CFA204610BD48380100CE
:108AD00070B590B0044604A815460E4603F070FA2F
:108AE00007A8FFF7E3FF684603F06AFA0D4902A8FA
:108AF000FFF7EAFC02A904A800F0A1FE6A4631468D
:108B000004A801F04DF8012809D12368064A1B6A20
:108B10000292019A039202A92A462046984710B071
:108B200070BD00BFE4050020783A010007B50023BE
:108B300000931A461946034803F04AFA03B05DF859
:108B400004FB00BF1C06002040010C300A46042331
:108B500000F0FC010C2000F0ABB90B4641010831DC
:108B600001F0F801184600F0D1B908B50221FFF76D
:108B7000F4FF08BD0B4641010C3101F0FC01184621
:108B800000F06EB938B50A0A05460C460421FFF715
:108B9000F1FFE2B205212846FFF7ECFF38BD08B52A
:108BA0000A460221FFF7E6FF08BD38B50A0A054666
:108BB0000C461021FFF7DEFFE2B211212846FFF735
:108BC000D9FF38BD10B5014604461022034800F015
:108BD000DAFAFF212046FFF7E2FF10BD270600204A
:108BE000F8B51F464B1E042B04460E46154619D8F1
:108BF000FFF7E8FF46EA070200212046FFF7BAFF29
:108C000055B129462046FFF7BDFF074801222146FE
:108C100000F0B9FA0120F8BD044B1988013189B27E
:108C20001980EFE70020F6E7270600202406002041
:108C300038B50B78FF2B054614460AD14B78FF2B2D
:108C40000ED18B78FF2B0BD1CB78FF2B08D10020D6
:108C500014E02BB94B781BB98B780BB9C87868B185
:108C60006CB12846FFF770FF21462846FFF79DFFAD
:108C700004480422294600F086FA012038BD204627
:108C8000FCE700BF2706002001460822014800F04B
:108C90007ABA00BF27060020B2F5006F2DE9F04137
:108CA00028BF4FF40062DFF8708004460E46154678
:108CB0002146404600F096F9032107462046FFF77B
:108CC0004CFF172801D01C281FD1AF42F0D33246E9
:108CD000214611482B4600F0DEF9202221460E489D
:108CE00000F051FA2046FFF740FFC3060FD40321DE
:108CF0002046FFF732FF06460028F3D12046FFF753
:108D000061FF35462846BDE8F0810025DFE71021E8
:108D10002046FFF744FFF5E727060020F7B5054694
:108D20000E4601461348174600F07AF904B274B9AA
:108D300003212846FFF711FF142805D020B1B0F118
:108D40001C0418BF4FF0FF34204603B0F0BDBC42F6
:108D5000A8BF3C46002CF7DD00230093324629468D
:108D6000A3B2044800F0E4F940222946014800F08B
:108D70000AFAE9E72706002013B501240A46009401
:108D800001462346024800F0D3F9204602B010BD48
:108D90002706002070470000F7B505460E4601463D
:108DA0000A481C46174600F01DF9A04204D2294685
:108DB000064800F017F9044600943B46324629461F
:108DC000024800F03DF9204603B0F0BD2706002020
:108DD00038B50B78054614462BB94B781BB98B7800
:108DE0000BB9C87840B144B12846FFF7ADFE28461C
:108DF0002146FFF7DAFE012038BD2046FCE70000DF
:108E000038B50146044620220C4800F0BCF9204643
:108E1000FFF7ABFE10F010050AD12046FFF7A5FEC4
:108E20000307F4D520461821FFF7B9FE284638BDC0
:108E300020461021FFF7B3FE0120F8E727060020A7
:108E4000024B0021187803F0C9BF00BF260600209E
:108E5000024B0121187803F0C1BF00BF2606002095
:108E6000F8B5114C114B05460F46204616460ECB61
:108E700004F03EF8FFF7E4FF290A204604F045F825
:108E8000E9B2204604F041F83946204604F03DF8A6
:108E90003146204604F039F8FFF7DAFF204604F0A7
:108EA00033F80120F8BD00BF240700202806002069
:108EB000F8B51D46134B06460F46134814460ECB15
:108EC00004F016F8FFF7BCFF310A0F4804F01DF854
:108ED000F1B20D480C4E04F018F839460A4804F077
:108EE00014F8013C6719BC4205D014F8011F304644
:108EF00004F00BF8F7E7FFF7ABFF034804F004F8C2
:108F00002846F8BD280600202407002070B5114B24
:108F1000114C05460E4620460ECB03F0E9FFFFF745
:108F20008FFF290A204603F0F0FFE9B2204603F044
:108F3000ECFF3146204603F0E8FF0021204603F015
:108F4000E4FF0546FFF784FF204603F0DDFF2846D7
:108F500070BD00BF280600202407002038B5174B3D
:108F6000174D1A7829703AB300244FF4FA601C7038
:108F700003F07AFD0121287803F008FF114803F07F
:108F8000A1FF21462046FFF7C1FF60F07F02D2B269
:108F900004212046FFF764FF65010C35EDB2022283
:108FA00029461E20FFF75CFF0134022229461F20BC
:108FB000FFF756FF082CEFD138BD00BF0800002096
:108FC000260600202407002038B520210546FFF79B
:108FD000C4FD000284B221212846FFF7BEFD2044D3
:108FE00080B238BD70B50E4600243046FFF7ECFF66
:108FF000054618B13046FFF7E7FF0446AC42F4D10E
:10900000204670BD38B526210546FFF7A6FD0002B3
:1090100084B227212846FFF7A0FD204480B238BD46
:1090200070B50E4600243046FFF7ECFF054618B138
:109030003046FFF7E7FF0446AC42F4D1204670BD4E
:109040002DE9F0410E463046242115469846BDF8DC
:109050001870FFF782FD252104463046FFF77DFD9D
:10906000284400EB042084B27101204614313C44B2
:109070003B464246A4B201F0FC01FFF719FF220A69
:1090800024213046FFF776FDE2B225213046FFF776
:1090900071FDBDE8F08107B5009313460022FFF78C
:1090A000CFFF03B05DF804FBF8B506460F461D463A
:1090B000144632B3144B15480ECB03F019FFFFF7DB
:1090C000BFFE310A114803F020FFF1B20F4803F050
:1090D0001CFF39460D480D4F03F017FF6B1E661E2F
:1090E0001C44A64206D00021384603F00EFF06F8C5
:1090F000010FF6E7FFF7ACFE044803F005FF284632
:10910000F8BD1546FBE700BF280600202407002015
:1091100082B01046ADF8060049011A46BDF80600B7
:10912000BDF80830183101F0F80102B0FFF7BCBFFC
:109130002DE9F7430E4680462821304691461D46CC
:109140009DF82870FFF709FD000284B229213046FE
:10915000FFF703FD0444A4B200954B462246314676
:109160004046FFF7D5FF5FB92C44A4B2220A28215C
:109170003046FFF7FFFCE2B229213046FFF7FAFC48
:1091800003B0BDE8F08310B50C4620460121FFF77F
:10919000F1FC01212046FFF7E0FC0028F9D110BDC9
:1091A000044B4FF000421A6000229A6002221A71AA
:1091B000704700BF28060020142200210E3005F061
:1091C00052BF10B50E31044602F00EFF204610BD0E
:1091D00010B51C31044602F007FF204610BD10B543
:1091E0002031044602F000FF204610BD10B52831A2
:1091F000044602F0F9FE204610BD406970478069C0
:10920000704730204B1C0870110902F00F02092A28
:1092100094BF3032373203F801290A460029F3D1CE
:109220007047000007B5002300931A46194603480B
:1092300002F0CEFE03B05DF804FB00BF3406002050
:109240002DE9F0418EB004468846164600212022C2
:1092500006A805F008FFFF231A461946009302A846
:1092600002F0B6FE04F15405574B04934322039BCE
:10927000059304A92846FFF779FB013000F0A1808F
:10928000524B069363688DF821601BBA0793330A2B
:109290008DF820301C22802306A926462846ADF8EA
:1092A0002230FFF76CFB1A2200210DF11E0005F0A1
:1092B000DAFE56F8080F0690B388ADF81C3010227D
:1092C00006A92846FFF75BFB2022002106A805F02F
:1092D000CAFE0627202206A92846FFF750FB013FB9
:1092E000F8D13B4B069340F23513ADF81C303D23CB
:1092F0008DF81F3007238DF8203001238DF82130A1
:109300003368CDF82230B388ADF8263031498DF876
:109310001E8040F60C430DF12A00ADF8283006F00F
:1093200010FEE27A0CA92046FFF76BFF227B0DF1BD
:1093300032012046FFF765FF627B0DA92046FFF74B
:1093400060FF1E2206A92846FFF719FBB8F1030F9C
:1093500028D140F23243ADF81830A37B8DF81A3093
:10936000E37B8DF81B30237C8DF81C30637C8DF8FB
:109370001D3040F23643ADF81E3094F824308DF89D
:10938000203094F825308DF8213094F826308DF86F
:1093900022300C2294F827308DF8233006A9284675
:1093A000FFF7EDFA0C4A0D4B06A9CDE90623284636
:1093B000FF2309228DF82030FFF7E1FA2846FFF756
:1093C000DBFA0EB0BDE8F081783A01000101060039
:1093D000638253638838010037060103060F3A3B66
:1093E0002DE9F0478CB005468846174603F022FB6E
:1093F00005F1540406462046FFF708FB002809DC67
:1094000003F018FB801B404500F21081322003F06E
:109410002BFBF0E7242203A92046FFF7D2FA9DF8A0
:109420000C30022B40F0FD80B5F87030432B40F03B
:10943000F880049E36BA3E60062205F108010AA8AB
:1094400005F0DEFD28B92B689E4202D36B689E4270
:1094500007D92046FFF76DFA002630460CB0BDE86C
:10946000F087079BC5F80E30CC262046FFF793FA0D
:10947000013EFAD1B04605F124092046FFF74CFA27
:10948000002840F3CF802046FFF785FA0F2800F030
:10949000818025DC032850D00FDC0028EDD0012886
:1094A00041D02046FFF777FAC7B2013FFFB2FF2F46
:1094B000E3D02046FFF76FFAF7E7062853D00C28D1
:1094C000EFD12046FFF767FAC7B2781C05F076FDAA
:1094D0003A460146A8612046FFF773FAAB6967E098
:1094E000362868D00CDC332800F08D803528D8D1A0
:1094F0002046FFF750FA2046FFF74DFAC6B2BCE708
:109500003B2873D0FF28B8D03A28CAD12046FFF7AD
:1095100042FA042205F130012046FFF752FA2B6B84
:109520001BBA2B63A9E72046FFF735FA042205F1A1
:109530001C012046FFF745FA9FE72046FFF72BFA6C
:109540000422074605F120012046FFF73AFAFFB250
:109550004FF0000A043F57458FDD2046FFF71BFA06
:109560000AF1010AF7E72046FFF715FA0422074639
:1095700005F128012046FFF724FAFFB24FF0000A58
:10958000043F57457FF779AF2046FFF704FA0AF109
:10959000010AF6E72046FFF7FEF9C7B2781C05F08E
:1095A0000DFD3A46014668612046FFF70AFA6B69ED
:1095B00003F8078061E72046FFF7EDF96B6A07467D
:1095C0008BB1494601A802F00FFDEA6E029B9A4258
:1095D00009D0FFB2013FFFB2FF2F3FF44EAF20464C
:1095E000FFF7D9F9F6E704224946A2E72046FFF73C
:1095F000D2F9042205F134012046FFF7E2F96B6B42
:109600001BBA6B6339E72046FFF7C5F9042205F161
:109610002C012046FFF7D5F9EB6A1BBAEB62AB636E
:109620002BE700262046FFF784F916E7FF2614E70C
:109630002DE9F34704464FF4FA61012003F01DF9C8
:109640002746606047F8540B3846FFF77DF9442100
:109650003846FFF705FA002800F08B8003F0EAF99E
:109660004FF00009804600254FF0030A94F850306F
:10967000032B1CD02BBB63680133636003F0DAF962
:109680004FF47A72A0EB08000121B0FBF2F2204601
:1096900092B2FFF7D5FD012384F85030002DE5D1BB
:1096A00003F0C8F9636CA0EB08009842DBD9384698
:1096B000FFF74AF9636801336360284602B0BDE8EA
:1096C000F087042B11D163680133636003F0B2F9B2
:1096D0004FF47A72A0EB08000321B0FBF2F22046AF
:1096E00092B2FFF7ADFD0223D6E7012B19D101AAF3
:1096F000A16C2046FFF774FE0228064636D1019B76
:10970000636003F097F94FF47A72A0EB080003212D
:10971000B0FBF2F2204692B2FFF792FD84F850605F
:10972000BCE7022BBAD101AAA16C2046FFF758FE74
:109730000528064615D1E36A84F850A013B94FF402
:109740006173E362236B13B9E36A5B082363D4E9B3
:109750000C320AB95A006263A363636BE3630125A9
:1097600084E7062802D184F8509097E7FF2EFAD0BC
:1097700094E70546A1E7F8B500250F460446C0E981
:109780000B554563C0E91052836485608581FFF7FE
:1097900013FD3B68A360BB88A38184F8505020462A
:1097A000BDE8F840FFF744BF38B5044603F042F97E
:1097B0000546206C00283ED0E26CA91A17D44FF45D
:1097C0007A7005F57A7291FBF0F300FB1311521ACF
:1097D0000133E264A26B59008A42ACBFD21A002264
:1097E000A263E26B9142CCBF0023D31AE36394F8E7
:1097F0005030032B1DD1A36B002B1ADC042384F8FB
:1098000050302046FFF714FF013094F85030032BFE
:1098100000D063B9E36B002B09DC002384F85030DF
:109820002046FFF7C9FC2046FFF702FF03302564FE
:1098300038BD0020E9E705F57A73E364F7E74B6884
:10984000436000230381704730B50139084610F8A2
:10985000013F002BFBD11C460A2511F8010F70B106
:10986000032C14DC2E2806D1FF2B10DC1019013438
:1098700003710023F1E7303805FB0303EDE7FF2B0D
:1098800004DC032C02DC22440120137130BD0020D3
:10989000FCE7000007B5002300931A461946034869
:1098A00002F096FB03B05DF804FB00BF3C0600200D
:1098B0002DE9F74305460E4603F0BCF805F10C040C
:1098C000288105F10801022202AD2046FFF757F872
:1098D000012325F8023D022229462046FFF74FF8D2
:1098E0004FF48073022229462046ADF80630FFF778
:1098F00046F80023022229462046ADF80630FFF73D
:109900003EF8022229462046FFF739F8022229466E
:109910002046FFF734F837463378E3B13E46B04689
:1099200018F8013B0BB12E2B13D1A6EB0709B9F1A7
:10993000000F0CDD01220DF1050120468DF8059088
:10994000FFF71DF84A4639462046FFF718F8474604
:10995000E2E74646E3E702A9012201F8033D20467B
:10996000FFF70DF84FF48076294602222046ADF825
:109970000660FFF704F8022229462046ADF806608B
:10998000FEF7FDFF012003B0BDE8F0832DE9F043B1
:1099900087B006460F46904603F04CF806F10C04DB
:1099A00005462046FFF732F800280BDC03F042F8AA
:1099B000401BB84200F2EA80322003F055F8FBF772
:1099C000E3FBEEE7726A73689A4240F0E280338DFF
:1099D000352B40F0DE802046FEF79EFF0B2840F33B
:1099E000DB800C220DEB02012046FEF7EAFFBDF8FA
:1099F0000E203189130A43EA0223BDF80C201BB262
:109A00009DB29142ADF8065001D1002B07DB2046F4
:109A1000FEF78FFF4FF6FC7007B0BDE8F08340F211
:109A20000F231D4005D02046FEF783FF4FF6FB7045
:109A3000F2E7BDF812301F0A47EA0327BFB2AFB9F9
:109A40002046FEF776FF4FF6FA70E5E79DF80A30FC
:109A50009BB92046FEF79FFF2046FEF79CFF20465D
:109A6000FEF799FF2046FEF796FF0135BDF810304E
:109A70005BBAAAB29BB29A4214DA01220DF10A0132
:109A80002046FEF79EFF9DF80A30002BDED09DF8A1
:109A90000A305A1E8DF80A20002BD7D02046FEF738
:109AA0007AFFF4E70026B14601220DF105012046B8
:109AB000FEF787FF9DF8053013F0C00F0AD193B170
:109AC0009DF805305A1E8DF8052043B12046FEF75B
:109AD00062FFF5E72046FEF75EFF8DF805909DF8E2
:109AE0000530002BE0D1022202A92046FEF769FFD3
:109AF00002220DF10A012046FEF763FF2046FEF721
:109B00004AFF2046FEF747FF2046FEF744FF204667
:109B1000FEF741FF02220DF106012046FEF751FF3C
:109B2000BDF80830B3F5807F18D1BDF80A0040BAFF
:109B300085B2012D12D1BDF8062052BA92B2042A84
:109B400005D02046FEF7F5FE4FF6F77064E708F102
:109B500004012046FEF735FF28465DE70025BDF8E5
:109B600006305BBAAAB29BB29A4205F1010503DA4C
:109B70002046FEF710FFF2E70136B6B2B74293D1A6
:109B80002046FEF7D6FE4FF6F67045E74FF6FF701B
:109B900042E74FF6FE703FE74FF6FD703CE70000EE
:109BA0002DE9F341054688461746FFF74DFE04466A
:109BB00000283BD1204B6A685B689A4238D002F09B
:109BC00039FF05F10C0600F00F0101F58061304608
:109BD000FEF746FF01281CD1184B009335226B6815
:109BE000019369463046FEF7C1FE78B141462846EA
:109BF000FFF75EFE50B13046FEF7BEFE30B13A468A
:109C000041F288312846FFF7C1FE04463046FEF790
:109C10009BFE0B490B4802F024FA0A222146094810
:109C200002F081FA204602B0BDE8F0810124F9E794
:109C30006FF00104F6E700BF3C060020783A01000F
:109C40008F380100B0060020006903681B691847BF
:109C5000006903685B69184713B5006949680368C0
:109C6000034C01919B6900946946984702B010BD6E
:109C7000783A010000690368DB69184700690368E6
:109C80009B6A18470069003018BF01207047006CBC
:109C900070470164704710B590F83830044633B906
:109CA00020690368DB689847002808DA10BD03685C
:109CB0009B6898470028F3D14FF0FF30F6E794F8FF
:109CC0002220A2F10803022BF0D8A36A002BC2BF06
:109CD000E36A0133E3620A2AE8D1E36B013BE36301
:109CE000002BE3D1092384F82230DFE710B50446C6
:109CF000006903681B6A984794F82230083B022BDE
:109D000007D8A36A002B04DD0028A2BFE36A1B1852
:109D1000E36210BD73B590F82230092B04460ED1D2
:109D20000026206903689B68984740B12069036852
:109D3000DB689847C5B20A2D1CD184F8225094F8EC
:109D400022300A2B04D1E36B13B9092384F82230A3
:109D500094F82230092B22D0206903689B68984729
:109D600094F822300A2B03D1E36B9842A8BF18461F
:109D700002B070BD0D2DD4D0284605F0EBF80028B8
:109D8000CFD0E06BADF8046010228DF804500021B4
:109D9000050101A806F03EFA2844E063C1E700206F
:109DA000E6E7000000234FF0FF32C0E90A23084A2B
:109DB00080F8223012680263064A4362126880F813
:109DC0003830C36347F2305342630364704700BFC7
:109DD000100000201400002038B504461D46002065
:109DE0004FF47A73C4E901030B4B2360C4E90412F6
:109DF00004F1180002F0E4F80123258484F84430CB
:109E000084F84530054904F1480002F09EFD2046E3
:109E1000FFF7C8FF38BD00BFF4380100CE3901009C
:109E200010B50446006903685B6A98472046BDE8A0
:109E30001040FFF7B7BF012380F8223070470000C1
:109E400038B504460069154602F00BF9044920694B
:109E500002F007F929462069BDE8384002F018B938
:109E6000DF37010038B504460D460069114602F09F
:109E7000F8F81D49206902F0F4F82946206902F03B
:109E8000F0F81A49206902F003F994F84530F3B16B
:109E90006369B3B11649206902F0E3F8D4E904011B
:109EA00002F0DFF8238C502B08D01249206902F011
:109EB000D8F80A22218C206902F033F9206902F0D7
:109EC000D7F80D4B0D491A682046FFF7B9FF94F8F3
:109ED000443023B10A4A0B492046FFF7B1FF012362
:109EE00084F82230002038BDB8380100BA380100AB
:109EF000C4380100232F01000C000020CB380100E2
:109F0000D6380100DC38010038B504460069154632
:109F100002F0A7F80549206902F0A3F82946206954
:109F20000A22BDE8384002F0FEB800BFDF3701006A
:109F300010B50446006902F09BF8022384F8223031
:109F400010BD70B590F82230012B04460D46164620
:109F500001D8FFF7EDFF20690368324629465B68A8
:109F6000BDE87040184770B590F82230012B0446C8
:109F70000D4601D8FFF7DCFF2069036829461B68FE
:109F8000BDE87040184710B50446206903689B6817
:109F9000984720B120690368DB689847F5E710BD52
:109FA0002DE9F347994690F82230083B022B0446EE
:109FB0000E469246DDE90A7804D8FFF7E4FF204612
:109FC000FFF7F0FE94F82250012D44D894F8443065
:109FD00063B1D4E90401228C0368002934D12149FA
:109FE0000091E16901919B6969462EE0206903684F
:109FF0009B6A98470028ECD0314652462046FFF72E
:10A0000031FF0646E0B9B9F1000F04D04A461649BF
:10A010002046FFF715FF002F20DD3A461349204662
:10A02000FFF772FFB8F1000F18D001252046FFF7A7
:10A030007FFF2DB123683A465B684146204698472A
:10A04000304602B0BDE8F087DB6998470028D3D1DD
:10A050004FF0FF36F4E76FF00106F1E7002DEFD186
:10A06000E4E700BF783A010094380100A13801000C
:10A0700090F82230012B01D8FFF75ABF7047FFF745
:10A08000F7BF000007B500234FF0FF32CDE90023F2
:10A09000024AFFF785FF03B05DF804FBE7380100D3
:10A0A0002DE9F04790F82230012B044651D9DFF812
:10A0B000D8800025032700236362022384F822301E
:10A0C00002F0B8FC464682464FF00A090A2D46D0F7
:10A0D00002F0B0FC236CA0EB0A00984245D2236842
:10A0E00020469B68984748B323682046DB6898471A
:10A0F000431C0546ECD094F82230022B05D0032BEC
:10A100000FD002F097FC8246E0E733782A2B01D08B
:10A1100083421AD17278731C0AB984F822701E46E1
:10A12000EFE7A0F13002092A95BF636A042309FB17
:10A13000032384F8223098BF6362E2E74FF47A7019
:10A1400002F092FCC2E70A2D06D16FF00300BDE8D1
:10A15000F0876FF00100FAE76FF00200F7E7636A3B
:10A16000C72B02DC652B18BF002594F82230042B86
:10A17000E9D1606AC72801DC65289CD10A2D18BF87
:10A180006FF00200E3E700BFB038010010B50368CC
:10A190000446DB68984794F82230A3F10802022AAB
:10A1A000C0B232D9052B31D0072B39D0042B54D172
:10A1B000226B137883420BD1531C2363537823B94A
:10A1C000C4E90A33052284F822200A281DD136E08A
:10A1D000636B197881420BD15A1C62635B78002B48
:10A1E000F3D1012384F83830062384F82230ECE7D9
:10A1F0001B4909688A42F7D11A4A12689342F3D17F
:10A200000D28F1D1072384F8223010BDA0F13002CF
:10A21000092AE9D8A36A0A2101FB0323A362D4E730
:10A220000A28F2D194F838309BB1092384F82230FF
:10A230000023E36394F82230083B022BE5D9042382
:10A2400084F82230064B1B682363064B1B6863634C
:10A25000DBE7082384F82230ECE70A28D5D1E9E7C8
:10A26000100000201400002038B5044602F0E2FB84
:10A27000054694F82230083B022B13D902F0DAFB92
:10A28000236C401B98420DD2236820469B68984758
:10A2900018B12046FFF77AFFE8E74FF47A7002F032
:10A2A000E3FBE6E794F82230083B022B94BF002042
:10A2B0006FF0020038BD10B590F82230083B022B39
:10A2C000044601D9FFF7D0FFA06A10BD7FB505464F
:10A2D00008460E46FFF7EFFF1649044601A802F0B4
:10A2E00034FB002C0EDD214601A802F007FB48B923
:10A2F0000021284602F029FB01A802F0E1FA2846D5
:10A3000004B070BDF36AA34209D0304602F038F9B8
:10A31000431C04D0C1B201A802F07EFBE7E7002C89
:10A3200002DD039B9C42E3D101A9284602F0B9FA61
:10A33000E2E700BFCE39010038B590F82230083B83
:10A34000022B054601D9002038BDFFF7B4FF0130CC
:10A35000F9D02846EC6AFFF7AEFF8442B4BF002074
:10A360000120F1E7FFF7E8BFFFF7E6BF07B50023DD
:10A3700000931A461946034801F02AFE03B05DF81F
:10A3800004FB00BF4406002000B55DF804FB00207C
:10A39000704700B501205DF804FB80687047C1601C
:10A3A00070472DE9F84380460D46174601EB020938
:10A3B0000C46A145A4EB050609D0D8F8003040466C
:10A3C000DB689847431C03D004F8010BF1E73E46D5
:10A3D0003046BDE8F883C368013304D1806900309A
:10A3E00018BF012070470120704743696BB1C269F3
:10A3F000012A0AD95A1C42611970C369013BC36121
:10A40000436900221A700120704700207047000045
:10A4100010B5D0E904435A1C42610A460248E118CB
:10A42000FFF7B7FF012010BD18030020C3680133F8
:10A4300010B504460ED16369B3F5FA4F0EDA2368FE
:10A440002046DB689847202806DD2368C1B25B6997
:10A4500020469847012002E00130ECD1002010BDD9
:10A460000346C068421C03D04FF0FF32DA607047E9
:10A47000196931B19A6922B1481C1861013A08780A
:10A480009A61704708B50346C068421C03D04FF07C
:10A49000FF32DA6008BDD3E90412501C5861114440
:10A4A0000148FFF774FFF5E7180300200368FF2158
:10A4B0001B68184710B5182004F080FD044618B139
:10A4C0001822002104F0CFFD204610BD70B50646CD
:10A4D0000C46D4B1237C65681B0704D4E16811B134
:10A4E0003046FFF7F3FF237C03F00F03042B03D167
:10A4F000606908B104F06AFD206808B104F066FDE7
:10A50000204604F063FD2C46E3E770BD2DE9F04FD3
:10A51000036885B0DB6805460E469847421C044632
:10A5200004D14FF0FF3005B0BDE8F08F2D2832D1B7
:10A530002B682846DB689847431C0446F1D04FF04F
:10A54000FF330093A4F13003092B4FF000070DD81F
:10A550004FF00A082B682846DB689847A0F13003C3
:10A56000303C092B08FB07470446F3D92E2C14D0A6
:10A5700024F02003452B10D0009B7B437361337C78
:10A58000022262F3030333742B6828465B69E1B24D
:10A5900098470020C7E70123D3E7384603F01CFFA4
:10A5A0002E2C8046894639D12B68DFF818B1DB683C
:10A5B00028469847002704464FF0000A52465B465B
:10A5C0004046494603F072FF80468946A4F13000B8
:10A5D00003F002FF42464B4603F0B2FD2B68804673
:10A5E000DB68284689469847A0F13003092B07F11C
:10A5F000FF370446E2D924F02003452B2AD12B68EB
:10A600002846DB6898472B28044609D12B68284642
:10A61000DB68984704464FF0010A0AE00027EAE7A2
:10A620002D28F8D12B682846DB6898474FF0FF0AA1
:10A6300004464FF0000B0A22A4F13003092B0DD879
:10A6400002FB0B3B2B680392DB6828469847039A72
:10A650000446F1E74FF0010A4FF0000B009803F0B9
:10A66000BBFE42464B4603F021FFCDE900015846B0
:10A6700003F0B2FE80465046894603F09DFE024636
:10A680000B464046494603F011FF8046384689464E
:10A6900003F0A2FE02460B464046494603F050FD39
:10A6A00002460B460020074902F070FC02460B46AA
:10A6B000DDE9000103F0FAFE04F0F0F9337C70618B
:10A6C00003225EE70000244019B10A22496901F023
:10A6D00006BD084670470000F8B506462DED028B12
:10A6E000D1B391ED058A18EE100A03F087FEB5EE9E
:10A6F000C08AF1EE10FA04460D4606D51A493046D6
:10A7000001F0AFFC05F100431D462946204604F048
:10A71000A5F90A2201460746304601F00EFD13490D
:10A72000304601F09EFC384603F046FE02460B46DA
:10A730002046294603F002FD09A3D3E9002303F0D4
:10A74000FFFC00220A4B03F0B1FE04F087F90A2255
:10A750000146304601F00AFDBDEC028B0020F8BD39
:10A760009A9999999999A93FB33E0100DC32010069
:10A7700000002440F8B50368DB6806460F4698479A
:10A78000222803D04FF0FF342046F8BD3B7C042242
:10A7900062F303033B7400F003FB05460028F1D08D
:10A7A00033683046DB689847431C044611D0222C9E
:10A7B00036D01F2C34DD5C2C04D02946E0B200F0EA
:10A7C00005FBEDE733683046DB689847421C0446DA
:10A7D00003D1284600F022FBD6E7622817D007DC19
:10A7E0002F2803D05C2801D02228D9D12946E6E7BA
:10A7F0006E280FD004DC6628D2D129460C20DEE773
:10A8000072280AD07428CBD129460920D7E72946D7
:10A810000820D4E729460A20D1E729460D20CEE7B3
:10A82000284600F0DFFA00247861ADE738B50D4620
:10A830001D49044601F015FC7DB3013D15F8011FCB
:10A8400059B31F2907D9222905D05C2903D02046F6
:10A8500001F00BFCF2E75C21204601F006FC2978B0
:10A860000C2914D007D8092915D00A2911D0082994
:10A87000E4D16221EBE72229E9D003D80D29DDD10B
:10A880007221E4E72F29E2D05C29E0D0D6E76621E7
:10A89000DDE76E21DBE77421D9E72221204601F0B4
:10A8A000E4FB002038BD00BF7E3901004969FFF795
:10A8B000BDBF0368DB6810B504469847431C0AD047
:10A8C0002028236802DCDB682046F6E7C1B25B691A
:10A8D00020469847002010BD03682DE9F047DB684B
:10A8E00004460E46914698477B2803D04FF0FF3030
:10A8F000BDE8F087337C062262F3030333742046FD
:10A90000FFF7D7FF23682046DB6898477D2844D0AF
:10A910002368C1B25B6920469847FF274FF0000AC1
:10A92000FFF7C8FD05460028E0D08FB3F060204651
:10A93000FFF7BFFF29462046FFF71CFF0130D5D0A7
:10A940002046FFF7B6FF6B692B602368C5F814A09B
:10A95000DB68204698473A28C8D12046FFF7A9FF70
:10A960004A462946204600F01BF80130BED020465A
:10A97000FFF79FFF23682046DB6898472C28A846EE
:10A980004FF00007CCD07D3818BF4FF0FF30AFE755
:10A99000C8F80400C0F80880C9E70020A8E7000054
:10A9A000F7B504460D461746FFF783FF013002D185
:10A9B0004FF0FF3011E023682046DB689847431CC6
:10A9C0000646F5D02368C1B25B6920469847222E1F
:10A9D00005D129462046FFF7CDFE03B0F0BD2D2E50
:10A9E00003D0A6F13003092B04D829462046FFF7EF
:10A9F0008DFDF2E75B2E05D13A462946204600F050
:10AA00009DF8EAE77B2E05D13A4629462046FFF716
:10AA100063FFE2E76E2E17D102AE002346F8083D31
:10AA2000236804221B6931462046984704280246C1
:10AA3000BED12149304605F0C4FA0028B8D12B7C9C
:10AA40006FF303032B74C8E7662E19D1002300931C
:10AA50008DF80430236805221B6969462046984713
:10AA60000528A5D105221549684605F0AAFA00284F
:10AA70009ED12B7C2875012262F303032B74ACE773
:10AA8000742E95D102AE002346F8083D23680422B7
:10AA90001B693146204698470428024688D1084958
:10AAA000304605F08EFA002882D12A7C012363F318
:10AAB00003022A742B7590E76E3901007339010087
:10AAC00079390100F8B5064617460D4611B900243C
:10AAD0002046F8BDFFF7EEFC04460028F7D02846D4
:10AAE000FFF7E7FE3A4621462846FFF759FF0130B7
:10AAF000EED121463046FFF7E9FCE8E70022FFF7F8
:10AB0000E1BF000010B588B04FF0FF320023039280
:10AB1000094A00920446CDE901330846CDE9041301
:10AB2000079309B105F031FA069069462046FFF710
:10AB3000E5FF08B010BD00BFAC3901002DE9F843B6
:10AB40000368DB6804460F46914698475B2803D0AC
:10AB50004FF0FF30BDE8F8833B7C052262F303032E
:10AB60003B742046FFF7A5FE23682046DB68984724
:10AB70005D282BD02368C1B25B6920469847FF2629
:10AB8000FFF798FC05460028E2D0D6B1F8602046D1
:10AB9000FFF78FFE4A4629462046FFF701FF06468B
:10ABA0000028D5D12046FFF784FE23682046DB68C5
:10ABB00098472C28A846E3D05D3818BF4FF0FF30E7
:10ABC000C8E7C8F80400C0F80880E0E70020C1E743
:10ABD00038B5054651B3CC687B2101F046FA013007
:10ABE00002D14FF0FF3038BDB4B121682846FFF7DD
:10ABF0001DFE0130F5D03A21284601F036FA013029
:10AC0000EFD02146284600F013F80130E9D06468FF
:10AC100014B12C212846E0E77D21284601F025FAD1
:10AC200001304FF0FF3018BF0020DCE70846DAE7BC
:10AC3000E9B10B7C03F00F03062B18D8DFE803F013
:10AC400004070D0F111315000A4901F00ABA0B7D14
:10AC50000BB10949F9E70949F7E7FFF735BDFFF7F8
:10AC60003BBDFFF723BE00F00EB8FFF7B1BF0020D9
:10AC7000704700BF6E390100793901007339010056
:10AC80001046FFF7D5BF38B50546F1B1CC685B215A
:10AC900001F0EBF9013002D14FF0FF3038BD54B173
:10ACA00021462846FFF7C4FF0130F5D0646814B18F
:10ACB0002C212846ECE75D21284601F0D6F9013029
:10ACC0004FF0FF3018BF0020E8E70846E6E7CB6802
:10ACD0000022D0B201320BB15B68FAE77047C86856
:10ACE00020B11AB1013AD2B24068F9E7704738B5DD
:10ACF000CC68154634B12946206805F0DEF808B165
:10AD00006468F7E7204638BD4AB1CB6813B9CA601A
:10AD100070470B4659680029FBD15A609360704711
:10AD2000F8B505460E4617461C4673B1186808B1BB
:10AD300004F04CF9384605F00DF922462060314602
:10AD40002846BDE8F840FFF7DFBFF8BD10B50C4658
:10AD5000FFF7B0FB28B1037C4461022262F30303D6
:10AD6000037410BD70B50D46194604461646FFF72C
:10AD7000EDFF3246034629462046BDE87040FFF706
:10AD8000CFBF000007B5002300931A4619460348B9
:10AD900001F01EF903B05DF804FB00BF4C06002073
:10ADA00038B50C2004F00AF9044650B1064820607A
:10ADB0004FF480752A46002104F055F900236560A0
:10ADC000A360204638BD00BF50070020D1E9012311
:10ADD000934204D20A68D0548B6801338B60002000
:10ADE00070470000826838B5044622B103681344F6
:10ADF00013F8013C1BB121460020FFF7E7FFA068D4
:10AE000004F0DCF8054628B1034905F09AF820461D
:10AE100004F0DCF8284638BD5007002008B104F0E3
:10AE2000D5B8704710B5054C204601F021F92046F1
:10AE30000349BDE8104001F00BB900BFB006002087
:10AE4000C8390100F0B503789FB0044643B3194BED
:10AE5000194F1B68986803F06BFF2046164905F0F0
:10AE6000F7F81EAD012445F8780D3946002005F0AD
:10AE7000EFF81E2C264645F8240002D001340028A5
:10AE8000F3D10E4B009F1C6874B12168384605F061
:10AE90004EF838B96368294630469847FFF7C2FF35
:10AEA0001FB0F0BDA468EFE70549064801F0E6F8D9
:10AEB000F4E700BF38000020B838010098060020F1
:10AEC000CF390100B0060020F8B505460C200F462A
:10AED00004F074F80C4B04461860284605F055F849
:10AEE000013004F06BF82946064605F02AF828469A
:10AEF00005F04BF800233354044B1A68A260C4E9F0
:10AF000000671C60F8BD00BF9806002058060020AE
:10AF100070B51648164D01F091FBC4B20A2C0CD046
:10AF20000D2C0AD0082C15D12146104801F09DF8AF
:10AF30002B7873B1013B2B700BE02B780D4E0E4933
:10AF40000A480024F45401F08CF83046FFF77AFFE9
:10AF50002C7070BD2146054801F087F82B783A2BFC
:10AF60009FBF5A1C2A70034AD454F2E7B00600204F
:10AF70009C0600205C060020CC39010010B5044C72
:10AF8000204601F055FB10B1FFF7C2FFF8E710BDF6
:10AF9000B0060020044A00231370044A0146044806
:10AFA000136001F004BB00BF9C060020580600207F
:10AFB000B006002070B504460D4601F03BFDA061CF
:10AFC000A068036829461B68BDE87040184770B543
:10AFD00004460D46164601F02DFDA061A0680368E9
:10AFE000324629465B68BDE87040184710B50446F4
:10AFF000C06803F0EBFF204610BD2DE9F041054687
:10B000000E4601F017FD4FF47A778046A868036872
:10B010009B689847044658B901F048FD01F00AFDC5
:10B02000AB8AA0EB08007B439842EFD3204605E0B3
:10B03000A8680368DB68984730700120BDE8F0819C
:10B0400038B5148821441546FFF7D7FF08B10134FD
:10B050002C8038BD2DE9F74F02AD002625F8026D92
:10B060008A462A46C1680446FFF7EAFF18B900205D
:10B0700003B0BDE8F08FE3680DF1080993F8008094
:10B0800009F8036D0127BDF80630052B07D14FF0F5
:10B09000FF33A068E36303685B6A9847E7E74946C4
:10B0A0002046FFF7AAFF0028E1D0BDF80630E2688D
:10B0B000591CADF806109DF80510D1549DF80530C7
:10B0C00003F07F0207FB02661A064FEAC717DAD4BD
:10B0D0009DF8063008F0F008013BB8F1300F8AF80F
:10B0E00000301DD12A46E1682046FFF7A9FF00285D
:10B0F000BDD02A46E1682046FFF7A2FF0028B6D05F
:10B10000E2689AF80030134459789D78137805EB7B
:10B1100001259B07ADB201D50235ADB2022701E092
:10B1200000273D46BDF806B0A7EB0B0707EB0B0267
:10B1300096422AD949462046FFF75FFF002896D05D
:10B14000A06B88B1B8F1300F0ED19AF80020C2F18F
:10B15000FF2202F57F02FE325A44AA4204D9026855
:10B160009DF8051012689047BDF80620218A91428B
:10B1700008D9E1689DF805008854BDF80620013221
:10B18000ADF806200BF1010BD0E7A26B22B9218AA2
:10B19000594538BFADF80620BDF8060068E773B51D
:10B1A0000025DC1103F07F06A3B20CB146F0800647
:10B1B0000DF1080C681C6544C0B205F8046C054626
:10B1C000002CEED1C0F10405515501ADA04205DDC2
:10B1D000231A1344615D59710134F7E7013002B05D
:10B1E00070BDF8B5064617461C46FFF7D8FFB36892
:10B1F000C0B21A680444C0F10501556839442246BA
:10B200001846A847054601F015FCB061A8B2031B1B
:10B2100058425841F8BD10B5C368E0221A70C3689F
:10B2200000225A7004468068E168036802225B6865
:10B230009847A0684FF0FF33E36303685B69984762
:10B24000A06803685B6A984701F0F4FBC4E9060054
:10B2500010BD023330B598B20C46631A14F8015B86
:10B260009BB21DB1431C155498B2F6E7C11A0A44AB
:10B27000191202F8021C02F8013C30BD38B505462F
:10B28000806808B9002038BD03689B6A9847EC6B5A
:10B2900068B9002CF6D1A8686FF00203EB6303686D
:10B2A0005B699847A86803685B6A9847EAE7B4FA5D
:10B2B00084F04009E7E700002DE9FF470C9D9DF869
:10B2C00040A00446894617461E46FFF7D7FF804632
:10B2D000002840F0DF80A06803689B6A9847002838
:10B2E00040D00123E3826E4B029345F25443ADF804
:10B2F0000C3004238DF80E30052302A91944E268AE
:10B3000011F8051CD15401330C2BF6D1002D3DD082
:10B310009DF838309DF834205B0143F0040343EA84
:10B32000C203DBB2BAF1000F01D043F002031FB138
:10B33000002E2DD143F08003E2681373638AE26824
:10B340001B125373E368628A9A73218A484604F099
:10B350005FFE238A113098421DD9A06803685B6A9A
:10B36000984797E0A068216B0368A28E39B1DB692A
:10B3700098470128B5D06FF00103E3638AE049499B
:10B380009B690291E16A039102A9F1E72B46C9E7A3
:10B3900043F0C003D0E749460F23E2682046FFF799
:10B3A00058FF814605B3218A284604F031FE09F191
:10B3B00002031844238A9842CFD84B462946E268B4
:10B3C0002046FFF746FF218A05460F9804F020FE2D
:10B3D000238A023028449842BFD82B46E2680F994E
:10B3E0002046FFF736FF814617B3218A384604F01E
:10B3F0000FFE09F102031844238A9842ADD84B4648
:10B40000E26839462046FFF724FF814686B1218A4B
:10B41000304604F0FDFD09F102031844238A9842E6
:10B420009BD84B46E26831462046FFF712FF814623
:10B43000A9F105039BB2E26810212046FFF7D1FE77
:10B4400001F0F8FAC4E906004FF47A75A0680368C1
:10B450009B68984758B901F0EDFAE369C01AA38ACE
:10B460006B439842F2D36FF00303E36375E70DF18A
:10B4700007012046FFF7EEFD04287FF46EAFE36876
:10B48000DD785DB901F0D6FA4FF00108E06184F88B
:10B490002050E563404604B0BDE8F087E5635CE713
:10B4A00000044D51783A010010B586B0012404948F
:10B4B0000B9C03949DF8284002949DF8244001942D
:10B4C000089C0094FFF7F8FE06B010BD2DE9F34785
:10B4D0000446FFF7D3FE8046D0B101F0ABFA628A92
:10B4E0004FF47A735343E269821A9A42074603D8AB
:10B4F000A269821A93421FD294F8203063B16FF090
:10B500000303A068E36303685B6A98474FF0000891
:10B51000404602B0BDE8F087E268C0211170E268E1
:10B520005370A068E168036802225B689847C4E929
:10B530000677012384F82030A06803689B68984749
:10B540000028E5D00DF107012046FFF783FD83B207
:10B550000646002B73D0E368E7611A7802F0F00228
:10B56000302A57D1626A002AD2D09DF80720991854
:10B57000901C49781D5C05EB0125ADB2D11C194426
:10B580002A46184403F056FDE3689DF807202B4433
:10B59000134400229A70E1689DF807C091F800906A
:10B5A00009F00609B2B20CF10200B9F1020F084429
:10B5B000666A0CF10303A2EB0C0225D12B440CF1BB
:10B5C000050C11F803E00B44521B93F801A06544ED
:10B5D000053A29440AEB0E2AB047E36840221A7064
:10B5E000E36883F80190E3681FFA8AFA4FEA2A2297
:10B5F0009A70E36883F803A0A068E16803680422F6
:10B600005B689847A76183E72B44033A521B1944B0
:10B61000B0477DE7C02A0BD1D0221A70E368002220
:10B620005A70A068E168036802225B6898476FE778
:10B63000D02A7FF46DAF002384F8203068E72046DD
:10B64000FFF71CFE002808BF4FF0000860E72DE957
:10B65000F0470446884617461D469DF82060FFF7D0
:10B660000DFE50B3B4F810904046494604F0D0FCAB
:10B67000EB1D1844814520D341460523E26820464E
:10B68000FFF7E7FD00211FFA81FC4318AC459BB290
:10B69000E26801F1010104D217F80CC002F803C0FE
:10B6A000F1E7002EA3F1050320469BB214BF312120
:10B6B0003021BDE8F047FFF794BD0020BDE8F087DA
:10B6C00073B505460E4614466AB1018A104604F069
:10B6D0009FFC034600220092314622462846FFF78F
:10B6E000B6FF02B070BD1346F4E7F7B505460E4647
:10B6F0001F46144662B1018A104604F089FC0346D5
:10B700000097224631462846FFF7A1FF03B0F0BD5F
:10B710001046F4E770B50D460446018A28461646E1
:10B7200004F076FC45B3012E26D8238A09308342E3
:10B7300022D32046FFF7A2FDF0B1E38A01339BB28A
:10B74000C3B1E382E38AE2681B125371E368E28AC1
:10B750009A71E268294607232046FFF77AFDE368DD
:10B760001E54031FE26820469BB28221BDE8704050
:10B77000FFF737BD0123E4E7002070BD0022FFF78B
:10B78000C9BF70B50D460446018A284604F040FC46
:10B7900025B3238A0930834220D32046FFF76EFD6C
:10B7A000E0B1E38A01339BB2B3B1E382E38AE2689A
:10B7B0001B125371E368E28A9A71E26829460723F3
:10B7C0002046FFF746FD431FE26820469BB2A221B8
:10B7D000BDE87040FFF705BD0123E6E7002070BD1E
:10B7E00001638286704741627047C06B704738B50D
:10B7F00004460D4609B9002038BD038A4BB90846F6
:10B8000003F0DCFBE060E0682582003018BF012017
:10B81000F2E7C06804F096FA0028F3D1EBE70000E5
:10B8200070B50C4B00250446456040F8283B0E4699
:10B8300000F0C6FB4FF0FF33E363A660A5632582EB
:10B840004FF480712046FFF7D2FF0F236382A3825B
:10B85000204670BDE839010007B5002300931A4661
:10B860001946034800F0B4FB03B05DF804FB00BFC9
:10B87000A00600208271054A417112680449B2FB9A
:10B88000F1F14FF47A724A43C26070471800002009
:10B8900040420F0038B504460D464079022101F0C0
:10B8A00075FA01F0C7F8A0F5FA60A060657438BDBC
:10B8B00070B505460E460024687901F0A1FAB04241
:10B8C000A3B206D1EA689A4204F10104F4D84FF019
:10B8D000FF33184670BD30B50D46D1B0044601F0B7
:10B8E000A9F83DB9A368C31AB3F5FA6F02D2207C58
:10B8F00051B030BD00250221A0602560607925711E
:10B9000001F044FA012001F0AFF80121607901F063
:10B910003DFA2946607901F061FAA379153B012BC4
:10B9200000F28C8040F24C40013800BF00BF00BFE5
:10B9300000BF00BF00BF00BF00BF00BF00BF00BF0F
:10B9400000BF00BF00BF00BF00BF00BF00BF00BFFF
:10B9500000BF00BF00BF00BF00BF00BF00BF00BFEF
:10B9600000BF00BF00BF00BF00BF00BF00BF00BFDF
:10B9700000BF00BF00BF00BF00BF00BF00BF00BFCF
:10B9800000BF00BF00BF00BF00BF00BF00BF00BFBF
:10B9900000BF00BF00BF00BF00BF00BF00BFC3D1DA
:10B9A0006079022101F0F2F9607C00283BD0013877
:10B9B00000BF00BF00BF00BF00BF00BF00BF00BF8F
:10B9C00000BF00BF00BF00BF00BF00BF00BF00BF7F
:10B9D00000BF00BF00BF00BF00BF00BF00BF00BF6F
:10B9E00000BF00BF00BF00BF00BF00BF00BF00BF5F
:10B9F00000BF00BF00BF00BF00BF00BF00BF00BF4F
:10BA000000BF00BF00BF00BF00BF00BF00BF00BF3E
:10BA100000BF00BF00BF00BF00BF00BF00BF00BF2E
:10BA200000BF00BFC3D172B600212046FFF740FF20
:10BA3000013007D10020207462B659E7142001F0CC
:10BA400013F8ADE701212046FFF732FF0130F1D0B6
:10BA5000002500212046FFF72BFF01214DF80500AE
:10BA60002046FFF725FF0DEB05030835B5F5A07F50
:10BA70005860EED162B600225DF832500DEBC20381
:10BA8000691C586801D0431C02D1002020742FE7A4
:10BA9000D1108542635C4FEA4303DBB202F101023D
:10BAA00038BF43F00103282A6354E5D16178237835
:10BAB00022790B44A1780B44E1780B44DBB29A4223
:10BAC000E3D10120E2E700002DE9F8430D462DED1A
:10BAD000028B11460446FFF7FEFE00287ED0A379B4
:10BAE0000B3B0B2B7AD8DFE803F0063F79797979A5
:10BAF000797979796565A378E07808EE103A0106DE
:10BB0000B8EE488A48BFFFEE007A00F00F0048BF49
:10BB100037EEC88A02F060FC31A3D3E9002302F0BB
:10BB2000C5FC064618EE100A0F4602F067FC0B46ED
:10BB300002463946304602F003FB02F0AFFF0346EF
:10BB40006DB102F05BFC2AA3D3E9002302F0AEFC46
:10BB5000254B002202F0F4FA02F0A0FF0346BDECF0
:10BB6000028B1846BDE8F883E078A67800F00F0055
:10BB700002F032FC1AA3D3E9002302F097FC07EE8F
:10BB8000906AF8EE677A804617EE900A894602F0CE
:10BB900035FC02460B464046494602F0D1FA02F017
:10BBA0007DFF3206034648BF80F00043002DD6D00B
:10BBB0001846C6E7A678E378300200F4FE40184342
:10BBC00007EE900AF8EEE77A17EE900A02F016FCFC
:10BBD00003A3D3E9002302F069FCE0E7034BBEE7CF
:10BBE0009A9999999999B93F000040400000C07F07
:10BBF000CDCCCCCCCCCCFC3FD0B50446FFF76BFE13
:10BC000090B3A3790B3B0B2B2ED8DFE803F006068D
:10BC10002D2D2D2D2D2D2D2D1C1C607802F0DCFBE3
:10BC200014A3D3E9002302F041FC064620780F4616
:10BC300002F0D2FB02460B463046394602F080FA4B
:10BC400002F02CFFD0BD208840BA80B207EE900AE7
:10BC5000F8EEE77A17EE900A02F0D0FB05A3D3E9DD
:10BC6000002302F023FCEBE70148EBE7AFF3008091
:10BC70000000C07F9A9999999999B93F10B50446E7
:10BC8000C06803F0A3F9B4F90600002802DB002124
:10BC900001F07CF8204610BD70B50546C0680E4620
:10BCA00003F094F9EC7C2A7C94420CBF0324042416
:10BCB00014FB06F4A4B2AC80204603F07FF9E860E0
:10BCC00028B12246002103F0CEF96E8070BDA88015
:10BCD0006880FBE7F0B4FF29C1F38107C1F381124B
:10BCE000C1F30115477401F003078CBF0021012146
:10BCF0000170C168C47C067CC2740574877461B12C
:10BD0000A41B6142A2EB050561416A426A4191426E
:10BD100003D04188F0BCFFF7BFBFF0BC704738B517
:10BD2000437804460D4633B1B0F90600002802DB23
:10BD3000002101F02BF86378E5804BB12846012102
:10BD400001F024F828460021BDE8384001F046B84B
:10BD500038BD70B50E460021044641700172C160C5
:10BD6000416119461546FFF7B5FF31462046FFF7FA
:10BD700093FF20462946FFF7D2FF204670BD70B5DD
:10BD800040F2FA5404FB00F303F500431B14B3F52F
:10BD9000FF7F98B222DAFE2BD8B242DDC0F1FE005E
:10BDA000C5B20023FF204E1CC943C9B27043013203
:10BDB00001EB2020504300F47F4406FB03F006FB18
:10BDC00005F301EB202001EB232150434A431202EB
:10BDD00044EA102002F47F02104370BDB3F57F7F68
:10BDE0000DDAB0F53F7FDBB28BBFC3F1FC0302334A
:10BDF000D8B2DBB294BFFF20FF230025D3E7A042D7
:10BE000011D040F2FA44A042DBB204D80433DDB2D0
:10BE10000020FF23C7E7C3F1FA03DBB20020FF25B0
:10BE2000C1E70023FBE700231846F8E770B5044696
:10BE3000083015460E4600F0C3F8FF23064A84F882
:10BE400022300023266025712361A382C4E90622E3
:10BE50002384204670BD00BFB33E01000161828291
:10BE600070470000024B002908BF194681617047E6
:10BE7000B33E0100024B002908BF1946C16170475B
:10BE8000B33E01000184704773B50D460169044655
:10BE9000164639B92B4BC2685B689A4202D1002022
:10BEA00002B070BDA28A002AF9D094F8223005F0C1
:10BEB00007000341DB0738D515F47E7F08BF238CCC
:10BEC000206804BF03F47E731D43036800292ED04D
:10BED0005B6A98470128E2D13C21206800F0C5F850
:10BEE0000A222946206800F01CF9237933BB164941
:10BEF000206800F0ADF8A169206800F0B2F82021B8
:10BF0000206800F0B2F8E169206800F0AAF823790F
:10BF1000B3B90E49206800F09BF83146206800F064
:10BF2000A0F8206803689B6A98470120B8E7084991
:10BF30000091E16801911B6A6946CAE70549D7E7A4
:10BF40000549E7E7A8060020F0390100F6390100AD
:10BF5000783A010011260100013A010008B5FFF707
:10BF600093FF08BD07B5002300931A4619460348FE
:10BF700000F02EF803B05DF804FB00BFA806002017
:10BF80002DE9F84306460D46071D00F10709002478
:10BF900017F8011B0A22284600F0DCF82E21804603
:10BFA000284600F062F84F4540440444F0D10A228C
:10BFB000F179284600F0CEF82044BDE8F88300006F
:10BFC000024A026000224260704700BF783A0100D6
:10BFD00030B58371034D9DF80C30056001714271DD
:10BFE000C37130BD783A0100024A02600A684260BB
:10BFF000704700BF783A01000B68436070472DE935
:10C00000F04106460D4601EB02080C464445A4EB00
:10C01000050707D0336814F8011B1B6830469847A2
:10C020000028F3D13846BDE8F08170B504460846D3
:10C030000D4603F0AAFF23680246294620465B68A6
:10C04000BDE87040184709B1FFF7EFBF08467047D9
:10C0500008B5FFF7F8FF08BD03688A685B680968E0
:10C06000184708B5FFF7EFFF08BD03681B681847BE
:10C070000149FFF7DABF00BFCC39010038B50546EA
:10C08000FFF7E1FF04462846FFF7F2FF204438BDE2
:10C0900038B50546FFF7D7FF04462846FFF7E8FF07
:10C0A000204438BD70B58AB00D460AA9002301F8B6
:10C0B000043D012A98BF0A22B5FBF2F402FB145694
:10C0C000F3B2092E94BF30333733DBB2254601F883
:10C0D000013D002CF0D1FFF7B6FF0AB070BD2DE98D
:10C0E000F04107460E4615462AB90368C9B21B68D7
:10C0F000BDE8F04118470A2A05D1002905DBBDE853
:10C10000F041FFF7CFBFD2B2F9E72D21FFF7ADFF26
:10C110002A46044671423846FFF7C4FF2044BDE872
:10C12000F081FFF7DCBF38B50546FFF7D8FF0446BE
:10C130002846FFF79DFF204438BD10B42AB9036894
:10C140005DF8044B1B68C9B21847D2B25DF8044BC6
:10C15000FFF7A8BFFFF7F1BF38B50546FFF7EDFFC2
:10C1600004462846FFF784FF204438BDFFF7E5BFAB
:10C170002DE9F84F19460646104614461D469DF80F
:10C18000287002F02DFC28B14C493046BDE8F84F2C
:10C19000FFF74BBF25F000494FF0FF32484B2046D8
:10C1A000494602F01DFC48B94FF0FF32444B20468F
:10C1B000494602F0F7FB08B94249E6E74FF0604212
:10C1C000414B2046294602F001FC08B13F49DCE71B
:10C1D0004FF060423E4B2046294602F0D9FB002832
:10C1E000F4D1002200232046294602F0D1FBD0B131
:10C1F0002D213046FFF739FF05F1004382461D46E9
:10C200003449DFF8D8904FF0000B00204FF00008C1
:10C210005FFA8BF39F4208D942464B4602F070FA10
:10C220000BF1010BF4E78246EAE722462B4601F0C8
:10C2300087FF0D46044602F011FC0A2201468046A3
:10C240003046FFF72FFF8244A7B3404602F0B4F810
:10C2500002460B462046294601F070FF04460D4673
:10C2600030461D49DFF87490FFF7DFFE4FF00008FD
:10C270008244013FFFB2FF2F1CD04B46424620466E
:10C28000294602F013F90D46044602F0BFFB0A22CC
:10C29000014683463046FFF722FF8244584602F0AB
:10C2A0009BF802460B462046294601F047FF04460C
:10C2B0000D46DEE75046BDE8F88F00BF7C3A01002E
:10C2C000FFFFEF7F803A0100FFFFEF41843A01005A
:10C2D000FFFFEFC10000E03FDC320100000024401E
:10C2E0009DF800100091FFF743BF08B540220021E0
:10C2F00002F0B9FE0022C0E9102208BD026C10B5A0
:10C30000531C446C03F03F039C421CBF81540364E4
:10C3100010BD0023C0E910337047D0E910239342C9
:10C320001FBFC25C013303F03F03436414BF1046D8
:10C330004FF0FF307047D0E91030181A48BF403036
:10C340007047D0E91023934214BFC05C4FF0FF3018
:10C350007047036C406C013303F03F031B1A5842D3
:10C36000584170470649074A074B9B1A03DD043BB7
:10C37000C858D050FBDC00F04DF8F4F761F800002D
:10C38000C43E01000000002088020020FEE7FEE716
:10C39000FEE7FEE7FEE7FEE7FEE7FEE7FEE7FEE775
:10C3A000094B1B78062B0CD1084B1B681A0708D1C8
:10C3B000074B186800F0F000A0F1300358425841D4
:10C3C00070470020704700BFE00F00F0E40F00F05E
:10C3D000E80F00F00C4B1B78062B10D10B4B1B68A1
:10C3E0001A070CD10A4B186800F0F003302B08D064
:10C3F00000F0E000A0F1400358425841704700208F
:10C4000070470120704700BFE00F00F0E40F00F01C
:10C41000E80F00F008B5FFF7C3FF10B14A4B4B4AD5
:10C420001A60FFF7D7FF28B1494B4A4A1B68C3F38C
:10C4300042331360FFF7B4FF20B1474AD36823F0BB
:10C440008073D360FFF7C6FF40B14FF080430022F6
:10C45000C3F80C21C3F81021C3F83825FFF7A0FF5B
:10C4600010B13E4B03221A60FFF79AFF40B13C4BDC
:10C4700005221A6001229A6700229A603F225A60C0
:10C48000384B1B78062B50D1374B1B681B074CD100
:10C49000364B1B6803F0F003502B46D14FF080520F
:10C4A000334BD2F80414C3F82015D2F80814C3F89B
:10C4B0002415D2F80C14C3F82815D2F81014C3F8B8
:10C4C0002C15D2F81414C3F83015D2F81814C3F888
:10C4D0003415D2F81C14C3F84015D2F82014C3F850
:10C4E0004415D2F82414C3F84815D2F82814C3F818
:10C4F0004C15D2F82C14C3F85015D2F83014C3F8E8
:10C500005415D2F83414C3F86015D2F83814C3F8AF
:10C510006415D2F83C14C3F86815D2F84014C3F877
:10C520006C15D2F84424C3F87025124AD2F888302A
:10C5300043F47003C2F88830BFF34F8FBFF36F8F9F
:10C540000D4B0E4A1A6008BD74C007400DF0ADBA1D
:10C55000440200103C050040F0ED00E0A005004062
:10C5600010560040E00F00F0E40F00F0E80F00F07C
:10C5700000C0004000ED00E0180000200090D00353
:10C5800010B5044600F056FAE06023682046DB68E8
:10C590009847002808DA00F04DFAE368C01AA3684B
:10C5A0009842F2D34FF0FF3010BD0120704703686E
:10C5B0001322DB69184770470369C3F81C15036928
:10C5C000D3F81C21002AFBD00022C3F81C21012033
:10C5D0007047000010B490F95C30144C59090122E6
:10C5E000203103F01F0302FA03F344F821300369FA
:10C5F0005DF8044B0421C3F8081303695A6003690A
:10C60000DA6003690022C3F8002502694FF0FF33A6
:10C61000C2F80C350269C2F814350269C2F808354F
:10C6200002691430C2F81035FFF773BE00E100E074
:10C630001430FFF780BE1430FFF783BE1430FFF7CD
:10C640006CBE0000036990F85E2010B5C3F80C259D
:10C65000036990F85D20C3F8142590F86120036900
:10C66000012A01BF90F85F40C3F81045036990F8B4
:10C67000604006BFC3F8084503690022B1F5966F14
:10C68000C3F86C2569D9B1F5166F69D9B1F5965F14
:10C6900069D9B1F5165F68D9B1F5615F67D9B1F5B0
:10C6A000964F66D9B1F5E14F65D9B1F5164F64D90A
:10C6B000B1F5614F64D9B1F5963F64D9B1F5E13F69
:10C6C00063D9B1F5613F63D9364B994263D9B1F56E
:10C6D000E12F63D9B1F5612F94BF4FF070634FF034
:10C6E00080530269C2F8243503690422C3F8002587
:10C6F00001690023C1F808310169C1F81C310169E1
:10C7000001230B6001698B600169C1F8042390F972
:10C710005C20510902F01F0293406031224A42F826
:10C72000213090F95C30002BBDBF03F00F0302F6FF
:10C73000FC32D2189B18B5BF60236022137683F8B1
:10C74000002390F95C300122590903F01F0302FA1B
:10C7500003F3154A42F8213010BD4FF49E23C0E781
:10C760004FF41D23BDE7114BBBE7114BB9E7114B4C
:10C77000B7E7114BB5E7114BB3E74FF41D03B0E733
:10C780004FF46B03ADE70E4BABE74FF0EB73A8E74D
:10C790004FF06C73A5E74FF08063A2E74FF0E863BA
:10C7A0009FE700BF90D0030000E100E000B013005D
:10C7B0000050270000F03A0000A04E0000C07500B5
:10C7C00000903A012DE9F0411E4600254FF47A739E
:10C7D000C0E901530D4B044640F8143B1746884608
:10C7E000FFF783FD0A4AC4F8108084F85C7052F8A1
:10C7F000263084F85D309DF8183052F8233084F8E4
:10C800005E3084F861502046BDE8F081903A010026
:10C81000083A010010B50369D3F8082104464AB16B
:10C82000D3F818151430C9B2FFF768FD2369002248
:10C83000C3F8082110BD00000148FFF7EBBF00BF9F
:10C84000B006002007B519230093022218230349DC
:10C850000348FFF7B7FF03B05DF804FB002000407A
:10C86000B006002010B5044628B103F037FA90FB5B
:10C87000F4F303FB1404204610BD884210B50446AF
:10C8800003DA081AFFF7EEFF0444204610BD10B586
:10C89000029C401AE41A6043521A90FBF2F01844CA
:10C8A00010BD0023C0E9003310B50C68836004603C
:10C8B0004C6844608C688460C1E900338B6010BDB3
:10C8C00010B50446006802F081FB204610BD10B58B
:10C8D0000446006808B102F079FB00232360C4E934
:10C8E000013310BD38B504460D460068013103F030
:10C8F00029FA10B1C4E90005012038BD036810B55C
:10C90000044623B143688B4201D3012010BD204669
:10C91000FFF7E8FF0028F9D0A368002BF5D12268C3
:10C920001370F2E770B50E46114604461546FFF740
:10C93000E5FF20B92046FFF7CAFF204670BDA5607D
:10C940003146206803F0FDFAF7E738B500230446C6
:10C95000C0E9003383600D4639B1084603F015FB8A
:10C96000294602462046FFF7DDFF204638BD38B590
:10C97000054600680C4668B16A688B689A4207D31E
:10C98000096803F0DEFAA368AB600023A36038BD3A
:10C9900002F01CFB23682B6063686B60A368AB60CC
:10C9A0000023C4E90033F1E7884210B50B46044682
:10C9B00004D0096821B19A68FFF7B4FF204610BD82
:10C9C000FFF785FFFAE710B500230446C0E90033FE
:10C9D0008360FFF7E9FF204610BD884210B504468A
:10C9E00001D0FFF7C4FF204610BD70B505460E46C6
:10C9F00009B9002070BD6AB1846814442146FFF76C
:10CA00007DFF0028F5D02868AB683146184403F054
:10CA100098FAAC600120EDE707B500238DF804100B
:10CA2000012201A98DF80530FFF7DFFF03B05DF8A3
:10CA300004FBFEE70A4B19680A4B30B5D3F804052E
:10CA40000C060D0A44EA00024FF47A712B46A2FB51
:10CA5000014501FB0355E00B40EA454030BD00BFF6
:10CA6000140700200010014038B5044648B1FFF714
:10CA7000E1FF054600F01AF8FFF7DCFF401BA0427B
:10CA8000F8D338BD074B0022C3F8042182B0D3F895
:10CA90000431054A0193019B13680133DBB2136033
:10CAA00002B0704700100140140700207047704723
:10CAB00008B500F017F8FFF7FAFF0120FFF7D4FFE1
:10CAC000F7F73AF9034CF7F739F9002CFBD0AFF33D
:10CAD0000080F8E70000000002F070BA02F06EBAC1
:10CAE00002F074BA2A4BE02283F811234FF400328B
:10CAF000C3F880211A604FF080430122C3F8182543
:10CB00009A6003F588330021C3F808150221C3F8A1
:10CB10000413C3F844131A604FF01023D3F8002213
:10CB2000002A03DBD3F80432002B2FDA194B012241
:10CB3000C3F80425D3F80024002AFBD04FF01022BC
:10CB40001521C2F80012D3F80024002AFBD04FF0C0
:10CB500010231522C3F804220E4B1A46D3F80014F2
:10CB60000029FBD00021C3F80415D2F80034002BB3
:10CB7000FBD0BFF34F8F0849084BCA6802F4E0624C
:10CB80001343CB60BFF34F8F00BFFDE7704700BF7B
:10CB900000E100E000E0014000ED00E00400FA05E3
:10CBA000192837B50CD84B4B53F82030052B00F023
:10CBB000828007D8032B12D07BD8022B00F0818013
:10CBC000002074E01D2B78D003D81C2BF8D105224F
:10CBD00006E01E2B73D01F2BF2D1082200E00222A8
:10CBE0003D4B196808296EDD0A296FDD0D29B5BF97
:10CBF0000C240E24022303233848C0F8F035012307
:10CC0000C0F8003500200546030103F1804303F519
:10CC1000E04301300828C3F81455C3F81055F3D188
:10CC20002F4B18682F4B1B6800021B0303F4805323
:10CC300000F4E0601843294BC3F81805C3F8142525
:10CC4000C3F810250DF10602C3F82C260122C3F803
:10CC500030261A60D3F80021002AFBD00022C3F846
:10CC6000002101225A601D4B1A46D3F80401002806
:10CC7000FBD00020C3F8040101209860D2F81431E1
:10CC8000002BFBD00023C2F81431BDF906209A42D4
:10CC9000124AB8BFADF80630A142C2F80035BDF95E
:10CCA000060004D035BF611A091BC840884003B094
:10CCB00030BD032294E7042292E7062290E7072280
:10CCC0008EE701228CE70824002395E70A2401233C
:10CCD00092E700BF083A01002800002000700040E1
:10CCE0002C00002020070020192830B53CD8224B0A
:10CCF00053F82000214B00221D4653F82240B4F186
:10CD0000FF3F32D11E4C45F822006FEA41411D4DD4
:10CD10001D4B246853F822306FEA514125F8121058
:10CD2000012101FA04F4C3F86005013CC3F864056D
:10CD300005EB4202C3F86805C3F86C050020C3F890
:10CD40000015C3F80C05C3F80405C3F80845C3F87B
:10CD50001405C3F81005C3F82025C3F82415C3F83B
:10CD60002815C3F82C05996030BD8442CAD0013221
:10CD7000032AC2D1F8E700BF083A01001C000020D6
:10CD80003000002018070020B83A010019280FD8F9
:10CD9000114B53F8203003290AD8DFE801F00216BE
:10CDA0000A1003F5E0734FF0A042002142F823106F
:10CDB000704703F5E0734FF0A0420C21F6E703F54E
:10CDC000E0734FF0A0420421F0E703F5E0734FF069
:10CDD000A0420321EAE700BF083A010019280CD855
:10CDE000064B53F82020012393404FF0A04211B985
:10CDF000C2F80C357047C2F808357047083A010090
:10CE000019289FBF4FF0A043054AD3F8103552F8B8
:10CE100020009ABF23FA00F000F0010000207047C4
:10CE2000083A010038B50025057329B90B4B0C4AA7
:10CE30000C48232101F082FE01600B4951F82220A9
:10CE4000027151F8233083719DF8103051F823306E
:10CE500043710223C371856038BD00BFC43A01002D
:10CE6000273B0100D23A0100083A0100037B23B9B5
:10CE700043738373036101230373704784B00DF11F
:10CE8000100C0CE90E009DF808100268002301291F
:10CE9000C2F80035039B12D00BD303290CD0C2F883
:10CEA0005435019BC2F824350123C2F8003504B083
:10CEB000704743F00203F2E743F00403EFE743F067
:10CEC0000603ECE710B5FFF7D1FF03688279C3F8DA
:10CED00008254279C3F80C250279C3F81025034BC5
:10CEE000BDE810400ECBFFF7C9BF00BF38070020D8
:10CEF00010B485B001AC84E80E0094E80E0005B0D3
:10CF00005DF8044BFFF7BABF70470368C3F81C1500
:10CF1000D3F80821002AFBD0D3F818050022C3F863
:10CF20000821C0B27047000007B5094B09490A48FB
:10CF30004FF080421A6000229A6002221A710B237D
:10CF400000930C220D23FFF76DFF03B05DF804FB87
:10CF50003807002000300040240700200B4601461F
:10CF6000184601F00DBE0000C0F3C7537F3B162BDF
:10CF7000024605DC002B04DB0348184122EA0000CE
:10CF8000704700F000407047FFFF7F002DE9F04F31
:10CF9000DFF808938DB006460F4614461D4600F094
:10CFA0007FF999F90080B8F1FF3FCDE9000136D053
:10CFB00022462B462046294601F012FD834670BBCF
:10CFC00032463B463046394601F00AFD0022824691
:10CFD0000023002840F0A0803046394601F0CEFC06
:10CFE00010B3002200232046294601F0C7FC8346E7
:10CFF000002867D00122A24B029200210022CDF826
:10D0000028A0CDE90467CDE90645CDE908120393D0
:10D01000B8F1000F41D09B4C0023CDE90034DDE98D
:10D0200000010DB0BDE8F08FDDE9000100F060FF08
:10D030008046002800F08B804FF0000A4FF0000B74
:10D0400052465B46DDE9000101F098FC0028E6D07D
:10D050003046394600F04CFF0028E0D020462946F3
:10D0600000F046FF0028DAD099F90030844A039294
:10D0700004210022022BCDE90467CDE90645CDE964
:10D0800008AB02910A9203D002A800F037FF50B912
:10D0900001F084FD2223036005E002A800F02EFFCA
:10D0A000002800F098800A9B1BB101F077FD0A9BD5
:10D0B0000360DDE90834CDE90034DDE900010DB09D
:10D0C000BDE8F08F2046294600F012FF0028A6D0C8
:10D0D000002200232046294601F05AFC00289ED059
:10D0E000674A99F90030CDF828B00121CDE90467ED
:10D0F000CDE90645CDE90212002B71D0624900202E
:10D10000022BCDE908016FD101F048FD2123036016
:10D110000A9B002BCDD0C8E72046294601F02EFC03
:10D1200000283FF47CAF01230293564B5449CDF8BD
:10D1300028B00022B8F1020FCDE90467CDE9064519
:10D140000391CDE90823A8D1CDE9002367E7304654
:10D15000394600F0CDFE00283FF46EAF2046294648
:10D1600000F0C6FE00283FF467AFDDE9002310465B
:10D17000194601F035FC99F900A0002866D1032377
:10D18000DFF8FCC00A9029462046029300223F4B5C
:10D19000CDF80CC0CDE90645CDE9046701F086F96C
:10D1A000002204460D46002330463946BAF1000FEE
:10D1B00020D1374F4FF06046CDE9086701F0E8FB1A
:10D1C00018BB02A800F09AFE0028A1D101F0E6FCED
:10D1D000222303609CE701F0E1FC2123036062E766
:10D1E00000230024CDE9083402A800F087FE0028BF
:10D1F0008ED189E7274F0026CDE9086701F0C8FBEB
:10D20000A0B9BAF1020FE1D0DBE72046294600F0D1
:10D210007DFE22462B4601F0B1FBA0B91E4B99F9C9
:10D2200000A04FF06042CDE90823EAE720462946F6
:10D2300000F06CFE22462B4601F0A0FB18B9124B01
:10D240000022CDE9082399F900A0DAE701220C4B6E
:10D25000CDF828800292CDE90467CDE90645039315
:10D26000BAF1000FBCD0002200231046194601F08D
:10D2700047FABAF1020FCDE908013FF445AFB3E731
:10D28000643B01000000F03F0000F0FF0000E03FC1
:10D29000FFFFEF470000F07FFFFFEFC734000020E3
:10D2A0002DE9F04F23F0004555EA020493B00DD06C
:10D2B000794E21F00044B4420F4682460FDD04F15E
:10D2C000404404F5801454EA0A035BD1734C0023F4
:10D2D000CDE90034DDE9000113B0BDE8F08F9846D8
:10D2E00094464ED0B542EADC6B4EB54266D0002F74
:10D2F0008B468146CDE9022364DB0026BCF1000F9A
:10D300000ED1654B9D4246D0644B9D4200F0978004
:10D31000B8F1804F00F0B280614B984500F0CC83AB
:10D320004846594600F0E0FDCDE90001BAF1000F92
:10D3300006D1002C60D0594B27F040429A425BD076
:10D34000FF0F013F56EA070300F08280554B9D42D4
:10D3500040F3B08003F104739D4240F34184524B8B
:10D360009C4240F38280B8F1000F40F3828048A3D2
:10D37000D3E900231046194601F098F8CDE90001E1
:10D38000A8E728B1494813B0BDE8F04F00F0B8BD98
:10D39000A542F7DCA8E704F1404303F5801353EA04
:10D3A0000A0393D0404B9C4240F39083B8F1000FA6
:10D3B0005FDBDDE90234CDE900348BE7BCF1000F1F
:10D3C00095D07CE73A4B9D4237DCA3F154739D42E4
:10D3D00093DD2B15A3F2FF33142B40F3E983C3F144
:10D3E00034032CFA03F202FA03F3634585D102F009
:10D3F0000102C2F1020681E7B8F1000F07DADDE9A8
:10D4000000230020254901F07BF9CDE90001002F20
:10D41000BFF660AF04F1404404F5801454EA0603FB
:10D4200000F03C84012E7FF455AFDDE90045224633
:10D4300005F10043CDE900234CE702265EE7B8F191
:10D44000000FC0F24F8348465946CDE9000141E73D
:10D450004A4648465B46594600F070FE02460B4677
:10D4600001F04EF9CDE9000134E7B8F1000FFFF605
:10D470007EAF00230024CDE900342BE74A4648461E
:10D480005B46594601F012F8CDE9000122E700BFE2
:10D490009C7500883CE4377E0000F07F0000F03F80
:10D4A0000000E03F0000E041FFFFEF3F683B01006C
:10D4B000FFFF3F43B4F5801F80F28F83DDE9000159
:10D4C0000022CF4B00F0F2FFCDE900010C466FF0D7
:10D4D000340C2315CB4DC4F31302A3F2FF3342F0F7
:10D4E0007F5403EB0C01AA420B9144F4401440F327
:10D4F0006F83C54B9A4240F3F38300220023CDE9AA
:10D50000082301310B91A4F58014CDE91023BF4B02
:10D510000022CDE906230025DDE90001DDE906232F
:10D520002146824600F00AFEA346DDE90623804636
:10D53000894650462146CDE90CAB00F001FE02467B
:10D540000B460020B14901F0DBF80A460146CDE95F
:10D550000E12134649460246404600F0A7FF6310EC
:10D5600043F0005382468B4603F500238C46CDE9F9
:10D5700004AB5919D3460023CDE900BC0093DDE983
:10D5800000AB002004460D4602460B465046594665
:10D5900000F08CFF02460B464046494600F0CEFDA7
:10D5A000DDE90623804689462046294600F0C6FD6F
:10D5B00002460B46DDE90C0100F0C0FD52465B4619
:10D5C00000F074FF02460B464046494600F0B6FDA7
:10D5D000DDE90E2300F06AFFDDE90445CDE906012F
:10D5E00022462B462046294600F060FF72A3D3E96D
:10D5F000002304460D4600F059FF71A3D3E9002330
:10D6000000F09EFD22462B4600F050FF6EA3D3E9AA
:10D61000002300F095FD22462B4600F047FF6CA347
:10D62000D3E9002300F08CFD22462B4600F03EFF9C
:10D6300069A3D3E9002300F083FD22462B4600F0C6
:10D6400035FF67A3D3E9002300F07AFD2246804628
:10D6500089462B462046294600F028FF02460B4605
:10D660004046494600F022FF524604460D465B46BE
:10D67000DDE9040100F064FDDDE9062300F016FF9A
:10D6800022462B4600F05CFD5246804689465B46AA
:10D690005046594600F00AFF00225D4BCDE90C01CF
:10D6A00000F04EFD42464B4600F04AFD00980D4604
:10D6B000044622462B465046594600F0F7FE00220B
:10D6C00082468B46524B2046294600F037FDDDE965
:10D6D0000C2300F033FD02460B464046494600F05D
:10D6E0002DFDDDE9042300F0E1FE22468046894657
:10D6F0002B46DDE9060100F0D9FE02460B46404606
:10D70000494600F01DFD8046894602460B465046BC
:10D71000594600F015FD009833A3D3E900230446D1
:10D720000D4600F0C3FE5246CDE904015B4620469B
:10D73000294600F003FD02460B464046494600F0EC
:10D74000FDFC2BA3D3E9002300F0B0FE2AA3D3E90C
:10D750000023804689462046294600F0A7FE02465F
:10D760000B464046494600F0EBFCDDE9102300F093
:10D77000E7FC80460B98894600F02EFE4246824622
:10D780008B464B46DDE9040100F0DAFCDDE90823B5
:10D7900000F0D6FC52465B4600F0D2FC00985246A0
:10D7A0005B4604460D4600F0C9FCDDE9082300F0A5
:10D7B000C5FCDDE904232DE0EF4E454A287ECA3F33
:10D7C00065DBC9934A86CD3F01411DA96074D13FF5
:10D7D0004D268F515555D53FFFAB6FDBB66DDB3F07
:10D7E000033333333333E33F000000E009C7EE3F38
:10D7F000FD033ADC09C7EE3FF5015B14E02F3EBEA6
:10D80000000040438E98030079B60B000000F03F03
:10D810000000084000F092FC0B4602464946404694
:10D8200000F08CFC013E56EA070382468B46DDE998
:10D83000020114BFD84BD94B0022CDE90423024684
:10D840000B46CDE9002300230093DDE90067324653
:10D850003B4600F073FC22462B4600F027FEDDE934
:10D860000223804689465046594600F01FFE024674
:10D870000B464046494600F063FC324680468946E6
:10D880003B4620462946CDE9028900F00FFE0B46B3
:10D89000024606460F464046494600F051FCC04B42
:10D8A000994204460D468A4640F3268101F13F43E2
:10D8B00003F5E003034340F0F781A3A3D3E900237A
:10D8C000DDE9020100F03CFC3246804689463B46D9
:10D8D0002046294600F032FC02460B4640464946A7
:10D8E00001F074F8002840F0DF81A8464FEA285381
:10D8F000A3F2FE324FF4801313415344C3F30A5290
:10D90000A84DA2F2FF321541C3F3130423EA050127
:10D910000020C2F1140B44F48014BAF1000F024647
:10D920000B4644FA0BFB30463946B8BFCBF1000B2F
:10D9300000F004FC02460B4606460F46DDE90201F4
:10D9400000F0FEFB4FEA0B5A0D46002480A3D3E9FA
:10D9500000232046294600F0A9FD3246804689462C
:10D960003B462046294600F0E9FB02460B46DDE92E
:10D97000020100F0E3FB78A3D3E9002300F096FD59
:10D9800077A3D3E9002306460F462046294600F038
:10D990008DFD02460B463046394600F0D1FB064667
:10D9A0000F4602460B464046494600F0C9FB424638
:10D9B0004B4604460D4600F0C1FB02460B4630467E
:10D9C000394600F0BBFB2246804689462B4620465E
:10D9D000294600F06BFD64A3D3E9002306460F46F9
:10D9E00000F064FD62A3D3E9002300F0A7FB3246F8
:10D9F0003B4600F05BFD60A3D3E9002300F0A0FBF1
:10DA000032463B4600F052FD5DA3D3E9002300F00F
:10DA100095FB32463B4600F049FD5BA3D3E900236A
:10DA200000F08EFB32463B4600F040FD02460B46BE
:10DA30002046294600F082FB06460F4602460B466A
:10DA40002046294600F032FD0022CDE900014FF0CA
:10DA500080433046394600F071FB02460B46DDE953
:10DA6000000100F04DFE424606460F464B4620465A
:10DA7000294600F01BFD42464B4600F061FB024682
:10DA80000B463046394600F059FB22462B4600F043
:10DA900055FB02460B4600203F4900F04FFB8A44ED
:10DAA000BAF5801FC0F22D815146DDE9042300F054
:10DAB000FDFCCDE900010DE4002FFFF631AC484636
:10DAC000594613B0BDE8F04F00F04CB9B8F1000F63
:10DAD000BFF6CFACDDE90234009304F100430193BB
:10DAE000FFF7F8BB4A465B4600202B4900F008FED2
:10DAF000CDE90001FFF7EEBB2B4B21F00048984524
:10DB000040F3E280294B0B4403430AD132463B46A3
:10DB100000F014FBDDE9022300F04EFF00283FF483
:10DB2000E5AE1BA3D3E90023DDE9040100F0BEFC50
:10DB300017A3D3E9002300F0B9FCCDE90001FFF7FA
:10DB4000C9BB00BFAFF30080FE822B654715973C31
:10DB500000000000432EE63FEF39FAFE422EE63F7A
:10DB6000396CA80C615C20BED0A4BE726937663ED9
:10DB7000F16BD2C541BDBB3E2CDE25AF6A56113FCD
:10DB800093BDBE166CC1663F3E5555555555C53FB4
:10DB900059F3F8C21F6EA5010000F03F0000F0BF6E
:10DBA000FFFF8F40FFFF0F00FFCB904000346F3F1F
:10DBB000BCF1000F40F09180C3F1140345FA03F269
:10DBC00002FA03F3AB4200F0A0806646FFF79CBB6D
:10DBD00000220023CDE9082397E44FF0000C78E4FD
:10DBE0005B4B9C427FF741AC5A4B9C423FF7BBAB2F
:10DBF000DDE900010022574B00F0A0FA46A3D3E96B
:10DC0000002304460D4600F051FC45A3D3E9002350
:10DC100082468B462046294600F048FC0022CDE98A
:10DC200000014D4B2046294600F040FC02460B46C1
:10DC30003DA1D1E9000100F081FA22462B4600F017
:10DC400035FC02460B460020444900F077FA224694
:10DC5000804689462B462046294600F027FC02468E
:10DC60000B464046494600F021FC31A3D3E900238E
:10DC700000F01CFC02460B46DDE9000100F05EFAF4
:10DC800002460B46804689465046594600F058FAEF
:10DC9000002004460D4652465B46BBE5DDE9002305
:10DCA00010461946FFF7D8BB23A3D3E90023DDE9CB
:10DCB000040100F0FBFB20A3D3E9002300F0F6FBF6
:10DCC000CDE90001FFF706BB244B98453FF70EAEA8
:10DCD000DDE900239246934637E60026FFF720BB96
:10DCE00017A3D3E90023CDE9082317A3D3E9002321
:10DCF000CDE910231A4B00224FF48025CDE90623ED
:10DD00000AE45A4600F090F9CFE602F00102C2F1AF
:10DD10000206FFF7F9BA00BF000000604715F73FA1
:10DD200044DF5DF80BAE543E555555555555D53F1E
:10DD3000FE822B654715F73F9C7500883CE4377ED3
:10DD40000000004003B8E23F06D0CF43EBFD4C3E5D
:10DD5000FEFFEF3F0000F03F0000D03F0000E03F3B
:10DD60000000F83F5F4A8A432DE9F0410D4607461F
:10DD700000F0948000290B460446064654DD0F153A
:10DD800000F0A780C3F31303A7F2FF3743F4801317
:10DD9000F20FF80702EB43034FEA460503D5ED0FF8
:10DDA00005EB4303B50000267F10B44616224FF45E
:10DDB00000110CEB010098424FEAD5744FEA45057B
:10DDC00003DC1B1A00EB010C0E44013A04EB430385
:10DDD0004FEA5101EDD11046964620244FF0004203
:10DDE00009E052D05B00013C03EBD5734FEA5202CD
:10DDF0004FEA450537D0634502EB0E01F1DD0029FE
:10DE000001EB020E0ADBE046A3EB0C03A94288BF3C
:10DE100003F1FF336D1A1044C446E3E7BEF1000F6F
:10DE2000F1DB0CF10108EFE721F00042024329D0B9
:10DE3000002945D10146CA0A153B4905002AFAD0F6
:10DE400012F4801001D048E030465200D40200F1B4
:10DE50000106F9D5C6F1200401FA06F6E1401F1AC1
:10DE600041EA02038EE72B4324D14408731003F1E7
:10DE70007F53F20703F5001348BF44F0004403EB5F
:10DE8000075127463846BDE8F081A942AAD80029A3
:10DE900001EB020EC2DB98460023BBE702460B46AD
:10DEA00000F004FB3A462B4600F04AF90746384694
:10DEB000BDE8F081411C16BF421C01365408D5E76D
:10DEC000024600F03BF902460B4600F019FC0746FB
:10DED000D8E71A4621463B46B2E70E4620244FF0CB
:10DEE000FF30BBE70000F07F21F000431946704788
:10DEF00041F0004101F58010C00F704700207047CD
:10DF000000200149704700BF0000F87F2DE9F04173
:10DF1000C1F30A57A7F2FF35132D82B002460B4614
:10DF20000C464FEAD178064633DC002D4EDB3B49E8
:10DF3000294103EA0100104326D049080B4052EA68
:10DF400003060CD04FF48023132D24EA010143FA79
:10DF500005F444EA01040CBF4FF0004600263049A6
:10DF600001EBC8082346D8E9004532462046294639
:10DF700000F0E6F8CDE9000122462B46DDE900017C
:10DF800000F0DCF802460B461046194602B0BDE828
:10DF9000F081332D07DDB5F5806FF5D100F0D0F8B5
:10DFA00002460B46F0E7A7F213474FF0FF31F94066
:10DFB0000842E9D049080842D1D04FF0804320EA16
:10DFC000010143FA07F741EA0706C8E721F00041DB
:10DFD0000143D9D0C3F3130101434E42104D0E4308
:10DFE000360B05EBC8055C0C06F40023D5E9006789
:10DFF000640443EA04010B463046394600F0A0F8B9
:10E00000CDE9000132463B46DDE9000100F096F81B
:10E0100021F00041024641EAC873B5E7FFFF0F0057
:10E02000703B010000000000F8B5C1F30A5304463C
:10E030000D460E4617460BBB21F000460346334300
:10E040001BD0354B002200F031FA344B9F4204467E
:10E050000D4635DBC1F30A530E46363B3B4440F2D6
:10E06000FE72934232DC002B11DD26F0FF4626F4CF
:10E07000E00646EA035520462946F8BD40F2FF7205
:10E080009342EBD102460B4600F05AF8F8BD13F16B
:10E09000350F28DA4CF250339F4222462B460ADDD8
:10E0A00019A1D1E9000100F03DF817A3D3E900233D
:10E0B00000F0FCF9F8BD16A1D1E9000100F032F83A
:10E0C00013A3D3E9002300F0F1F9F8BD22462B4653
:10E0D0000DA1D1E9000100F025F80BA3D3E900233D
:10E0E00000F0E4F9F8BD26F0FF4626F4E0063633EA
:10E0F00046EA0355204629460022094B00F0D6F98E
:10E10000F8BD00BFAFF300809C7500883CE4377E0B
:10E1100059F3F8C21F6EA50100005043B03CFFFF49
:10E120000000903C03F0004321F0004242EA03016A
:10E13000704700BF81F0004102E000BF83F0004360
:10E1400030B54FEA41044FEA430594EA050F08BF92
:10E1500090EA020F1FBF54EA000C55EA020C7FEA56
:10E16000645C7FEA655C00F0E2804FEA5454D4EBD3
:10E170005555B8BF6D420CDD2C4480EA020281EA9D
:10E18000030382EA000083EA010180EA020281EAD5
:10E190000303362D88BF30BD11F0004F4FEA013127
:10E1A0004FF4801C4CEA113102D0404261EB410136
:10E1B00013F0004F4FEA03334CEA133302D05242BC
:10E1C00063EB430394EA050F00F0A780A4F1010478
:10E1D000D5F1200E0DDB02FA0EFC22FA05F28018B2
:10E1E00041F1000103FA0EF2801843FA05F3594198
:10E1F0000EE0A5F120050EF1200E012A03FA0EFC17
:10E2000028BF4CF0020C43FA05F3C01851EBE37140
:10E2100001F0004507D54FF0000EDCF1000C7EEB5D
:10E2200000006EEB0101B1F5801F1BD3B1F5001F9B
:10E230000CD349085FEA30004FEA3C0C04F10104BA
:10E240004FEA445212F5800F80F09A80BCF1004FE3
:10E2500008BF5FEA500C50F1000041EB045141EA65
:10E26000050130BD5FEA4C0C404141EB010111F466
:10E27000801FA4F10104E9D191F0000F04BF014611
:10E280000020B1FA81F308BF2033A3F10B03B3F1EF
:10E2900020020CDA0C3208DD02F1140CC2F10C027F
:10E2A00001FA0CF021FA02F10CE002F11402D8BFDD
:10E2B000C2F1200C01FA02F120FA0CFCDCBF41EAA9
:10E2C0000C019040E41AA2BF01EB0451294330BD78
:10E2D0006FEA04041F3C1CDA0C340EDC04F1140455
:10E2E000C4F1200220FA04F001FA02F340EA03002C
:10E2F00021FA04F345EA030130BDC4F10C04C4F172
:10E30000200220FA02F001FA04F340EA0300294651
:10E3100030BD21FA04F0294630BD94F0000F83F49B
:10E32000801306BF81F480110134013D4EE77FEA7E
:10E33000645C18BF7FEA655C29D094EA050F08BFCA
:10E3400090EA020F05D054EA000C04BF19461046AB
:10E3500030BD91EA030F1EBF0021002030BD5FEAEF
:10E36000545C05D14000494128BF41F0004130BD17
:10E3700014F580043CBF01F5801130BD01F000456B
:10E3800045F0FE4141F470014FF0000030BD7FEADE
:10E39000645C1ABF194610467FEA655C1CBF0B46D9
:10E3A000024650EA013406BF52EA033591EA030FF0
:10E3B00041F4002130BD00BF90F0000F04BF0021E8
:10E3C000704730B54FF4806404F132044FF000051B
:10E3D0004FF0000150E700BF90F0000F04BF002194
:10E3E000704730B54FF4806404F1320410F00045FA
:10E3F00048BF40424FF000013EE700BF42004FEAF5
:10E40000E2014FEA31014FEA02701FBF12F07F4371
:10E4100093F07F4F81F06051704732F07F4208BF28
:10E42000704793F07F4F04BF41F40021704730B52F
:10E430004FF4607401F0004521F000411CE700BF7B
:10E4400050EA010208BF704730B54FF000050AE0FE
:10E4500050EA010208BF704730B511F0004502D5FF
:10E46000404261EB41014FF4806404F132045FEA01
:10E47000915C3FF4D8AE4FF003025FEADC0C18BFAA
:10E4800003325FEADC0C18BF033202EBDC02C2F19C
:10E49000200300FA03FC20FA02F001FA03FE40EA2E
:10E4A0000E0021FA02F11444BDE600BF70B54FF032
:10E4B000FF0C4CF4E06C1CEA11541DBF1CEA135510
:10E4C00094EA0C0F95EA0C0F00F0DEF82C4481EA78
:10E4D000030621EA4C5123EA4C5350EA013518BF98
:10E4E00052EA033541F4801143F4801338D0A0FB85
:10E4F00002CE4FF00005E1FB02E506F00042E0FB32
:10E5000003E54FF00006E1FB03569CF0000F18BF37
:10E510004EF0010EA4F1FF04B6F5007F64F54074DF
:10E5200004D25FEA4E0E6D4146EB060642EAC62172
:10E5300041EA55514FEAC52040EA5E504FEACE2EDF
:10E54000B4F1FD0C88BFBCF5E06F1ED8BEF1004FE2
:10E5500008BF5FEA500E50F1000041EB045170BD5E
:10E5600006F0004646EA010140EA020081EA0301A2
:10E57000B4EB5C04C2BFD4EB0C0541EA045170BD9E
:10E5800041F480114FF0000E013C00F3AB8014F118
:10E59000360FDEBF002001F0004170BDC4F1000461
:10E5A000203C35DA0C341BDC04F11404C4F12005E2
:10E5B00000FA05F320FA04F001FA05F240EA02003D
:10E5C00001F0004221F0004110EBD37021FA04F673
:10E5D00042EB06015EEA430E08BF20EAD37070BD2D
:10E5E000C4F10C04C4F1200500FA04F320FA05F08C
:10E5F00001FA04F240EA020001F0004110EBD3708E
:10E6000041F100015EEA430E08BF20EAD37070BDFD
:10E61000C4F1200500FA05F24EEA020E20FA04F3D6
:10E6200001FA05F243EA020321FA04F001F0004185
:10E6300021FA04F220EA020000EBD3705EEA430EF6
:10E6400008BF20EAD37070BD94F0000F0FD101F025
:10E650000046400041EB010111F4801F08BF013C5E
:10E66000F7D041EA060195F0000F18BF704703F09C
:10E670000046520043EB030313F4801F08BF013D23
:10E68000F7D043EA0603704794EA0C0F0CEA1355DF
:10E6900018BF95EA0C0F0CD050EA410618BF52EA99
:10E6A0004306D1D181EA030101F000414FF000009F
:10E6B00070BD50EA410606BF1046194652EA4306AD
:10E6C00019D094EA0C0F02D150EA013613D195EA21
:10E6D0000C0F05D152EA03361CBF104619460AD169
:10E6E00081EA030101F0004141F0FE4141F4700173
:10E6F0004FF0000070BD41F0FE4141F4780170BD63
:10E7000070B54FF0FF0C4CF4E06C1CEA11541DBFC7
:10E710001CEA135594EA0C0F95EA0C0F00F0A7F8C9
:10E72000A4EB050481EA030E52EA03354FEA0131F6
:10E7300000F088804FEA03334FF0805545EA131309
:10E7400043EA12634FEA022245EA111545EA1065D1
:10E750004FEA00260EF000419D4208BF964244F168
:10E76000FD0404F5407402D25B084FEA3202B61A87
:10E7700065EB03055B084FEA32024FF480104FF45B
:10E78000002CB6EB020E75EB030E22BFB61A7546CF
:10E7900040EA0C005B084FEA3202B6EB020E75EB62
:10E7A000030E22BFB61A754640EA5C005B084FEACA
:10E7B0003202B6EB020E75EB030E22BFB61A754697
:10E7C00040EA9C005B084FEA3202B6EB020E75EBA2
:10E7D000030E22BFB61A754640EADC0055EA060E63
:10E7E00018D04FEA051545EA16754FEA06164FEAA6
:10E7F000C30343EA52734FEAC2025FEA1C1CC0D152
:10E8000011F4801F0BD141EA00014FF000004FF0DE
:10E81000004CB6E711F4801F04BF01430020B4F19F
:10E82000FD0C88BFBCF5E06F3FF6AFAEB5EB030C57
:10E8300004BFB6EB020C5FEA500C50F1000041EB54
:10E84000045170BD0EF0004E4EEA113114EB5C0421
:10E85000C2BFD4EB0C0541EA045170BD41F48011F4
:10E860004FF0000E013C90E645EA060E8DE60CEAFC
:10E87000135594EA0C0F08BF95EA0C0F3FF43BAF19
:10E8800094EA0C0F0AD150EA01347FF434AF95EAD0
:10E890000C0F7FF425AF104619462CE795EA0C0FB4
:10E8A00006D152EA03353FF4FDAE1046194622E781
:10E8B00050EA410618BF52EA43067FF4C5AE50EA5B
:10E8C00041047FF40DAF52EA43057FF4EBAE12E74B
:10E8D0004FF0FF3C06E000BF4FF0010C02E000BF2C
:10E8E0004FF0010C4DF804CD4FEA410C7FEA6C5C0F
:10E8F0004FEA430C18BF7FEA6C5C1BD001B050EAB2
:10E90000410C0CBF52EA430C91EA030F02BF90EA9C
:10E91000020F0020704710F1000F91EA030F58BF5B
:10E92000994208BF90422CBFD8176FEAE37040F0BD
:10E93000010070474FEA410C7FEA6C5C02D150EA5B
:10E94000013C07D14FEA430C7FEA6C5CD6D152EA16
:10E95000033CD3D05DF8040B704700BF84461046DB
:10E9600062468C461946634600E000BF01B5FFF7DA
:10E97000B7FF002848BF10F1000F01BD4DF808EDAA
:10E98000FFF7F4FF0CBF012000205DF808FB00BF7B
:10E990004DF808EDFFF7EAFF34BF012000205DF8D5
:10E9A00008FB00BF4DF808EDFFF7E0FF94BF012022
:10E9B00000205DF808FB00BF4DF808EDFFF7CEFF23
:10E9C00094BF012000205DF808FB00BF4DF808ED62
:10E9D000FFF7C4FF34BF012000205DF808FB00BF33
:10E9E0004FEA410C7FEA6C5C02D150EA013C0AD14B
:10E9F0004FEA430C7FEA6C5C02D152EA033C02D13D
:10EA00004FF0000070474FF0010070474FEA41029D
:10EA100012F5001215D211D56FF47873B3EB625270
:10EA200012D94FEAC12343F0004343EA505311F097
:10EA3000004F23FA02F018BF404270474FF0000029
:10EA4000704750EA013005D111F0004008BF6FF067
:10EA5000004070474FF00000704700BF4A0011D2DD
:10EA600012F5001211D20DD56FF47873B3EB625228
:10EA70000ED44FEAC12343F0004343EA505323FA34
:10EA800002F070474FF00000704750EA013002D1A9
:10EA90004FF0FF3070474FF0000070474FEA4102DF
:10EAA000B2F1E04324BFB3F5001CDCF1FE5C0DD9EC
:10EAB00001F0004C4FEAC0024CEA5070B2F1004F36
:10EAC00040EB830008BF20F00100704711F0804F39
:10EAD00021D113F13872BCBF01F00040704741F4FE
:10EAE00080114FEA5252C2F11802C2F1200C10FA02
:10EAF0000CF320FA02F018BF40F001004FEAC123E6
:10EB00004FEAD32303FA0CFC40EA0C0023FA02F389
:10EB10004FEA4303CCE77FEA625307D150EA01335F
:10EB20001EBF4FF0FE4040F44000704701F000402F
:10EB300040F0FE4040F40000704700BF1FB51C4687
:10EB4000094B1B680546D86852B1084B0091CDE9C6
:10EB5000013207492B46224600F0A8F901F030FDAA
:10EB6000044B1A46F2E700BF38000020803B01004A
:10EB70008D3B0100CE3901000A22002101F04ABB81
:10EB800010B5054C13462CB10A4601460220AFF3DE
:10EB9000008010BD2046FCE700000000014B186813
:10EBA000704700BF3800002008B5074B044613B17A
:10EBB0000021AFF30080054B1868836A03B19847C2
:10EBC000204603F0D3FC00BF000000001C3C010005
:10EBD0008A892DE9F041054610070C4658D44B6848
:10EBE000002B05DC0B6C002B02DC0020BDE8F08163
:10EBF000E66A002EF9D0002312F480522F68216AB1
:10EC00002B6032D0606DA3895A0705D56368C01A9E
:10EC1000636B0BB1236CC01A00230246E66A216ABB
:10EC20002846B047431CA38906D129681D2948D826
:10EC3000294ACA40D60744D500226260D904226915
:10EC4000226004D5421C01D12B6803B96065616B59
:10EC50002F600029C9D004F14403994202D028460C
:10EC600000F00AFA00206063C0E701232846B0479D
:10EC7000411CC8D12B68002BC5D01D2B01D0162BF1
:10EC800001D12F60B1E7A38943F04003A381ADE731
:10EC90000F69002FA9D093070E6808BF4B690F605A
:10ECA00018BF0023A6EB07088B60B8F1000F9CDDAE
:10ECB00043463A46216AA66A2846B047002806DC41
:10ECC000A38943F04003A3814FF0FF308EE7074450
:10ECD000A8EB0008E9E700BF0100402038B50B6948
:10ECE00005460C46DBB118B183690BB900F072F828
:10ECF0000C4B9C4209D16C68B4F90C307BB12146B5
:10ED00002846BDE83840FFF763BF074B9C4201D15E
:10ED1000AC68F1E7054B9C4208BFEC68ECE70020CB
:10ED200038BD00BFDC3B0100FC3B0100BC3B0100E7
:10ED3000014620B9044B0549186800F0C9B8044BD6
:10ED40001868FFF7CBBF00BF1C3C0100DDEC0000E2
:10ED500038000020002310B50446C0E9003383606A
:10ED600081814366C281C0E9043383611946082268
:10ED70005C3000F078F9054B6362054BA362054BEC
:10ED8000E362054B2462236310BD00BF31FE000027
:10ED900057FE00008FFE0000B3FE0000014900F0A6
:10EDA00097B800BFDDEC000070B54A1E68255543DA
:10EDB0000E4605F1740100F0ADF9044640B10021A2
:10EDC000C0E900160C30A06005F1680200F04BF9B4
:10EDD000204670BD836910B5044633BBC0E91233C9
:10EDE0000365124B124A1B688262984204BF0123DA
:10EDF000836100F01FF86060204600F01BF8A060FF
:10EE0000204600F017F80022E06004216068FFF758
:10EE1000A1FF01220921A068FFF79CFF0222122115
:10EE2000E068FFF797FF0123A36110BD1C3C0100C0
:10EE30009DED0000F8B51B4B1E68B369074613B97A
:10EE40003046FFF7C7FF4836D6E90134013B03D50A
:10EE5000336833B13668F7E7B4F90C506DB16834F4
:10EE6000F4E704213846FFF79FFF30600028F1D116
:10EE70000C233B6004462046F8BD0B4B6566C4E995
:10EE80000055A560C4E90335C4E9055508222946A3
:10EE900004F15C0000F0E7F8C4E90D55C4E912552F
:10EEA000E9E700BF1C3C01000100FFFF0EB403B501
:10EEB000014603AB054853F8042B0068019300F0AA
:10EEC000ABF902B05DF804EB03B0704738000020E6
:10EED0002DE9F8438046894600F14804002614B91C
:10EEE0003046BDE8F883D4E90175013F01D52468B7
:10EEF000F5E7AB89012B07D9B5F90E30013303D003
:10EF000029464046C84706436835EEE770B50D4EC2
:10EF10000D4CA41BA4100025A54209D10B4E0C4C8E
:10EF200003F026FBA41BA4100025A54205D170BD4B
:10EF300056F8253098470135EEE756F825309847C2
:10EF40000135F2E708020020080200200802002034
:10EF50008402002010B5044600F022F820444078D6
:10EF600000F0440010BD931E222B10B50C4604D9AE
:10EF700000230B701C46204610BD0A2A09D1002828
:10EF800007DA2D230B7040420121214401F0FAF9E8
:10EF9000F1E70021F9E7FFF7E6BFD0F8EC00704792
:10EFA000044B054A1B681B6A002B08BF1346D3F8A5
:10EFB000EC007047380000209C000020024B014606
:10EFC000186800F0A7B800BF38000020024B0146C7
:10EFD000186800F051B800BF3800002082B001B9B5
:10EFE00001A942B14BB113780B601278101C18BF05
:10EFF000012002B070471046FBE76FF00100F8E710
:10F0000030B50024A24201D1002007E0035D0134A5
:10F010000D1915F8015CAB42F4D0581B30BD10B58A
:10F02000431E0A44914200D110BD11F8014B03F870
:10F03000014FF7E7884210B501EB020307D8421EE3
:10F0400099420AD011F8014B02F8014FF8E78342C8
:10F05000F5D98118D21AD34200D110BD13F8014D51
:10F0600001F8014DF7E702440346934200D170478F
:10F0700003F8011BF9E7000038B50546002945D023
:10F0800051F8043C0C1F002BB8BFE41802F0D0F973
:10F090001F4A1368104633B9636014602846BDE800
:10F0A000384002F0C6B9A3420CD9216862189342D5
:10F0B00004BF1A685B68636004BF52182260046072
:10F0C000ECE713465A680AB1A242FAD919685818EF
:10F0D000A0420BD120680144581882421960DDD14A
:10F0E000106852685A6001441960D7E702D90C23AE
:10F0F0002B60D3E7206821188A4204BF1168526848
:10F10000626004BF091821605C60C7E738BD00BFBA
:10F110004407002070B5CD1C25F0030508350C2DE3
:10F1200038BF0C25002D064601DBA94203D90C236C
:10F130003360002070BD02F07BF9214A146821463B
:10F1400091B9204C23681BB9304600F003FE2060C3
:10F150002946304600F0FEFD431C24D10C233360C9
:10F16000304602F066F9E4E70B685B1B18D40B2B02
:10F170000FD90B60CD50CC18304602F05AF904F18B
:10F180000B00231D20F00700C31AD3D05A42E250CF
:10F19000D0E78C424B6816BF636013600C46EBE708
:10F1A0000C464968CCE7C41C24F00304A04205D0F7
:10F1B000211A304600F0CEFD0130CFD02560DBE7CC
:10F1C00044070020480700209368013B002B10B43F
:10F1D000936007DA9469A34201DB0A2902D110BCCB
:10F1E00001F00EB91368581C10601970084610BC65
:10F1F0007047F8B506460F461446D518AC4201D103
:10F20000002007E03A4614F8011B3046FFF7DCFF08
:10F21000431CF3D1F8BD00002DE9F04F9DB00C4622
:10F2200017460393064618B183690BB9FFF7D2FD61
:10F230007B4B9C4257D17468A38918075DD523691D
:10F24000002B5AD00023099320238DF82930302336
:10F250008DF82A304FF0010BB846454615F8013BB2
:10F260000BB1252B54D1B8EB070A0BD053463A46C5
:10F2700021463046FFF7BDFF013000F0C280099BF8
:10F280005344099398F80030002B00F0BA80002313
:10F290004FF0FF32CDE90523049307938DF85330E7
:10F2A0001A93A846052218F8011B5E4802F070F870
:10F2B000049B78BBD90644BF20228DF853201A073F
:10F2C00044BF2B228DF853202A782A2A2AD0079A65
:10F2D000A84600200A25414611F8013B303B092B86
:10F2E00069D960B324E0504B9C4201D1B468A3E7D4
:10F2F0004E4B9C4208BFF4689EE72146304601F021
:10F30000F1F800289ED04FF0FF301DB0BDE8F08F1F
:10F31000A846A2E7434A801A0BFA00F0184304906B
:10F320004546BEE7039A111D12680391002A01DBCE
:10F33000079204E0524243F002030792049398F8C4
:10F3400000302E2B0ED198F801302A2B38D1039B98
:10F350001A1D1B680392002BB8BF4FF0FF3308F152
:10F3600002080593324D98F800100322284602F057
:10F370000FF840B14023401B03FA00F0049B034305
:10F3800008F10108049398F800102A488DF8281015
:10F39000062208F1010701F0FBFF002837D0264BB9
:10F3A0001BBB039B073323F0070308330393099B1D
:10F3B0004B44099350E705FB0232012088468AE757
:10F3C000002308F10108059319460A25404610F864
:10F3D000012B303A092A03D9002BC3D00591C1E78C
:10F3E00005FB012101238046F0E703AB0093224691
:10F3F000124B04A9304600F0B3F8B0F1FF3F81464C
:10F40000D5D1A3895B063FF57EAF09987DE703ABB5
:10F4100000932246094B04A9304600F04DFBECE76F
:10F42000DC3B0100263C0100FC3B0100BC3B010031
:10F430002C3C0100303C010061F50000F3F10000BC
:10F440002DE9F04788B0002B149F109DDDE9121ABA
:10F450001E4627F02007BBBF03F100431E460023D2
:10F460002D23462F14460B7004D0452F00D10135B3
:10F47000022300E0032307AA049206AACDE902A210
:10F48000CDE900352246334601F03EF9472F80464C
:10F4900002D1119BDB0726D5462F08EB050911D1B8
:10F4A00098F80030302B0AD1002200232046314644
:10F4B000FFF764FA18B9C5F10105CAF80050DAF887
:10F4C000003099440022002320463146FFF756FAC7
:10F4D00038B93022079B4B4505D2591C07911A7049
:10F4E000F8E7CDF81C90079B159AA3EB080340465C
:10F4F000136008B0BDE8F087F7B500290446BABF2D
:10F5000049422D232B23092904F8022B437020DDC7
:10F510000DF107031F460A2691FBF6F506FB1511B0
:10F520003031092D03F8011C03F1FF32294609DCB3
:10F530003031023B02F8011CBB42224604D3101AB0
:10F5400003B0F0BD1346E7E713F8012B04F8012BD5
:10F55000F2E7302319448370021DC170EFE7000009
:10F560002DE9F04F91B00C461A9F93461E46054672
:10F5700001F084FE03680993184600F006FD00239D
:10F580000E933B680A90073323F0070303F1080248
:10F5900094F81880D4F800A03A60D3E90023C4E9B5
:10F5A0001223D4E9127929F000430B934FF0FF3274
:10F5B000A64B0B993846FFF713FA68BB4FF0FF32A2
:10F5C000A24B0B993846FFF7EDF928BB0022002328
:10F5D00038464946FFF7DCF910B12D2384F8433053
:10F5E0009B4F9C4BB8F1470F98BF1F4603232361E5
:10F5F0002AF0040323604FF0000900965B460FAA2F
:10F600002146284600F0E2F9013040F090804FF0AA
:10F61000FF3011B0BDE8F08F3A464B4638464946B8
:10F62000FFF7DEF910B18C4F8C4BDBE76368591C98
:10F630004AF480620EA90DA840D1062363600DF143
:10F640003303CDE901234FF0000C63682260CDE95C
:10F65000030800933A464B46CDE9051C2846FFF7C0
:10F66000EFFE08F0DF03472B074609D10D9BD81C9E
:10F6700002DB6268934247DDA8F102085FFA88F86E
:10F68000B8F1650F0D9924D80139424604F15000B4
:10F690000D91FFF731FF0E9A1318012A814623615D
:10F6A00002DC2268D10701D5013323619DF8333094
:10F6B000002BA2D02D2384F843309EE7B8F1670FCA
:10F6C00000F06E81B8F1470FB9D1002BB7D10123FB
:10F6D000B4E7B8F1660F19D1002963680CDD216128
:10F6E00013B92268D20702D501330B4423610D9B65
:10F6F000A3654FF00009D9E713B92268D00701D5F7
:10F700000233F3E70123F1E74FF06708DDE90D323B
:10F71000934205DB22682361D107E8D50133E5E791
:10F72000002BD4BFC3F1020301231344DEE7236897
:10F730005A0507D423693A4659462846B04701304E
:10F7400029D164E7B8F1650F40F2D7800022002389
:10F75000D4E91201FFF712F988B30123404A594650
:10F760002846B04701303FF452AFDDE90D239A42FD
:10F7700002DB2368D8070ED5DDE909235946284660
:10F78000B04701303FF443AF002704F11A080E9B45
:10F79000013BBB4209DC23689F0700F1FD80E06864
:10F7A0000F9B9842B8BF184633E70123424659469B
:10F7B0002846B04701303FF42AAF0137E7E70D9BF9
:10F7C000002B2BDC0123264A59462846B04701303E
:10F7D0003FF41DAF0D9B23B90E9B13B92368D907C6
:10F7E000D9D5DDE9092359462846B04701303FF411
:10F7F0000EAF4FF0000804F11A090D9B5B42434520
:10F8000001DC0E9B97E701234A4659462846B0473C
:10F8100001303FF4FCAE08F10108EEE70E9AA36D4B
:10F820009A42A8BF1A46002A904607DD1346594659
:10F830003A462846B04701303FF4E9AE04F11A03D6
:10F840004FF0000A28EAE8780B9315E0FFFFEF7FFE
:10F85000803A0100373C01007C3A01003B3C01004A
:10F860006C39010001230B9A59462846B0470130F4
:10F870003FF4CDAE0AF1010AD4F85890A9EB080381
:10F880005345EFDCDDE90D239A424F4414DB236836
:10F89000DA0711D40E9B0D99A3EB0902A3EB010922
:10F8A0009145A8BF9146B9F1000F0DDC002729EA68
:10F8B000E97904F11A0818E0DDE9092359462846D8
:10F8C000B0470130E6D1A2E64B463A4659462846B3
:10F8D000B0470130EAD19AE601234246594628460C
:10F8E000B04701303FF493AE0137DDE90D239B1A99
:10F8F000A3EB0903BB42EFDC4DE70E9A012A01DCC2
:10F90000DB0738D501233A4659462846B04701302F
:10F910003FF47DAEDDE9092359462846B047013062
:10F9200007F101073FF473AE0E9B002203F1FF388D
:10F93000D4E912010023FFF721F8C0B943463A4643
:10F9400059462846B04701300DD160E601234246B2
:10F9500059462846B04701303FF459AE01370E9B57
:10F96000013BBB42F2DC4B4604F15002E4E60027C7
:10F9700004F11A08F3E70123E1E70123424659465F
:10F980002846B04701303FF442AE0137E3680F9A92
:10F990009B1ABB42F1DC02E7002704F11908F5E7E6
:10F9A000002B3FF494AE4FF0000CCDE9051C0DF197
:10F9B00033012260CDE90308CDE9012100933A46E5
:10F9C0004B462846FFF73CFD07464FE62DE9F0473A
:10F9D00091461F468A680B69DDF820809342B8BFC4
:10F9E0001346C9F8003091F8432006460C4612B180
:10F9F0000133C9F800302368990642BFD9F80030B6
:10FA00000233C9F80030256815F0060507D104F166
:10FA1000190AE368D9F800209B1AAB4228DC94F855
:10FA200043302268003318BF012392062DD404F11D
:10FA3000430239463046C047013020D02368E5688C
:10FA4000D9F8002003F00603042B08BFAD1AA36801
:10FA500022690CBF25EAE57500259342C4BF9B1AB5
:10FA6000ED184FF000091A344D451AD1002008E076
:10FA70000123524639463046C047013003D14FF08A
:10FA8000FF30BDE8F0870135C3E7E1185A1C30208C
:10FA900081F84300224494F8451082F84310023361
:10FAA000C5E70123224639463046C0470130E6D03B
:10FAB00009F10109D8E700002DE9F04301F1430CF9
:10FAC0000C46097E85B06E291746064698460C9A64
:10FAD00000F0B38022D8632936D00AD8002900F07C
:10FAE000B980582900F0838004F1420584F842105F
:10FAF00032E0642901D06929F6D12068136805062F
:10FB000003F104012AD51B681160002B03DA2D22B2
:10FB10005B4284F843206F480A2239E0732900F0E1
:10FB20009D8008D86F2920D07029DDD1236843F04B
:10FB30002003236003E0752917D07829D4D17823D6
:10FB400084F84530644855E01368191D1B6811603E
:10FB500004F1420584F8423001238CE01B681160F7
:10FB600010F0400F18BF1BB2CFE713682568181DAF
:10FB70001060280601D51B6802E06806FBD51B88CB
:10FB800054486F2914BF0A220822002184F8431028
:10FB90006568A560002DC0F29580216821F0040100
:10FBA0002160002B3DD1002D40F08E806546082A53
:10FBB0000BD12368DB0708D5236962689A42DEBF50
:10FBC000302305F8013C05F1FF35ACEB050323615B
:10FBD000CDF800803B4603AA21463046FFF7F6FEEB
:10FBE00001304DD14FF0FF3005B0BDE8F08339480A
:10FBF00084F84510136821681D1D1B6815600A06EE
:10FC00000BD5CA0744BF41F0200121601BB922680F
:10FC100022F0200222601022B7E74D0648BF9BB2B7
:10FC2000EFE76546B3FBF2F102FB1133C35C05F865
:10FC3000013D0B460029F5D1B9E7136825686169D4
:10FC4000181D106028061B6801D5196002E06A06BD
:10FC5000FBD51980002323616546B9E71368191D98
:10FC600011601D6862680021284601F091FB08B10F
:10FC7000401B606063682361002384F84330A7E77A
:10FC800023692A4639463046C0470130AAD0236846
:10FC90009B0713D4E068039B9842B8BF1846A3E7BC
:10FCA00001234A4639463046C04701309AD00135D3
:10FCB000E368039A9B1AAB42F2DCEBE7002504F100
:10FCC0001909F5E7002BACD1037884F8423004F130
:10FCD00042056CE73F3C0100503C010038B5134B36
:10FCE0001C68A36B7BB91820FFF768F9104A114B09
:10FCF000A063C0E90023104B83600B2383810122A2
:10FD00000023C0E90423A16B0C480A694B690C4C21
:10FD1000504304FB0300A2FB04230344541C43F19F
:10FD20000005C1E9044525F0004038BD3800002039
:10FD30000E33CDAB34126DE6ECDE05002DF45158D8
:10FD40002D7F954C024B0A460146186801F05CBEB7
:10FD50003800002038B5064C0023054608462360CD
:10FD600002F0EEFB431C02D1236803B12B6038BDC7
:10FD7000500800200CB430B5174B0C1E9DB01D6808
:10FD800008DA8B232B604FF0FF301DB0BDE8304008
:10FD900002B070474FF40273ADF8143014BF04F191
:10FDA000FF332346049307934FF6FF7302900690A8
:10FDB000ADF81630209A21AB02A92846019301F034
:10FDC000A3FE431CBCBF8B232B60002CDDD0029B09
:10FDD00000221A70D9E700BF380000200EB430B5F9
:10FDE0009CB01FAC4FF4017254F8045BADF81420C2
:10FDF0000290069000F0C9F80B4B039007900B930C
:10FE00000A48019400230F9314934FF6FF73ADF843
:10FE100016302A46234602A9006801F0C5FF1CB02F
:10FE2000BDE8304003B0704753FE000038000020AA
:10FE300010B50C46B1F90E1002F05EFA0028ABBF07
:10FE4000636DA3891B1823F48053ACBF6365A38142
:10FE500010BD002070472DE9F0411F468B89DB055E
:10FE600005460C46164605D502230022B1F90E10B0
:10FE700001F012FAA389B4F90E1023F48053A38180
:10FE800032463B462846BDE8F04100F019BB10B5AC
:10FE90000C46B1F90E1001F0FFF9431CA38915BF00
:10FEA000606523F4805343F48053A38118BFA3817A
:10FEB00010BDB1F90E1000F08BBBF8B506460F4629
:10FEC00016F8014BFFF76CF8204417F8015B4378F4
:10FED00003F00303012B08BF2034FFF761F8284427
:10FEE000427802F00302012A08BF2035601B01D1CD
:10FEF000002DE5D1F8BD10B503461A785C1C3AB95F
:10FF0000013B11F8012B03F8012F002AF9D110BD94
:10FF10002346F2E7C9B2034610F8012B1AB18A4210
:10FF2000F9D118467047002918BF0023F9E710F8E7
:10FF3000012B11F8013B012A28BF9A42F7D0D01AB1
:10FF40007047034611F8012B03F8012B002AF9D161
:10FF500070470000024B0146186800F003B800BF6C
:10FF60003800002070B5064608460C4600F00DF833
:10FF7000451C29463046FFF7CDF8064618B12A46FB
:10FF80002146FFF74CF8304670BD034613F8012BAD
:10FF9000002AFBD1181A0138704730B503461C7887
:10FFA0005D1C44B912F1FF3204D311F8014B03F880
:10FFB000014B14B930BD2B46F1E7002AF2D11A707B
:10FFC000F0E710B56AB10139841810F8013B11F857
:10FFD000012F934203D1A04201D0002BF5D1981AF2
:10FFE00010BD1046FCE770B50139044602B970BD7A
:10FFF000234611F8015F03F8015B561E2DB9144426
:020000021000EC
:10000000A342F4D003F8015BFAE71C463246EDE761
:1000100010B5034601448B4202D01A785C1C0AB921
:10002000181A10BD2346F6E738B503460D4669B9E0
:10003000BDE83840FFF76EBF431C0446294618460A
:10004000FFF768FF0028F7D1204638BD0024F5E708
:10005000134B2DE9F0411D68AC6D06460F46B4B94F
:100060005020FEF7ABFFA865C0E90044C0E9024498
:10007000C0E90444C0E90A44C0E90C44C0E90E44A4
:10008000C0E91044C0E91244846104774462AA6D57
:10009000394630460123BDE8F04100F003B800BF07
:1000A00038000020F0B518B9106808B9F0BD204636
:1000B00004460F4614F8015B17F8016B1EB96DB9C1
:1000C00015602846F2E7B542F6D1002BEFD1146057
:1000D0000370EBE72B460DE026B91C4623460F467E
:1000E00013F8015B17F8016BB542F5D1002DF1D083
:1000F000002121701360D9E72DE9F0478046894639
:1001000092461E460F463D46089815F8014BFEF7ED
:1001100044FF2044437813F0080332D12D2C32D110
:100120007C78BD1C0122002E5DD0102E09D1302C10
:1001300007D12B7803F0DF03582B4FD16C781026B2
:100140000235002A14BF4FF000416FF00041002734
:10015000B1FBF6FC384606FB1C1EA4F13003092B4C
:1001600017D81C46A64223DD7B1C07D084451CD330
:1001700001D1A64519DB00FB0640012715F8014B0C
:10018000EBE72F46BFE72B2C04BFBD1C7C781A463B
:10019000C9E7A4F14103192B01D8373CE2E7A4F1E8
:1001A0006103192B04D8573CDCE74FF0FF37E5E734
:1001B0007B1C08D12223C8F800300846BAF1000F92
:1001C00007D1BDE8F08702B14042BAF1000FF8D084
:1001D0000FB105F1FF39CAF80090F2E73024002E84
:1001E000AFD10826ADE7302CA3D00A26A9E700003E
:1001F00037B5064C064D2468246A002C08BF2C46EF
:100200000094FFF779FF03B030BD00BF3800002035
:100210009C000020084B37B51C68084D236A002B52
:1002200008BF2B46009313460A4601462046FFF7B7
:1002300063FF03B030BD00BF380000209C000020E9
:100240002DE9F0478046894692461E460F463D46B8
:10025000089815F8014BFEF7A0FE2044437813F0F0
:10026000080330D12D2C30D17C78BD1C0121002E0B
:100270005CD0102E09D1302C07D12B7803F0DF038E
:10028000582B4ED16C78102602354FF0FF320023E8
:10029000B2FBF6F206FB02FC6FEA0C0C1846A4F166
:1002A0003007092F17D83C46A64223DD002B1EDB62
:1002B00082421CD301D1A44519DB00FB0640012377
:1002C00015F8014BEBE72F46C1E72B2C04BFBD1CF3
:1002D0007C781946CBE7A4F14107192F01D8373CA8
:1002E000E2E7A4F16107192F04D8573CDCE74FF08F
:1002F000FF33E5E7002B09DA2223C8F800304FF07E
:10030000FF30BAF1000F07D1BDE8F08701B14042DC
:10031000BAF1000FF8D00BB105F1FF39CAF800901F
:10032000F2E73024002EB0D10826AEE7302CA4D05E
:100330000A26AAE737B5064C064D2468246A002C25
:1003400008BF2C460094FFF77BFF03B030BD00BF11
:10035000380000209C000020024B01461868FFF77F
:10036000F9BC00BF3800002010B50446FEF718FEA7
:100370002044437803F00303022B08BF203C2046AF
:1003800010BD0000F0B51D4B8BB005460C466E4607
:1003900003F1200C18685968374603C708336345D2
:1003A0003E46F7D118681B793B71931E222B3860AB
:1003B0004FF0000304D923701C4620460BB0F0BD5B
:1003C000661EB5FBF2F00AAF02FB10553D44591C06
:1003D00015F8285C06F8015F054668B960542344A7
:1003E0002246191B101B8142E7DD1178187802F8AC
:1003F000010B03F80119F4E70B46E2E7613C010049
:10040000F8B50E461446054618B183690BB9FEF7D8
:10041000E1FC214B9C422AD16C68A369A360A389AB
:100420001A072ED5236963B323692068C01A63694C
:10043000F6B28342374604DC21462846FEF74EFCDE
:1004400028BBA368013BA36023685A1C22601E706E
:1004500063690130834204D0A389DB0719D50A2ED2
:1004600017D121462846FEF739FC90B10FE00B4B1F
:100470009C4201D1AC68D0E7094B9C4208BFEC68B4
:10048000CBE72146284600F02DF80028CCD04FF0CD
:10049000FF373846F8BD00BFDC3B0100FC3B0100E4
:1004A000BC3B010049B1FF2A85BF8A2303600A7063
:1004B0004FF0FF3098BF012070470846704700009A
:1004C00038B5074C054608461146002222601A46F8
:1004D00002F044F8431C02D1236803B12B6038BDFD
:1004E00050080020324B70B51D6806460C4625B1F9
:1004F000AB6913B92846FEF76DFC2E4B9C420FD119
:100500006C68B4F90C309AB215072CD4D00611D40B
:100510000922326043F04003A3814FF0FF303EE0F8
:10052000254B9C4201D1AC68EBE7244B9C4208BFB1
:10053000EC68E6E7510712D5616B41B104F1440361
:10054000994202D03046FEF797FD00236363A389EA
:1005500023F02403A3810023636023692360A3891C
:1005600043F00803A38123694BB9A38903F42073E3
:10057000B3F5007F03D02146304600F0C3FEA289C8
:1005800012F001030CD00023A36063695B42A361F6
:10059000236953B9B4F90C3013F08000BAD170BD9F
:1005A000920758BF6369A360F2E70020F7E700BF36
:1005B00038000020DC3B0100FC3B0100BC3B01009B
:1005C00008B5062001F004FF012001F0CFFF000074
:1005D00038B5064C002305460846236001F078FF35
:1005E000431C02D1236803B12B6038BD50080020A2
:1005F0002DE9F74F03690C69A3428046C0F282805F
:10060000013C01F114074FEA840C00F1140657F87D
:10061000245056F8240006EB0C03013507EB0C09B7
:100620000193B0FBF5F595B34FF0000A3846B64696
:10063000D34650F8042B93B205FB03A34FEA134AA9
:100640009BB2ABEB0303120CDEF800B005FB02A279
:1006500013FA8BF34FEA124A1FFA82FBDEF80020EE
:10066000CBEB124202EB23429BB243EA02438145A9
:100670004FEA224B4EF8043BDBD256F80C3033B92C
:10068000019B043B9E421A4630D3C8F810404046B6
:1006900001F0E6F8002825DB013530464FF0000C6C
:1006A00057F8042BD0F800E093B2ACEB0303120C24
:1006B00013FA8EF3C2EB1E4202EB23429BB243EAD3
:1006C0000243B9454FEA224C40F8043BE8D256F8C1
:1006D000242006EB84032AB9043B9E421A460BD31E
:1006E000C8F81040284603B0BDE8F08F1268043BFC
:1006F000002ACAD1013CC5E71268043B002AEFD1A9
:10070000013CEAE70020EEE72DE9F04F456A95B09D
:1007100016461F460446DDF88480CDE902673DB9E0
:100720001020FEF74BFC6062C0E901550560C56012
:10073000636A196851B15A684A60012393408B601B
:10074000204600F0ABFE636A00221A603B1EBBBF6E
:1007500023F00043039300230122ACBFC8F800300C
:10076000C8F80020AE4BDDF80C8033EA08031BD13B
:10077000209A42F20F731360029B23B9C8F313004F
:10078000002800F04B85229B53B9A64B21E0A64BD5
:1007900006930833229A1360069815B0BDE8F08FCF
:1007A000A04B06930333F5E7DDE90267002200233F
:1007B00030463946FEF7E2F8824660B1209A0123BE
:1007C0001360229B002B00F02685984B229A136021
:1007D000013B0693E0E712AB019313AB0093324663
:1007E0003B46204601F0B3F8C8F30A558346002D76
:1007F0007CD0C7F3130343F07F59B04649F4401946
:10080000A5F2FF35CDF840A00022894B404649466D
:10081000FDF794FC7CA3D3E90023FDF747FE7CA3FE
:10082000D3E90023FDF78CFC064628460F46FDF76A
:10083000D3FD79A3D3E90023FDF738FE02460B462A
:1008400030463946FDF77CFC06460F46FEF7DEF8DB
:1008500000228246002330463946FEF799F848B117
:100860005046FDF7B9FD32463B46FEF787F808B91A
:100870000AF1FF3ABAF1160F59D86E4901EBCA01D5
:10088000DDE90223D1E90001FEF7A0F8002850D0ED
:100890000AF1FF3A00230D93129B5D1B6B1E079319
:1008A00043BF0023C5F1010907934FF00009BAF1D6
:1008B000000F40DB079BCDF830A053440793002383
:1008C00008931E9B092B00F28E80052BC4BF043BAE
:1008D0001E931E9BA3F10203CCBF00250125032B11
:1008E00000F28D80DFE803F07B7D2F6FDDE912538E
:1008F0001D4405F23240202813DDC0F14000029B68
:1009000008FA00F805F2124023FA00F048EA000065
:10091000FDF752FD01238046A1F1F879013D1093C6
:1009200072E7029BC0F1200003FA00F0F0E7012318
:10093000B1E70D90B0E7CAF1000308930023A9EBDB
:100940000A090C93BDE7012309931F9B002B75DD5A
:1009500004939846666A00227260042202F1140031
:10096000984271686FD9204600F064FD636A306078
:100970001B680693B8F10E0F00F2EE80002D00F018
:10098000EB80DDE90223BAF1000FCDE90E2378DD1B
:10099000284A0AF00F0302EBC303D3E900234FEA0E
:1009A0002A16F006CDE90A2369D5234BDDE90E01AD
:1009B000D3E90823FDF7A4FECDE9020106F00F06F6
:1009C00003251D4F50E0012309931F9B534403F15E
:1009D000010804934346012BB8BF0123BAE7002363
:1009E000B2E70023F0E7012500231E9309954FF09D
:1009F000FF3304939846002212231F92AAE7012393
:100A00000993F4E7AFF3008061436F63A787D23F98
:100A1000B3C8608B288AC63FFB799F501344D33FED
:100A20000000F07F903D0100873D01006D3901001D
:100A30000000F83FC03D0100983D010001230493F0
:100A400098461A46D9E701317160520086E7F107EE
:100A500008D5DDE90A01D7E90023FDF727FDCDE937
:100A60000A01013576100837002EF0D1DDE90A239E
:100A7000DDE90201FDF744FECDE902011BE002259C
:100A80009FE700F0A480CAF10006A24BA24F06F037
:100A90000F0203EBC203D3E90023DDE90E01FDF7EA
:100AA00005FDCDE90201361100230225002E40F09C
:100AB0008380002BE0D10D9B002B00F08A80DDE9C4
:100AC0000223CDE90A23DDE90A010022934BFDF759
:100AD0005FFF00287DD0B8F1000F7AD0049B002B77
:100AE00036DD00228E4BDDE90A01FDF7DFFCCDE9A2
:100AF0000201049E0AF1FF3701352846FDF76CFC20
:100B0000DDE90223FDF7D2FC0022864BFDF718FB3E
:100B1000A1F15075CDE90A010B95002E5CD10022A0
:100B2000814BDDE90201FDF709FB0A9A2B46CDE96D
:100B30000201FDF74BFF002840F084820A9A05F17C
:100B40000043DDE90201FDF723FF002840F0788231
:100B5000DDE90E23CDE90223139B002BC0F24E8169
:100B6000BAF10E0F00F34A816A4B03EBCA03D3E9D3
:100B70000023CDE904231F9B002B80F2D980B8F11C
:100B8000000F00F3D58040F05A820022664BDDE969
:100B90000401FDF78BFCDDE90223FDF70DFF46465E
:100BA0004746002840F03082069B069A5D1C3123A0
:100BB00013700AF1010A2BE2F20705D5D7E90023E9
:100BC000FDF774FC01350123761008376EE7022526
:100BD00071E75746464690E74E4B03EBC60353E991
:100BE0000201099B002B48D002460B4600204F49CA
:100BF000FDF786FDDDE90A23FDF7A0FACDE90A013C
:100C0000069DDDE90201FDF701FF1190FDF7E4FB10
:100C100002460B46DDE90201FDF790FA119B3033E5
:100C200005F8013BDDE90A23CDE90201FDF7B0FE3D
:100C3000002864D1DDE9022300203849FDF77EFA5F
:100C4000DDE90A23FDF7A4FE002840F0B780069BEB
:100C5000EB1A9E427FF77CAF0022314BDDE90A019F
:100C6000FDF724FC0022CDE90A012D4BDDE902014C
:100C7000FDF71CFCCDE90201C3E7DDE90A23FDF71E
:100C800015FC069BCDE90A019D191E46DDE902010E
:100C9000FDF7BCFE1190FDF79FFB02460B46DDE918
:100CA0000201FDF74BFA119B303306F8013BAE42CF
:100CB000CDE902014FF0000225D11C4BDDE90A010C
:100CC000FDF73EFA02460B46DDE90201FDF77EFE26
:100CD000002873D1DDE90A2300201449FDF72EFA1C
:100CE00002460B46DDE90201FDF752FE00283FF403
:100CF0002FAF15F8013C302B05F1FF3201D0BA4679
:100D00004BE01546F5E7064BFDF7D0FBCDE90201B8
:100D1000BCE700BFC03D0100983D01000000F03F6E
:100D20000000244000001C40000014400000E03F90
:100D3000DDE90267069DDDE9042330463946FDF70B
:100D4000DFFCFDF763FE8146FDF746FBDDE904238A
:100D5000FDF7ACFB02460B463046394609F130063A
:100D6000FDF7ECF905F8016B069EAE1BB045024697
:100D70000B4636D1FDF7E4F9DDE9042306460F46BC
:100D8000FDF724FEC8B9DDE9042330463946FDF7F6
:100D9000F5FD10B119F0010F0FD15946204600F0B2
:100DA0007DFB0023209A2B700AF101031360229B24
:100DB000002B3FF4F1AC1D60EEE4574615F8012C12
:100DC000392A05F1FF3306D1069A9A4207D130231A
:100DD0001370013713461A7801321A708FE71D46D7
:100DE000ECE70022994BFDF761FB00220023064649
:100DF0000F46FDF7C3FD00289DD0CEE7099A002AD3
:100E000000F088801E9A012A6DDC109A002A66D0B4
:100E100003F23343089E4D46079A01211A442046A7
:100E20009944079200F0DAFB0746002D0BDD079B83
:100E3000002B08DDAB42079AA8BF2B46A9EB03099C
:100E4000ED1AD31A0793089BEBB1099B002B65D0D1
:100E50008EB139463246204600F060FC5A460146C3
:100E60000746204600F0C3FB59460A90204600F092
:100E700015FB0A9B9B46089B9A1B04D059462046AB
:100E800000F04CFC83460121204600F0A7FB0C9BA0
:100E90000646002B00F0C9811A460146204600F0A4
:100EA0003DFC1E9B012B06463EDC029B002B37D1EE
:100EB000039BC3F31303002B34D1039B23F00043A4
:100EC0001B0D1B052BB1079B0133079309F101098A
:100ED000012308930C9B002B28D101202EE0129BAC
:100EE000C3F1360396E7089B08F1FF36B342BFBF54
:100EF000089B0896F21A0C9BB7BF9B189E1B0C937D
:100F00000026B8F1000FB9BFA9EB080500234D4634
:100F1000434681E7089E099F4D4686E7089AADE75C
:100F20000023D6E7029BD4E700230893336906EB3E
:100F30008303186900F004FBC0F12000079B1844EC
:100F400010F01F0047D0C0F12003042B3BDD079BAE
:100F5000C0F11C008144054403440793B9F1000F1C
:100F600005DD59464A46204600F026FC8346079B8D
:100F7000002B05DD31461A46204600F01DFC0646D2
:100F80000D9B53B33146584600F06AFC002824DA22
:100F9000002359460A22204600F097FA099B0AF1DD
:100FA000FF3A8346002B00F04781002339460A228E
:100FB000204600F08AFA049B002B07464EDC1E9B5D
:100FC000022B4BDD11E0C9D0079A1C331A44994417
:100FD0001D441346C1E70346F6E7B8F1000F37DCBE
:100FE0001E9B022B34DDCDF81080049B63B9314683
:100FF0000522204600F069FA01460646584600F0F0
:101000002FFC00283FF7D0AD1F9B069D6FEA030A17
:101010004FF000093146204600F040FA002F3FF41F
:10102000BCAEB9F1000F05D0B94503D04946204602
:1010300000F034FA3946204600F030FAADE60026DA
:101040003746E1E7BA463746AEE500BF0000244028
:10105000099BCDF81080002B00F0F580002D05DDF8
:1010600039462A46204600F0A7FB0746089B002B7E
:101070004CD07968204600F0DDF93A690232054625
:10108000920007F10C010C30FDF7C9FF012229463F
:10109000204600F091FB069B0793029B03F001039F
:1010A000B9460893074631465846FFF7A1FA494624
:1010B000054600F13008584600F0D2FB3A4602904F
:1010C0003146204600F0E6FBC368024603BB0146FA
:1010D0000990584600F0C4FB099A03461146204681
:1010E000099300F0DBF9099BA3B91E9A92B9089AFB
:1010F00082B9B8F1390F29D0029B002B01DD05F12F
:101100003108079B5D1C83F8008083E73846C2E7FF
:101110000123E3E7029A002A04DB24D11E9A12BBC2
:10112000089A02BB002BECDD59460122204600F054
:1011300043FB3146834600F093FB002803DCE0D1FB
:1011400018F0010FDDD0B8F1390FD8D1079B079AFD
:101150005D1C3923137015F8013C392B05F1FF3262
:101160004ED0013353E0079A002B02F1010506DD52
:10117000B8F1390FEAD008F10108079BC3E7069BD5
:10118000049A05F8018CEB1A934221D059460023AA
:101190000A22204600F099F9B94583464FF0000332
:1011A0004FF00A024946204605D100F08EF98146EB
:1011B0000746079577E700F088F93946814600230E
:1011C0000A22204600F081F90746F2E74FF00009B5
:1011D00059460122204600F0EFFA3146834600F0DE
:1011E0003FFB0028B7DC02D118F0010FB3D115F88E
:1011F000013C302B05F1FF327FF40CAF1546F6E7CA
:10120000069B934205D1069A0AF1010A3123137015
:1012100000E715469FE7174BFFF7DBBA229B002B31
:101220007FF4B5AA144BFFF7D4BA1E9B012B7FF7AE
:101230003CAE0C9B089350E6049B002B03DC1E9BEA
:10124000022B3FF7D2AE069D31465846FFF7D0F944
:1012500000F1300805F8018B069B049AEB1A9A42BC
:10126000B4DD594600230A22204600F02EF98346B9
:10127000EAE700BF6C390100873D0100044B1B68A1
:10128000186A044B002808BF1846F030704700BFAA
:10129000380000209C00002038B5074C0546084661
:1012A0001146002222601A4601F03AF9431C02D18D
:1012B000236803B12B6038BD5008002070B50E467E
:1012C000B1F90E10002996B014461D4607DA002326
:1012D0002B60B3891A0610D44FF480630EE06A467F
:1012E00001F0CCF80028F2DB019A02F47042A2F57A
:1012F00000535A425A412A60EEE7402300202360FF
:1013000016B070BD8B8973B59D0706460C4607D590
:1013100004F14703236023610123636102B070BDC0
:1013200001AB6A46FFF7CAFF009905463046FDF754
:10133000F1FE48B9B4F90C309A05EFD423F0030359
:1013400043F00203A381E3E70D4BB362A38920605E
:1013500043F08003A381009B6361019B20615BB12B
:10136000B4F90E10304601F09BF828B1A38923F0A0
:10137000030343F00103A381A3891D43A581CDE7A6
:101380009DED0000000000000000000000000000D3
:1013900001F0FF01102A2BDB10F0070F08D010F826
:1013A000013B013A8B422DD010F0070F42B3F6D12A
:1013B000F0B441EA012141EA014122F007047FF043
:1013C00000070023F0E80256083C85EA010586EA9A
:1013D000010685FA47F5A3FA87F586FA47F6A5FAD6
:1013E00087F68EB9EED1F0BC01F0FF0102F00702E2
:1013F00032B110F8013B013A83EA010313B1F8D18D
:101400000020704701387047002D06BF354603386D
:10141000073815F0010F07D1013015F4807F02BFA6
:10142000013015F4C03F0130F0BC0138704700BFF7
:101430007047704770B5456A04460E463DB91020A6
:10144000FDF7BCFD6062C0E901550560C560656AD5
:10145000EB6883B1636ADB6853F82600B8B90121F1
:1014600001FA06F56A1D9200204600F0BFFA60B14D
:10147000C0E901650EE021220421204600F0B6FA01
:10148000636AE860DB68002BE4D1002070BD02686D
:1014900043F826200023C0E90333F7E770B5446A18
:1014A00006460D463CB91020FDF788FD7062C0E984
:1014B00001440460C4603DB1736A6A68DB6853F834
:1014C0002210296043F8225070BD2DE9F0410D69CA
:1014D0001F4606460C4601F1140C0023DCF8000000
:1014E00081B202FB01710F0C000C02FB007089B28B
:1014F000013301EB00419D424FEA10474CF8041BB9
:10150000ECDCD7B1A368AB4212DC61683046013134
:10151000FFF790FF2269023204F10C01804692002D
:101520000C30FDF77CFD21463046FFF7B7FF4446FF
:1015300004EB850301355F6125612046BDE8F0813C
:10154000020C12040346B2B90304102013F07F4FBB
:1015500004BF1B02083013F0704F04BF1B0104309E
:1015600013F0404F04BF9B000230002B06DB5B00F2
:1015700003D5013070470020E8E72020704703685A
:1015800013F0070201460BD0DA0723D4980749BFAE
:101590005B089B0801200B605CBF0B60022070475A
:1015A00098B2A8B91B0C102013F0FF0F04BF1B0A40
:1015B00008301A0704BF1B0904309A0704BF9B08B0
:1015C0000230DA0702D45B0806D001300B607047A6
:1015D0001046E9E7002070472020704710B50C4600
:1015E0000121FFF727FF01224461026110BD2DE9AF
:1015F000F74F14460A6923699A42B8BF0B468846DA
:10160000BCBFA0461C46D8F81070D4F81090D8F88B
:101610000830D8F8041007EB0906B342B8BF01310F
:10162000FFF708FF00F1140505EB860E2B4600229C
:10163000734516D304F1140208F1140102EB890377
:1016400001EB87070093009B019293420CD8002E78
:1016500003DD5EF8043D002B5DD0066103B0BDE8FC
:10166000F08F43F8042BE3E7B2F800B0BBF1000FB2
:1016700023D08946AC464FF0000859F8044BDCF8FB
:1016800000A0A3B21FFA8AFA0BFB03A34FEA144A85
:10169000DCF8004043444FEA14480BFB0A8404EB97
:1016A0001344E2469BB243EA04434F454FEA1448D1
:1016B0004AF8043B2BD8CCF80480019BB3F802A075
:1016C0000432BAF1000F20D02B688946A8464FF0AB
:1016D000000BB9F800C0B8F802400AFB0C445C44A7
:1016E000C4469BB243EA04434CF8043B59F8043B1C
:1016F000B8F804B01B0C0AFB03B303EB14434F45CB
:101700004FEA134B05D8C8F8043004359BE7D4469C
:10171000B3E7E046DDE7013E99E700002DE9F84335
:10172000154612F0030206460F4607D0013A214C37
:10173000002354F82220FFF7C8FE0746AD1035D02D
:10174000746A3CB91020FDF739FC7062C0E90144AD
:101750000460C460D6F82480D8F808404CB940F240
:1017600071213046FFF73AFF0023C8F8080004460D
:1017700003604FF00008EB070AD539462246304691
:10178000FFF735FF394681463046FFF787FE4F4663
:101790006D100BD0206838B9224621463046FFF73D
:1017A00026FF2060C0F800800446E4E73846BDE824
:1017B000F88300BF883E01002DE9F0470C464FEA50
:1017C000621A236949680AEB0309A36807461646AB
:1017D00009F10105AB4232DB3846FFF72BFE00234F
:1017E000804600F114011A4653452BDB20692AEA92
:1017F000EA7A04F1140316F01F0201EB8A0103EBED
:10180000800C25D0C2F1200E00201E688A4696402A
:1018100030434AF8040B53F8040B9C4520FA0EF0B1
:1018200014D8486008B109F10205013D3846C8F8EE
:1018300010502146FFF732FE4046BDE8F0870131E7
:101840005B00C7E741F823200133CDE75146DCE7D1
:10185000043953F8042B41F8042F9C45F9D8E4E7E8
:1018600003690A699B1A30B50CD192001430143107
:101870008418114454F8045D51F8042D954203D0A6
:1018800005D30123184630BDA042F3D3FAE74FF049
:10189000FF33F7E72DE9F0470D4607461146284686
:1018A0001446FFF7DDFF061E08D131463846FFF724
:1018B000C1FD0123C0E90436BDE8F087A4BF23467B
:1018C0002C4638466168A6BF1D4600260126FFF754
:1018D000B1FD2B69C660266905F1140904F11402F3
:1018E00002EB860709EB830800F114054FF0000EA8
:1018F00052F804AB59F8044B1EFA8AF1A3B2C91A84
:10190000230CC3EB1A4303EB214389B24FEA234E66
:10191000C84541EA0343944645F8043BE8D8BC4532
:1019200004D355F8043D83B10661C5E75CF8041B98
:101930001EFA81F31A1402EB11429BB243EA0243EE
:101940004FEA224E45F8043BE9E7013EE9E72DE97D
:10195000F34101211C469046DDE90865FFF76AFD69
:10196000C4F31302C4F30A54074634BB0192B8F11E
:10197000000227D002A840F8082DFFF700FE0099CA
:10198000F0B1019AC0F1200302FA03F30B43C24005
:101990007B610192019BBB61002B14BF02210121DD
:1019A0003961C4B1A4F2334404443460C0F1350059
:1019B0002860384602B0BDE8F08142F48012D5E7D5
:1019C0007961E7E701A8FFF7DAFD019B7B6101215F
:1019D00039612030E5E707EB8103A0F23240306047
:1019E0001869FFF7ADFDC0EB4110E1E738B502FB28
:1019F00001F42146FDF78EFB054618B12246002171
:101A0000FDF731FB284638BDF8B5074614460E46AB
:101A100021B91146BDE8F840FDF77CBB22B9FDF7BE
:101A20002BFB25462846F8BD00F04AFDA0420FD208
:101A300021463846FDF76EFB05460028F2D03146B8
:101A40002246FDF7ECFA31463846FDF715FBE9E78B
:101A50003546E7E72DE9F0478E689E4282460C4600
:101A60009046994637D88A8912F4906F31D025680C
:101A700009696F1A6569022305EB450595FBF3F5C6
:101A800009F101033B449D4238BF1D46530530D543
:101A90002946FDF73FFB064650B90C23CAF8003033
:101AA000A38943F04003A3814FF0FF30BDE8F087E6
:101AB0003A462169FDF7B3FAA38923F4906343F012
:101AC0008003A381266165613E44ED1B2660A5600D
:101AD0004E464E4500D94E46324641462068FDF7F7
:101AE000A9FAA3689B1BA36023681E4426600020FC
:101AF000DCE72A46FFF788FF06460028E2D1216985
:101B00005046FDF7B9FAC8E72DE9F04F9DB0804681
:101B100003938B891D060C4616460FD50B696BB9CE
:101B20004021FDF7F7FA2060206128B90C23C8F89E
:101B300000304FF0FF30C7E040236361002309937A
:101B400020238DF8293030238DF82A304FF0010BF7
:101B500037463D4615F8013B0BB1252B3ED1B7EB7F
:101B6000060A0BD05346324621464046FFF772FF25
:101B7000013000F0A480099B534409933B78002B6B
:101B800000F09D8000234FF0FF32CDE90523049340
:101B900007938DF853301A932F46052217F8011B2F
:101BA0004F48FFF7F5FB049BD0B9D90644BF20226C
:101BB0008DF853201A0744BF2B228DF853202A7822
:101BC0002A2A15D0079A2F4600200A25394611F8EF
:101BD000013B303B092B4DD9B8B10FE02F46B8E798
:101BE0003F4A801A0BFA00F0184304903D46D3E7B1
:101BF000039A111D12680391002A01DB079204E089
:101C0000524243F00203079204933B782E2B0CD1EF
:101C10007B782A2B33D1039B1A1D1B680392002B60
:101C2000B8BF4FF0FF33023705932E4D39780322AA
:101C30002846FFF7ADFB38B14023401B03FA00F004
:101C4000049B034301370493397827488DF8281003
:101C500006227E1CFFF79CFB002838D0234B13BBC9
:101C6000039B073323F0070308330393099B4B447B
:101C700009936DE705FB023201200F46A6E700231A
:101C80000137059319460A25384610F8012B303ADA
:101C9000092A03D9002BC8D00591C6E705FB01210D
:101CA00001230746F0E703AB00932246104B04A93B
:101CB0004046FDF755FCB0F1FF3F8146D6D1A389E0
:101CC0005B063FF536AF09981DB0BDE8F08F03AB5A
:101CD00000932246064B04A94046FDF7EDFEEAE7D5
:101CE000263C01002C3C0100303C010061F5000065
:101CF000551A010038B54B1C144603D14FF0FF357F
:101D0000284638BD938923F020039381636B526882
:101D1000CDB28BB1A36B934208DD23685A1E2260BB
:101D200003F8015C636801336360E9E7214600F072
:101D30006BFB0028F1D0E1E72169236851B199429A
:101D400008D213F8011CA94204D1013B01322360DF
:101D50006260D5E7C4E90F3204F1440363630323EF
:101D6000A363234603F8465F23600123DCE710B535
:101D70000C46496B69B104F14403994201D0FDF767
:101D80007BF9236C63600020606313B1E36B236015
:101D900010BD2369236000236360A38943F02003FF
:101DA000A3814FF0FF30F3E72DE9F04FADF5257D2E
:101DB0000DF10C0801930023469347939E4BA29389
:101DC000DFF87C929D4BCDF8208106460C4692466A
:101DD000A3930A279AF80030002B00F02A81554679
:101DE000FDF7DEF815F801BB5844437813F00803FB
:101DF0001CD06368002B12DDFDF7D2F823681A7837
:101E000010444278120701D4AA46E3E7479A013208
:101E1000479262680133013A62602360E9E7A39B5D
:101E20002146304698470028E6D0EDE7BBF1250F64
:101E300040F08280459343939AF801302A2B03D1D6
:101E4000102343930AF10205AA4615F8011BA1F1DC
:101E50003002092A22D903227948FFF799FA38B1CA
:101E6000A0EB090301209840439B18434390AA46E6
:101E70009AF80030672B0AF101052BD8652B80F00A
:101E80009F80472B10D8452B80F09A80002B6CD078
:101E9000252B51D003234993449727E0459B07FB0B
:101EA0000313303B4593CFE75B2B6AD00CD8582BFC
:101EB000F0D1439A42F400724392102244926E2B66
:101EC0008CBF0423032310E0632B65D0642BE1D186
:101ED0004497F4E7702B4BD026D86E2B62D04CD8A9
:101EE000692BD7D100234493032349936368002BC4
